:0800000C322E352E302E323762
:1000000A718C9274B8AD936EB3BFC3A27DBD9B8051
:1000000A9EA183C3B09FA288ADB38BB5B98E9C98CD
:1000000A9598979F999E99E0D4C691E6D9E3C8A09E
:1000000AE0CBCFA4B3AFADAFAFB0B5B5B9B4B1B66D
:1000000AB8B8BABABBC0C0C4BFBCDFC1E3B4EAD98E
:0F00000ADCC2E7E7C5DFE3C81105F7C2F8E7EA94
:020000040800F2
:4080000098EC0020A5970308B7970308E9C60308BB970308BD970308BF9703080000000000000000000000000000000021830008C397030800000000E583000859840008BF
:40804000C9970308C9970308C9970308C9970308C9970308C9970308C9970308C9970308C9970308C9970308C9970308C9970308C9970308C9970308C9970308C997030850
:40808000C9970308C997030869300308C7350308DB360308C9970308C9970308C997030805970308119703081D970308AB960308B7960308C5960308D1960308D56003080D
:4080C000E5600308F5600308FF600308C9970308096A0308054103080F41030819410308C9970308C9970308C9970308299703083597030841970308F9960308C9970308A1
:40810000C9970308C9970308DB960308C9970308C9970308C9970308E7960308F1960308C9970308C9970308C9970308C9970308C9970308C9970308C997030881360308E3
:408140004F370308C5370308C9970308C9970308C9970308C9970308C9970308374103080961030819610308C9970308C9970308C9970308C9970308C997030800000000BC
:40818000C9970308C9970308414103084B410308C9970308C9970308136A0308C99703080000000000000000C997030800F002F800F073F80AA090E8000C82448344AAF1F6
:4081C0000107DA4501D100F068F8AFF2090EBAE80F0013F0010F18BFFB1A43F00103184770C6030090C603000A444FF0000C10F8013B13F0070408BF10F8014B1D1108BFAB
:4082000010F8015B641E05D010F8016B641E01F8016BF9D113F0080F1EBF10F8014BAD1C0C1B09D16D1E58BF01F801CBFAD505E014F8016B01F8016B6D1EF9D59142D6D37C
:40824000704700000023002400250026103A28BF78C1FBD8520728BF30C148BF0B607047632934F0E280732934F0E780002070471FB538F0DCFD9DE8030034F06BF833F007
:40828000E4FE34F0B9F904000020002137F000FF401C60601FBD10B510BD34F088F91146FFF7E6FF10F02BFF34F0B9F903B4FFF7F2FF03BC34F0EAF980F309887047EFF339
:4082C00009807047684680F3098804480078C00714BF0220032080F31488704794370408DFF818C0EFF305831B0618BF6047EFF31483DB0708BF604700DF704717F2030821
:40830000DFF818C0EFF305831B0618BF6047EFF31483DB0708BF604700DF70471DF40308EFF30980816911F8021C01B142E010B590E80F10E047BDE81040EFF3098C254B5B
:4083400093E80600914232D041B91EF0100F16D12149086820F00100086010E00CB41EF0100F06BF2CED108A0323012381F826302CE9F00FC1F82CC037F0E6FB0CBC1A60D5
:40838000D2F82CC0BCE8F00F92F8263013F0020F1ABFBCEC108A6FF0120E6FF0020E8CF3098813F0010F08BF704792F82500CCF80000704710B5094A1268914209D8084C02
:4083C00054F8214090E80F10A047EFF3098C8CE80F0010BD9007002034EF00E0D8C60308D8C6030810B537F063FABDE81040194B93E80600914208BF70470CB4EFF3098CD4
:408400001EF0100F06BF2CED108A0223002381F826302CE9F00FC1F82CC037F095FB0CBC1A60D2F82CC0BCE8F00F92F8263013F0020F1ABFBCEC108A6FF0120E6FF0020E78
:408440008CF3098813F0010F1CBF92F82530CCF8003070479007002010B537F045FCC4E710B536F0D7FE37F03FFCBEE70B49D1F800C04A685CF8043B1068184442F8040BDF
:408480008C4528BFA1F1DC0C8A4228BFA1F1DC02C1F800C04A6020F00040704790E600200146F948B0F8AA0000EE100AB8EE400A81ED080AF44890ED800A81ED010A90ED1C
:4084C000810A81ED020A90ED820A81ED030A90F8AF0000EE100AB8EE400A81ED050AEA4890F8AE000877E84890ED7D0A81ED000A90F8B00000EE100AB8EE400A81ED060A06
:40850000B7EE000A81ED040A012070474FF6FF76DFF878C300DF074639460120DFF870C300DF0421DB4880F8D01100BF002231460120DFF864C300DF0446012C17D100BFA2
:40854000D44890F8D10140F00101D24880F8D111B0F8DC014FF6FF71884207DACD48B0F8DC01401C81B2CB48A0F8DC11DEE7022CDCD1DFF828C300DF054605F0010000288F
:40858000D4D0C748FFF78CFFD0E7C54880ED0C0ADFEDC40AC0ED0D0ADFEDC20AC0ED0F0ADFEDC00AC0ED0E0A80ED0A0A704710B52DED0C8BB0EE409AB0EE608AF0EE419AC2
:4085C0009FEDB80AF0EE408A2022B549243101F1200033F0DAFD9FEDB40AC9EE000AB048C0ED090AB5EEC08AF1EE10FA04D1B0EE480AFFF7CAFF10E1B5EEC08AF1EE10FA00
:4086000007DDA74890ED120AB5EEC00AF1EE10FA0CD9B5EEC08AF1EE10FA0FD2A04890ED120AB5EEC00AF1EE10FA07DBB0EE480AFFF7ABFF2EF0ABFA99498866984A92ED9F
:40864000080ABCEEC00A10EE101A906E2EF0A5FA50BBB5EEC08AF1EE10FA0ADD9FED930A8F4880ED0A0A9FED8F0A914880ED000A11E09FED900A8A4880ED0A0AD0ED050A9D
:40868000B7EE001A81EE200AF0EE000A80EE201A874880ED001A824890ED0A0A80ED0C0A012085490870B8E09FED800AB4EEC08AF1EE10FA07DB9FED810A794880ED0A0A79
:4086C000F0EE488A80E09FED7B0AB4EEC08AF1EE10FA07D89FED7A0A714880ED0A0AF0EE488A71E0724890ED000A30EE290A80ED000A6B4890ED050ADFED720A20EE200A92
:408700006B48D0ED000A20EE200A10EE101A084638F01CFB41EC1D0BB0EE4D0AF0EE6D0A35F0AEFDB0EE40BAF0EE60BA5C4890ED060A10EE101A084638F008FB41EC1C0BAD
:4087400053EC1B2B38F00CF841EC1A0B37F0C2FC08EE900AF5EEC08AF1EE10FA05DD504890ED060AF0EE408A06E04D4890ED060AB1EE400AF0EE408A38EE880AF0EE408AC3
:40878000B5EEC08AF1EE10FA09DDF5EEC08AF1EE10FA04D89FED4C0AF0EE408A0DE0B5EEC08AF1EE10FA08D2F5EEC08AF1EE10FA03DB9FED460AF0EE408A394890ED000A64
:4087C00020EE280A80ED0A0A3B48007870B13448C0ED0C8A90ED0A0AD0ED090A30EE600A80ED0D0A00203449087016E09FED2D0A2B49243101F1200014F0B6FA284934313D
:40880000A1F1300014F044F9F0EE408A244890ED0C0A30EE280A80ED0C0A214890ED0A0AB5EEC00AF1EE10FA0BDD90ED0C0AB5EEC00AF1EE10FA04D29FED1A0A80ED0C0A91
:4088400054E0174890ED0A0AB5EEC00AF1EE10FA0BD290ED0C0AB5EEC00AF1EE10FA04DD9FED100A80ED0C0A40E00D4890ED0C0ADFED0E0AB4EEE00AF1EE10FA28DD9FEDBC
:408880000B0A80ED0C0A31E0081F0020C1FF030881F30308F03F0020E1F3030829F30308EC1400200000000000007A440000C842440300200000C8C24003002066662640BB
:4088C000666626C0DB0FC9400AD7233C0AD723BCF64890ED0C0A5FED090AB4EEE00AF1EE10FA03D21FED0D0A80ED0C0AEF4890ED0C0ABDEC0C8B10BD01B500BF0122694695
:40890000EB480068B03010F0AFFE20B99DF80000E84981F8B00000BFE748D0F8CC110120DFF898C300DF08BD10B52DED020B00BF04226946DE48006800F5FA7010F094FEBE
:4089400020B99DED000ADB4880ED7D0A00BFDA48D0F8CC110120DFF864C300DF1CBD01B500BF01226946D2480068AE3010F07CFE20B99DF80000CF4981F8AE0000BFCE4873
:40898000D0F8CC110120DFF834C300DF08BD01B500BF01226946C6480068AF3010F064FE20B99DF80000C34981F8AF0000BFC248D0F8CC110120DFF804C300DF08BD10B549
:4089C0002DED020B00BF04226946B948006800F5027010F049FE20B99DED000AB54880ED820A00BFB448D0F8CC110120DFF8CCC200DF1CBD10B52DED020B00BF0422694624
:408A0000AB48006800F5017010F02EFE20B99DED000AA84880ED810A00BFA748D0F8CC110120DFF898C200DF1CBD10B52DED020B00BF042269469E48006800F5007010F064
:408A400013FE20B99DED000A9A4880ED800A00BF9948D0F8CC110120DFF860C200DF1CBD01B500BF0222694691480068AA3010F0FBFD20B9BDF800008E49A1F8AA0000BFC6
:408A80008D48D0F8CC110120DFF830C200DF2F2004F076FB08BD10B58AB00446022C1FD1B2EE040A8DED090A9FED850A8DED020A1FED840A8DED030A9FED810A8DED040AF7
:408AC0009FED800A8DED060A01208DF820009FED7E0A8DED010AB1EE080A8DED070AA6E0042C1FD1B3EE080A8DED090A1FED910A8DED020A1FED950A8DED030A1FED950A4B
:408B00008DED040A1FED970A8DED060A01208DF820009FED6E0A8DED010AB1EE040A8DED070A84E0052C1FD1B3EE080A8DED090A1FEDA20A8DED020A1FEDA60A8DED030AA9
:408B40009FED630A8DED040A9FED620A8DED060A01208DF820009FED600A8DED010AB1EE040A8DED070A62E00E2C1FD1B2EE040A8DED090A9FED520A8DED020A1FEDB70A97
:408B80008DED030A9FED520A8DED040A9FED4D0A8DED060A01208DF820009FED500A8DED010AB2EE040A8DED070A40E0152C1FD1B2EE040A8DED090A9FED460A8DED020AF9
:408BC0001FEDC80A8DED030A9FED420A8DED040A9FED3C0A8DED060A01208DF820009FED3A0A8DED010AB1EE080A8DED070A1EE01FEDD40A8DED090A1FEDD60A8DED020A16
:408C00001FEDD80A8DED030A1FEDDA0A8DED040A1FEDDC0A8DED060A00208DF820001FEDDF0A8DED010A1FEDE10A8DED070A9DED090ABDEEC00A10EE101A08B2FFF710FF11
:408C4000DDED020AB0EE600AFFF7EFFEDDED030AB0EE600AFFF7CEFEDDED040AB0EE600AFFF7ADFE9DED060ABCEEC00A10EE101AC8B2FFF78CFE9DF82000FFF770FEDDEDFE
:408C8000010AB0EE600AFFF74FFE9DED070ABCEEC00A10EE101AC8B2FFF72EFE2F2004F06FFA542004F06CFA0AB010BDEC140020A4030020081F0020F03F002081F303088E
:408CC000000048420000A042F3FDD43CA69B443C000048430000F042BC74933C96438B3C204890ED0A0ABDEEC00A10EE100A00B270471C4890ED090ABDEEC00A10EE100A7B
:408D000000B2704780220270164A92ED010ADFED160A20EE200ABCEEC00A10EE102A91B241700A0A82700F4A92ED020ADFED0E0A20EE200ABCEEC00A10EE102A91B2C170E2
:408D40000A0A0271074A92ED030ADFED070A20EE200ABCEEC00A10EE102A91B241710A0A82717047EC1400200000C84270B5054601249048DFF840C200DF204670BD8F4961
:408D8000097801708E49416001218160002181764176704700B5A1B06846FFF7F0FF01208DF8180006219DF81920501CC0B28DF819000DF14B00815400208DF8190068466E
:408DC00001992DF0B5FB002021B000BD00B5A1B06846FFF7D4FF02208DF8180005219DF81920501CC0B28DF819000DF14B00815400208DF81900684601992DF099FB9DF848
:408E00001800401E0DF11B01085C21B000BD2DE9F74F814615464FF000081FFA89F7E8191FFA80FBBBF5005F02DD4FF0080854E02D2D02DD4FF040084FE04FF47A615D489A
:408E4000DFF880C100DF012802D14FF0100844E0842032F096FF044654B3FFF79BFFFFF7B5FF82462046FFF78AFFE81C20760221627E501C607604F14B008154390A627EDA
:408E8000501C607604F14B008154627E501C607604F14B008754627E014650182A46019933F02EF900206076204661682DF040FB94F8800001280BD1FFF788FF06460AF0EA
:408EC000020010B106F0020020B14FF0800801E04FF02008204632F08FFF3648DFF8E8C000DFB8F1000F05D03848007840EA0800364908704046BDE8FE8F2DE9F043A1B0E5
:408F000080460F4614460026BDB260191FFA80F9B9F5005F01DD082642E02D2C01DD40263EE06846FFF72BFFE01CC0B28DF8180003219DF81920501CC0B28DF819000DF1E1
:408F40004B008154290A9DF81920501CC0B28DF819000DF14B0081549DF81920501CC0B28DF819000DF14B0085549DF81920014650185522214633F03AF900208DF819005B
:408F8000684601992DF0D4FA9DF88000012806D122460DF11E01404633F0B2F800E0202626B10A480078304308490870304621B0BDE8F0837444002055F70308C206002018
:408FC0000038004049F8030865F70308A103002088B0016807914168069181680591C1680491016903914169029181690191C169009108B070477047FFFFFFFFFFFFFFFF3C
:40900000FE4890ED0A0A704710B52DED048BB0EE408A0446F94890ED720ADFEDF90A80EE201AB0EE419AF74890F8AE0058B1FFF7E7FFF0EE409A9FEDF41AF0EE480AFFF786
:40904000B6FAB0EE408AEF4890F89C00012803D1B1EE480AB0EE408A9FEDEC0AB4EEC08AF1EE10FA04D29FEDE90AB0EE408A0AE09FEDE70AB4EEC08AF1EE10FA03DD9FED6B
:40908000E40AB0EE408A062C4DD008DC022C12D0032C12D0042C0DD0052C5ED10CE00E2C06D0122C40D0132C08D0152C55D100E000BF00BF00BF00BF00BF00BFB5EEC08A8A
:4090C000F1EE10FA0ED2B1EE480AB0EE408A0021D04800782BF0E0F90121CF4800782BF0DBF919E0B5EEC08AF1EE10FA0ADD0121C84800782BF0D0F90021C74800782BF002
:40910000CBF909E00021C34800782BF0C5F90021C14800782BF0C0F9B0EE480ABF4800782FF0FCFC1AE000BFF0EE000A89EE200A9FEDB71AC8EE010A60EE890AB1EE001A0F
:40914000C0EE811A70EE218ADFEDB50AB0EE680AB44800782BF01AFA00E000BF00BFBDEC048B10BD70B52DED048B04460D46AE48007848B1012020700121AC4880F82910B2
:409180002DF005FDA9490862207830B101283BD002284DD003286CD157E0A44890F8290001280ED1A148016A28462DF027FDFA2807D2012020709D4890ED090A84ED010A5C
:4091C00021E014F052FF30B10220207014F049FF84ED010A17E0954890F8410001280ED19248816B28462DF009FDFA2807D2032020708E4890ED0F0A84ED010A03E09FEDBD
:409200008C0A84ED010A37E0884890F8290030B18648016A28462DF0F1FCFA2802D90020207004E0814890ED090A84ED010A23E014F01BFF30B10220207014F012FF84ED52
:40924000010A01E00020207016E0784890F8410030B17648816B28462DF0D0FCFA2802D90020207004E0714890ED0F0A84ED010A02E00020207000BF00BF94ED020A84ED87
:40928000030A2078F0B394ED050AB5EEC00AF1EE10FA5AD094ED010A10EE101A084637F055FD41EC190BB0EE490AF0EE690A34F027F9B0EE408AF0EE608A9FED5E0B53ECA0
:4092C000102B51EC180B37F00FFA3ED894ED010AB5EEC00AF1EE10FA04D19FED550A84ED020A36E094ED010AD4ED050A30EE600AD4ED020AB4EEE00AF1EE10FA0ADD94EDCA
:40930000020A00E02EE0D4ED050A30EE200A84ED020A1EE094ED010AD4ED050A30EE200AD4ED020AB4EEE00AF1EE10FA08D294ED020AD4ED050A30EE600A84ED020A08E096
:4093400094ED010A84ED020A03E094ED010A84ED020A94ED020A84ED040A0120334981F8480013E09FED320A84ED020A9FED300A84ED010A9FED2E0A84ED030A9FED2C0A10
:4093800084ED040A0020294981F8480094ED040A264880ED110ABDEC048B70BD10B52DED088B044603F045FEB0EE408A94ED090AD4ED0B0A30EE200AF0EE000A80EE201A55
:4093C000F0EE418A94ED080AD4ED0A0A30EE200AF0EE000A80EE201AB0EE419A94ED020AB4EEE80AF1EE10FA4CDD94F8440002283ED1B2EE040A03F03AF81FE07408002061
:4094000000007A44081F00206F12833A0000C8C20000C842B5060020B60600201407002003005841DB0600202D000020C8070020000000000000000000005940A0B994ED17
:40944000120A38EE400AF0EE040AB4EEE00AF1EE10FA09D24FF47A71E06C2DF09EFB30B101215020015502E000215020015508E0022084F8440084ED128A2DF088FBE064A7
:4094800000BF56E094ED020AB4EEC90AF1EE10FA2BD294F8440001281DD1B2EE040A02F084FFA0B994ED120A38EE400AF8EE040AB4EEE00AF1EE10FA09DD4FF47A71E06C96
:4094C0002DF06BFB30B101215020015502E000215020015508E0012084F8440084ED128A2DF055FBE06400BF23E0002084F8440094ED120A30EE480A10EE101A084637F084
:4095000025FC41EC1B0BB0EE4B0AF0EE6B0A33F0F7FFB0EE40AAF0EE60AA9FEDF70B53EC102B51EC1A0B37F019FA02D2002150200155BDEC088B10BD70B52DED0C8B044660
:409540000D4694ED0A0AF2EE040AB4EEE00AF1EE10FA0CD294ED0A0AFAEE040AB4EEE00AF1EE10FA03DD1FED4E0A84ED0A0A94ED0A0A5FED5D0AC0EE208A95ED020AD5ED09
:40958000080AB4EEE00AF1EE10FA18D895ED0C0AD5ED020A20EE200A1FED631AC0EE010A94ED780A20EE800A1FED6B1AC0EE010A95ED0D0A30EEC00A84ED620A25E095ED8A
:4095C000020AD5ED090AB4EEE00AF1EE10FA18DB95ED0C0AD5ED020A60EE200A1FED741A80EE810AD4ED780A60EE200A1FED7C1A80EE810AD5ED0D0A30EE200A84ED620A5D
:4096000003E01FED750A84ED620A95ED020AB5EEC00AF1EE10FA02D11FED878A18E094ED620A10EE101A084637F090FB41EC1B0BB0EE4B0AF0EE6B0A33F062FFB0EE40AA59
:40964000F0EE60AA51EC1A0B36F044FD08EE100A94ED620A10EE101A084637F077FB41EC1D0BB0EE4D0AF0EE6D0A33F049FFB0EE40BAF0EE60BA18EE900A37F067FB41EC3D
:409680001D0BB0EE4D0AF0EE6D0A33F039FFB0EE40CAF0EE60CA53EC1B2B51EC1C0B37F06BFA41EC1A0B36F015FD09EE100A89EE080AB0EE409A1E219148B0EE490A1BF008
:4096C0005FFBBDEC0C8B70BD2DE9F0412DED028B04460D468B4890F8BD010A287DD14FF432700159001D0151001FD4F8C4120151854800782FF0E0F9C4F8C4024FF432701A
:409700000059D4F8C412081A00EE100AB8EEC00ADFED7E0A80EE201A84EDB41A94EDB40AB2EE041AC0EE010A9FED790A20EE800A84EDC40A95ED020AD5ED080AB4EEE00ACF
:40974000F1EE10FA23D895ED0E0AD5ED020A20EE200A1FEDD11AC0EE010A94ED780A20EE800A1FEDD91AC0EE010A95ED0F0A30EEC00A84EDDA0A94EDDA0AB5EEC00AF1EED9
:4097800010FA37DD1FEDD60A84EDDA0A32E095ED020AD5ED090AB4EEE00AF1EE10FA25DB95ED0E0AD5ED020A20EE200A1FEDE81AC0EE010A94ED780A20EE800A1FEDF01A48
:4097C000C0EE010A95ED0F0A30EE800A84EDDA0A94EDDA0AB5EEC00A00E07DE0F1EE10FA08D21FEDED0A84EDDA0A03E01FEDF00A84EDDA0A434890F830000A2803D132270E
:409800004FF0480802E032274FF04108D4EDC40AB0EE600A394604F53E701BF0B1FAD4EDDA0AB0EE600A414604F554701BF0A8FA94EDD40AD4EDBE0A30EE600AF2EE040A67
:4098400020EE208A9FED330AB4EEC08AF1EE10FA04DD9FED300AB0EE408A0AE09FED2E0AB4EEC08AF1EE10FA03D29FED2B0AB0EE408A012104F53970B0EE480A1BF080FAC9
:4098800094EDD40A84EDDD0A94EDBE0A84EDC70A04261AE0711E04F55D7000EB810090ED000A04F55D7000EB860080ED000A04F5477000EB810090ED000A04F5477000EB0E
:4098C000860080ED000A701EC6B2002EE2DC94EDB90A124880ED150ABDEC028BBDE8F081084991F84A10062904D0064991F84A10122915D1012014E0000000000000F83F2D
:40990000B4070020081F0020D80600208DED244800606A4700007A4400007AC4C80700200020704710B52DED020B00BF04226946FE48006800F558700FF096FE20B99DED6D
:40994000000AFB4880EDD80A00BF1CBD10B52DED020B00BF04226946F448006800F557700FF082FE20B99DED000AF14880EDD70A00BF1CBD10B52DED020B00BF0422694648
:40998000EA48006800F556700FF06EFE20B99DED000AE74880EDD60A00BF1CBD10B52DED020B00BF04226946E048006800F555700FF05AFE20B99DED000ADD4880EDD50A67
:4099C00000BF1CBDDA4991F84A10032901D1012000E00020704710B52DED020B00BF04226946D248006800F55C700FF03DFE20B99DED000ACE4880EDDC0A00BF1CBD10B5C3
:409A00002DED020B00BF04226946C848006800F55B700FF029FE20B99DED000AC44880EDDB0A00BF1CBD10B52DED020B00BF04226946BE48006800F55A700FF015FE20B912
:409A40009DED000ABA4880EDDA0A00BF1CBD10B52DED020B00BF04226946B448006800F559700FF001FE20B99DED000AB04880EDD90A00BF1CBDAE4991F84A10042918D08B
:409A8000AB4991F84A10022913D0A94991F84A1005290ED0A64991F84A100E2909D0A44991F84A10152904D0A14991F84A10132901D1012000E00020704710B52DED028BFD
:409AC00084B00446FFF77EFF10B1B2EE048A01E0B7EE008A964890ED280A20EE080A84ED000AB0F8A80000EE100AB8EE400A84ED020A9FED900A84ED010A8D4890F89C00EE
:409B000084F82C008A4890F842106C3000EB810090ED000A84ED030A854890F84210743000EB810090ED000A84ED040A804890F842107C3000EB810090ED000A84ED050A46
:409B40007B4890F84210843000EB810090ED000A84ED060A764890ED700A84ED070A90ED710A84ED080A90ED720A84ED090A90ED730A84ED0A0A2AF065FC002874D0FFF795
:409B8000AFFE78B301216C4800782AF085FC00216A4800782AF080FC0021694800782AF07BFCB2EE040AFFF7F9FE9FED660AFFF7E1FEB7EE000AFFF7C9FE9FED5E0AFFF766
:409BC000B1FE9FED610AFFF742FF9FED600AFFF72AFF9FED5F0AFFF712FF1FEDB20AFFF7FAFE96E0FFE7FFF746FFE0B35948009094ED020AF0EE400A9FED570A01231A4640
:409C00005649574800782EF05BFC00214A4800782AF042FC0121494800782AF03DFC0121474800782AF038FC9FED4E0AFFF7B6FE9FED460AFFF79EFE9FED450AFFF786FE30
:409C40001FEDCC0AFFF76EFE9FED470AFFF7FFFE9FED3E0AFFF7E7FE9FED3D0AFFF7CFFE1FEDD40A01E003E044E0FFF7B4FE50E0FFF7A8FE70B33748009094ED020AF0EEA8
:409C8000400A9FED350A01231A463449344800782EF016FC0021284800782AF0FDFB0121264800782AF0F8FB0121254800782AF0F3FB9FED2C0AFFF771FE9FED240AFFF754
:409CC00059FE9FED230AFFF741FE1FEDEE0AFFF729FE1EE00021184800782AF0DDFB0121164800782AF0D8FB0121154800782AF0D3FB0EE01748009094ED020AF0EE400ABF
:409D00009FED150A012300221849154800782EF0D7FB94F82C0068BB00200090019002900346032212490390552024E0A4030020081F002000000000F0060020120700202C
:409D4000110700206F12833A00401C45000048420000FA43A0D80020A037A04B0018004014070020000048450080544500000140260700200DE02AF066FC0020009001903A
:409D8000029003460322FE49039056202AF05BFC15E0002000900190029003460322F849039055202AF04FFC002000900190029003460322F349039056202AF044FC0120FD
:409DC00004B0BDEC028B10BD2DED028B5421EE4832F037FA4FF46771EC4832F032FA5821EB4832F02EFAE848EA490860E8484830E9490860E548E949086000F5F070E8491A
:409E00000860A0F5DC70E749086000F5B070E649086000F59E70E54908604C30E4490860DB485430E3490860E348E4490860D6481430E34908609FEDE30A143880ED030ABB
:409E40009FEDE00AD24880ED130A9FEDDF0A80ED140AFFF7B7FD40B1DFF870C300DF06460A2202212CF09DFF0AE02AF0EBFA38B1DFF858C300DF0646012202212CF091FF10
:409E8000DFF848C300DF064602212CF0B9FFDFF83CC300DF064631460120DFF834C300DF0321CC4880F8541000BF00224FF6FF710320DFF824C300DF044604F00100002887
:409EC000F3D104F002000028EFD0DFF810C300DF054605F0010030B1AB481430FFF7EDFD182024F051FC05F002000028DDD0BC48007815F0CBFDA54880ED780AD0ED780A36
:409F0000B0EE600A142100F5E4701AF039FF2AF081FA78B1B348007815F075FF9B4880ED0A0AD0ED0A0AB0EE600A1E2110301AF027FF87E02AF086FA002823D0FFF7D0FCE5
:409F400008B3A948007815F05EFF904880ED8E0AA648007815F09AFD8C4880EDA40AD0EDA40AB0EE600A142100F51E701AF008FF8648D0ED8E0AB0EE600A142100F5087084
:409F80001AF0FEFE5EE09748007815F03CFF7F4880ED0A0AD0ED0A0AB0EE600A1E2110301AF0EEFE794890ED0A0AD0ED040A30EE600A20EE000AB0EE408A1E212030B0EEDE
:409FC000480A1AF0DDFE8A48007815F01CFF6F4880ED200AD0ED200AB0EE600A1E2168301AF0CEFE694890ED200AD0ED1A0A30EE600A20EE000AB0EE408A1E217830B0EE10
:40A00000480A1AF0BDFE5F48007815F0FCFE5F4880ED360AD0ED360AB0EE600A1E21C0301AF0AEFE5648007815F0EDFE574880ED4C0AD0ED4C0AB0EE600A1E2100F58C70FA
:40A040001AF09EFE50495148FFF73EFB4E494F48FFF772FA4C48FFF7A1F92CF098FD064631464948FFF77EF84748007820B1484890F84800002845D12AF0CCF990B11FED12
:40A08000D30A414880ED020A0020404908700021584800782AF000FA0021574800782AF0FBF9BCE02AF0CEF900282AD01FEDDF0A354880ED020A00203449087000214E48B7
:40A0C00000782AF0E9F900214C4800782AF0E4F90021484800782AF0DFF90021484800782AF0DAF90021474800782AF0D5F90021454800782AF0D0F90021444800782AF03F
:40A10000CBF98CE0224890F84800012836D11F48007898BB2AF07EF968B101201B4908700121354800782AF0B7F90121314800782AF0B2F973E02AF085F9F8B101201349E2
:40A14000087001212C4800782AF0A6F901212B4800782AF0A1F90121264800782AF09CF90121274800782AF097F90121254800782AF092F901212448007849E04FE000006B
:40A1800027070020260700202008002074080020C80700200000002004000020080000200C000020100000201400002018000020200000201C000020DC0B00202400002036
:40A1C000280000200000C8420000C8C2C1FF030881F30308F03F0020E1F3030829F3030893060020E4060020DC060020E1060020E7060020F5060020F60600200B070020A2
:40A20000F40600200D07002015070020F70600202AF042F90121FE4800782AF03DF9FD4991F84A00FC49D1ED020AB0EE600AFEF7EBFE3AE601B50BF091FE70B900BF012279
:40A240006946F64800689C300FF00EFA20B99DF80000F04981F89C0000BFF148016D0120DFF8C0C300DF132002F08AFF08BD10B52DED020B00249DED000AF2EE040AB4EE93
:40A28000E00AF1EE10FA05DDB2EE040A8DED000A02240BE09DED000AB5EEC00AF1EE10FA04D29FEDE10A8DED000A032400BF04226946DA480068A0300FF0D6F920B99DEDA5
:40A2C000000AD44880ED280A00BFD548016D0120DFF850C300DF182002F052FF20461CBD01B500BF02226946CC480068A8300FF0BBF920B9BDF80000C649A1F8A80000BFBF
:40A30000C748016D0120DFF81CC300DF08BD10B5FFF758FB58B144F62060FFF7E1FFB6EE000AFFF7A4FF0020FFF784FF1BE0FFF7D7FA50B12820FFF7D3FF9FEDBB0AFFF784
:40A3400096FF0020FFF776FF0DE0FFF794FB50B144F62060FFF7C4FF9FEDB30AFFF787FF0020FFF767FFAB4991F84A00FEF793FB012010BD70B52DED028BB0EE408A0446E0
:40A380000D460026012C04D0022C03D0032C4AD101E000BF00BFA54890ED140AB4EEC80AF1EE10FA05DD90ED140AB0EE408A03260CE09E4890ED130AB4EEC80AF1EE10FABD
:40A3C00004D290ED130AB0EE408A022610219748DFF85CC200DF012823D004EB44019348143000EB810080ED018A2CF0D0FB04EB44028E49143141F82200012104EB4402BC
:40A400008A48143000EB8200017204EB44018748143000EB810045728448DFF818C200DF00E0062601E0062600BF00BF3046BDEC028B70BD7D4890ED110A7047764890F896
:40A440005000012800D170470020FCE7774890ED150A70470020754991F84810012904D175490978012900D10120704701B500BF01226946694800684A300FF0F5F820B957
:40A480009DF80000634981F84A0000BFFFF73FFF6348016D0120DFF88CC100DF262002F06FFE08BD644890ED780A7047624890ED8E0A7047604890ED040A70475E4890ED19
:40A4C0001A0A70475C4890ED080A70475A4890ED300A7047584890ED460A704700B5FFF771FA30B15548007808B1012000BD0020FCE70020FAE700207047504800780228AB
:40A5000004D14F48007D012800D170470020FCE710B5FFF7E5F930B14A4800782AF0BEFB08B1012010BD0020FCE770B52DED068B0024FFF78FFF70B329F0A0FF58B300BF60
:40A54000FFF799FA38B3334890EDD50A10EE101A084636F0FBFB41EC180BFEF751FD10EE105A284636F0F2FB41EC1A0BB0EE4A0AF0EE6A0A32F0C4FFB0EE409AF0EE609AB7
:40A5800053EC182B51EC190B36F0E8F901D2012000E0002004462046BDEC068B70BD00201D4991ED020A1B4991F84220743101EB8201D1ED000AB4EEE00AF1EE10FA10DB0B
:40A5C000154991ED020A134991F84220843101EB8201D1ED000AB4EEE00AF1EE10FA00D80120704700200C4991ED020A094991F842206C3101EB8201D1ED000AB4EEE00A7F
:40A60000F1EE10FA2DD8044991ED020A01491BE0F7060020081F002020080020A4030020F03F002081F3030800000000C807002049F8030865F70308740800202C00002045
:40A64000402800201907002091F842207C3101EB8201D1ED000AB4EEE00AF1EE10FA00DB0120704700B50023FFF7BCFF10B9FFF796FF00B10123184600BD70B52DED068B7E
:40A680000024FFF7E7FE78B329F0F8FE60B3FFF7E9FF48B300BFFFF7EEF928B3FE4890EDD60A10EE101A084636F050FB41EC180BFEF7A6FC10EE105A284636F047FB41EC22
:40A6C0001A0BB0EE4A0AF0EE6A0A32F019FFB0EE409AF0EE609A53EC182B51EC190B36F003F802D2012001E001E0002004462046BDEC068B70BD70B52DED068B0024FFF78B
:40A70000A9FE70BB29F0BAFE58B300BFFFF7B3F938B3E14890EDD70A10EE101A084636F015FB41EC180BFEF76BFC10EE105A284636F00CFB41EC1A0BB0EE4A0AF0EE6A0AA7
:40A7400032F0DEFEB0EE409AF0EE609A53EC182B51EC190B36F002F901D2012000E0002004462046BDEC068B70BD70B52DED068B0024FFF780F970B3FFF76CFE58B329F072
:40A780007DFE40B300BFC44890EDD50A10EE101A084636F0DBFA41EC180BFFF797FE10EE105A284636F0D2FA41EC1A0BB0EE4A0AF0EE6A0A32F0A4FEB0EE409AF0EE609A46
:40A7C00053EC182B51EC190B36F0C8F801D2012000E0002004462046BDEC068B70BD70B52DED068B0024FFF746F978B3FFF732FE60B3FFF7F7FE48B329F040FE30B300BF19
:40A80000A54890EDD60A10EE101A084636F09EFA41EC180BFFF75AFE10EE105A284636F095FA41EC1A0BB0EE4A0AF0EE6A0A32F067FEB0EE409AF0EE609A53EC182B51EC45
:40A84000190B35F051FF02D2012001E001E0002004462046BDEC068B70BD70B52DED068B0024FFF708F970B3FFF7F4FD58BB29F005FE40B300BF884890EDD70A10EE101A25
:40A88000084636F063FA41EC180BFFF71FFE10EE105A284636F05AFA41EC1A0BB0EE4A0AF0EE6A0A32F02CFEB0EE409AF0EE609A53EC182B51EC190B36F050F801D201209D
:40A8C00000E0002004462046BDEC068B70BD70B52DED068B0024FFF7CEF870B3FFF7BAFD58B329F0CBFD40B300BF6B4890EDD50A10EE101A084636F029FA41EC180BFFF70F
:40A90000E9FD10EE105A284636F020FA41EC1A0BB0EE4A0AF0EE6A0A32F0F2FDB0EE409AF0EE609A53EC182B51EC190B36F016F801D2012000E0002004462046BDEC068B2F
:40A9400070BD70B52DED068B0024FFF794F878B3FFF780FD60B3FFF722FE48B329F08EFD30B300BF4C4890EDD60A10EE101A084636F0ECF941EC180BFFF7ACFD10EE105A63
:40A98000284636F0E3F941EC1A0BB0EE4A0AF0EE6A0A32F0B5FDB0EE409AF0EE609A53EC182B51EC190B35F09FFE02D2012001E001E0002004462046BDEC068B70BD70B5B5
:40A9C0002DED068B0024FFF756F870B3FFF742FD58BB29F053FD40B300BF2F4890EDD70A10EE101A084636F0B1F941EC180BFFF771FD10EE105A284636F0A8F941EC1A0B00
:40AA0000B0EE4A0AF0EE6A0A32F07AFDB0EE409AF0EE609A53EC182B51EC190B35F09EFF01D2012000E0002004462046BDEC068B70BD70B52DED088B0024FFF71CF868B31E
:40AA400029F01CFD50B300BFFFF740FDF0EE400AFFF740FD30EE800AB0EE408A0E4890EDD80A10EE101A084636F070F941EC190BFFF720FD30EE480A10EE105A284636F0BA
:40AA800065F941EC1B0BB0EE4B0AF0EE6B0A32F037FDB0EE40AA02E0081F00200DE0F0EE60AA53EC192B51EC1A0B35F057FF01D2012000E00020044600BF2046BDEC088BC4
:40AAC00070BDD24890ED030A704710B50124D04890F84A000E2811D0CD4890F84A0002280CD0CB4890F84A00152807D0C84890F84A00032803D129F0A5FC00B100240CB1D0
:40AB0000012010BD0020FCE710B50024FFF7A2FCA0B129F0B3FC88B1FFF7D7FF70B100BFFFF7CFFFBA48D0EDD90AB4EEE00AF1EE10FA01DD012000E000200446204610BD52
:40AB400010B50024FFF786FC98B129F097FC80B1FFF7BBFF68B1FFF7B4FFAD48D0EDDA0AB4EEE00AF1EE10FA01D2012000E000200446204610BD10B50024FFF76BFC98B9C9
:40AB800029F07CFC80B1FFF7A0FF68B1FFF799FF9F48D0EDDB0AB4EEE00AF1EE10FA01DD012000E000200446204610BD994890ED030A704710B50024FFF74CFCA0B129F06A
:40ABC0005DFC88B1FFF781FF70B100BFFFF7EEFF8F48D0EDD90AB4EEE00AF1EE10FA01DD012000E000200446204610BD10B50024FFF730FCA0B129F041FC88B1FFF765FFDD
:40AC000070B100BFFFF7D2FF8148D0EDDA0AB4EEE00AF1EE10FA01D2012000E000200446204610BD10B50024FFF714FCA0B929F025FC88B1FFF749FF70B100BFFFF7B6FF99
:40AC40007348D0EDDB0AB4EEE00AF1EE10FA01DD012000E000200446204610BD70B52DED068B002429F00AFC78B3FFF72EFF60B300BF674890EDDC0A10EE101A084636F0A5
:40AC800065F841EC180BFFF71CFFF0EE400AFFF78DFF30EEC00A10EE105A284636F056F841EC1A0BB0EE4A0AF0EE6A0A32F028FCB0EE409AF0EE609A53EC182B51EC190BEB
:40ACC00035F04CFE02D2012001E001E0002004462046BDEC068B70BD10B52DED028B9FED4E0AB0EE408A29F095FB28B14B4890ED030AB0EE408A11E029F0A4FB70B1FFF778
:40AD0000E0FEB0EE408AB3EE040AB4EEC08AF1EE10FA03D89FED400AB0EE408AB0EE480ABDEC028B10BD3E4890EDA40A704710B52DED068BFEF7D4FD20B1FFF7C2FEB0EE7A
:40AD4000408A0CE0324890F84A00032803D1354890ED038A03E0FFF7ADFBB0EE408A18EE100A35F0F3FF41EC1A0BB0EE4A0AF0EE6A0A32F0C5FBB0EE409AF0EE609A9FEDD7
:40AD80002A0B53EC102B51EC190B35F0ADFC03D89FED210AB0EE408AB0EE480ABDEC068B10BD00B50022FFF755FB90B1FEF798FD78B1FFF7B8FFF0EE400AFFF773FB9FEDEE
:40ADC0001C1A20EE010AF4EEC00AF1EE10FA00DD0122104600BD00B50022FFF73BFB90B1FEF77EFD78B1FFF79EFFF0EE400AFFF759FB9FED101A20EE010AF4EEC00AF1EE20
:40AE000010FA00D20122104600BD0000100C0020081F0020680C002000000000C00C002074080020180D002000000000000034406666663FCDCCCC3D10B5044629F0EAFA89
:40AE400000287DD0092C7CD005DC4CB1032C31D0062C77D158E00B2C75D00C2CF9D1E5E00120FE490870FA208861FA21FB48C1612BF08DFEF94948620121F84880F82810D2
:40AE8000D0ED080AB0EE600AF54800782DF046FE0020F24948604FF47A71F0488160416A0161002101759FEDEF0AEF4800782DF035FEF5E00120E9490870FA204860FA21B6
:40AEC000E64881602BF063FEE44908610121E3480175D0ED030AB0EE600AE34800782DF01DFE0020DD4988614FF47A71DB48C16101694162002180F828109FEDDA0AD848B1
:40AF000000782DF00BFECBE00120D44908704FF47A7088610021D148C1612BF038FECF4948620121CD4880F82810D0ED080AB0EE600ACB4800782DF0F1FD0020C74903E026
:40AF4000AFE011E0ABE03AE048604FF47A71C3488160416A0161002101759FEDC20AC24800782DF0DBFD9BE00120BC4908704FF47A7048600021B94881602BF008FEB74965
:40AF800008610121B5480175D0ED030AB0EE600AB54800782DF0C2FD0020B04988614FF47A71AE48C16101694162002180F828109FEDAC0AAA4800782DF0B0FD70E0022062
:40AFC000A6490870642048600021A44881602BF0DEFDA24908610121A0480175D0ED030AB0EE600AA04800782DF098FD64209B49886100219948C16101694162002180F807
:40B0000028109FED980A964800782DF087FD0020924981F87C000121904880F87D10022180F88B10002180F88C1039E002208B4908704FF47A7048600146884881602BF0EA
:40B04000A6FD86490861012184480175D0ED030AB0EE600A844800782DF060FD4FF47A707E49886101467D48C16101694162002180F828109FED7B0A794800782DF04EFD66
:40B080000020764981F87C000121744880F87D10022180F88B10002180F88C1000E000BFDDE229F0CFF90028FAD0102C75D2DFE804F074083E75ABFA74E7E6E5E47474E356
:40B0C000E2E10120654908704FF4FA70C8620146624801632BF05BFD6049886301215F4880F83C106148007829F0D6F900205B4948604FF47A7159488160816B01610021F2
:40B1000001750020554908644FF47A7153484164816BC164002180F850105348007829F0BBF900215248007829F0B6F996E201204A4908704FF4FA700864014647484164E4
:40B140002BF025FD4549C8640121444880F850104748007829F0A0F90020404948604FF47A713E488160C16C01610021017500203A49C8624FF47A7138480163C16C81639D
:40B18000002180F83C103848007829F085F900213648007829F080F960E25EE201202F4908704FF4FA70486001462C4881602BF0EEFC2A4908610121284801752A4800781B
:40B1C00029F06AF90020254908644FF47A71234841640169C164002180F8501000201F49C8624FF47A711D48016301698163002180F83C101D48007829F04EF900211C4875
:40B20000007829F049F929E20120144908704FF4FA70C8620146114801632BF0B8FC0F49886301210D4880F83C101048007829F033F94FF4FA700949086401460748416457
:40B240002BF0A5FC0549C8640121044880F850100748007829F020F9002013E058140020AD06002000000000AE06002005070020FC060020B5E172E129E1EEE0B7E080E00D
:40B2800049E010E0F74948600021F64881602BF07EFCF44908610021F2480175F248007829F0FAF8DAE10120EE4908703220C8623221EC4801632BF06AFCEA4988630121D1
:40B2C000E84880F83C10E948007829F0E5F83220E44908643221E34841642BF058FCE149C8640121DF4880F85010E148007829F0D3F80020DB4948600021DA4881602BF017
:40B3000046FCD84908610021D6480175D648007829F0C2F8A2E10120D24908704FF47A70C8620021CF4801632BF031FCCD4988630121CC4880F83C10CC48007829F0ACF86D
:40B340000020C84948604FF47A71C6488160816B0161002101750020C24908644FF47A71C0484164816BC164002180F85010BE48007829F091F80021BD48007829F08CF81B
:40B380006CE10120B74908704FF47A7008640021B44841642BF0FBFBB249C8640121B14880F85010B248007829F076F80020AD4948604FF47A71AB488160C16C01610021B8
:40B3C00001750020A749C8624FF47A71A5480163C16C8163002180F83C10A348007829F05BF80021A148007829F056F836E101209C4908704FF47A70486000219948816023
:40B400002BF0C5FB974908610121964801759648007829F041F80020924908644FF47A71904841640169C164002180F8501000208C49C8624FF47A718A480163016981635F
:40B44000002180F83C108948007829F025F800218748007829F020F800E10120814908704FF47A70C86200217E4801632BF08FFB7C49886301217B4880F83C107B480078B0
:40B4800029F00AF84FF47A70764908640021754841642BF07CFB7349C8640121714880F850107348007828F0F7FF00206D49486000216C4881602BF06AFB6A490861002137
:40B4C000684801756848007828F0E6FFC6E00220644908704FF47A7048600021614881602BF055FB5F49086101215E48017500215D48007828F0D0FF4FF47A705949C862BC
:40B5000000215848016301698163012180F83C1000215648007828F0BFFF4FF47A705149086400214F4841640169C164012180F8501000214E48007828F0AEFF00204949E6
:40B5400081F87C000221474880F87D10032180F87E1080F88B10002180F88C107EE00220404908706420486000213E4881602BF00EFB3C49086101213A4801753A48007852
:40B5800028F08AFF64203749C86200213548016301698163012180F83C103448007828F07BFF64202F49086400212E4841640169C164012180F850102D48007828F06CFF63
:40B5C0000020284981F87C000221264880F87D10032180F87E1080F88B10002180F88C103CE001201F4908704FF47A70486001461C4881602BF0CBFA1A4908610021194811
:40B60000017501211948007828F046FF4FF47A701449C8620021134801632BF0B8FA1149886301210F4880F83C101048007828F033FF00200B4908644FF47A71094841643B
:40B640002BF0A5FA0749C8640021064880F850100748007828F020FF00E000BF00BF0548047010BD58140020AE06002005070020FC0600203E03002001B59DF8000000EE1B
:40B68000100AB8EE400AFE4880ED030A9DF8000000EE100AB8EE400AF94880ED080A00BF01226946F748006840300DF0DDFF20B99DF80000F44981F8400000BF0120F34972
:40B6C000087008BD08B506464FF4C8774FF000080121EF4880F8A8119421E94830F0B1FD307818B94620FFF7C7FF11E0E64890F84050642D03DD6420FFF7BEFF08E00A2D64
:40B7000003DA0A20FFF7B8FF02E02846FFF7B4FF0020DB4981F88D0028F07CFEE8B10020FFF78AFBDB48DFEDDC0A9FEDDC0A01230022DB490090DB4800782CF0C1FED54878
:40B74000DFEDD50A9FEDD50A01230022D6490090D64800782CF0B4FE05E028F073FE10B10120FFF769FB0321C94880F8A81100BF012239464FF6FF70DFF834C300DF2BF06D
:40B7800006FA0446BE4890F88D00002874D101201DF075FF18BB28F03DFE68B1C548007818B9BA480078012805D10020FFF744FB0020B64908709EE028F044FE0028FAD051
:40B7C000BC480078052803D1B04800780128F2D10520FFF731FB0020AC4908708BE008F0E9FB20BB28F016FE70B1B2480078092803D1A648007801287DD10920FFF71CFBA3
:40B800000020A249087076E028F01CFE002872D0A8480078022803D19C48007801286AD10220FFF709FB00209849087063E028F0F1FD70B19F480078062803D193480078BA
:40B84000012858D10620FFF7F7FA00208F49087051E028F0F7FD28B396480078042803D18A480078012846D10420FFF7E5FA0020864908703FE0FFE7814890F88D00012895
:40B8800023D128F0C7FD70B18A4800780C2803D17E48007801282ED10C20FFF7CDFA00207A49087027E028F0CDFD20B3814800780D2803D17548007801281CD10D20FFF727
:40B8C000BBFA00207149087015E06D4890F88D00022810D128F0B6FD68B1764800780F2803D16A480078012805D10F20FFF7A4FA00206649087062480078012802D00228D8
:40B900007ED115E15E48007D28BB5D48406810B35B48016920462BF071F95949896888423FD3012156480175046128F073FD48B15348D0ED030AB0EE600A5C4800782DF083
:40B94000EDF82EE028F07EFD10B301215748007828F0A2FD25E04A48007D012821D148488068A8B14648016920462BF047F944494968884215D3002141480175046128F048
:40B9800049FD30B19FED4C0A484800782DF0C6F807E028F057FD20B100214448007828F07BFD374890F82800C8B935488069B0B13348416A20462BF021F93149C969884214
:40B9C0002BD301212E4880F828104462D0ED080AB0EE600A334800782DF0A0F81DE0284890F82800012818D12548C069A8B12448416A20462BF002F921498969884200E025
:40BA0000F6E10AD300211E4880F8281044629FED2A0A244800782DF081F8194890F85000A8B91748006C90B11548C16C20462BF0E5F81349496C884245D30121104880F8C8
:40BA40005010C4641D48007828F026FD3BE00C4890F85000012836D10948406C80B30848C16C20462BF0CAF80549096C88422AD30021034880F85010C4641048007820E0F9
:40BA800058140020A4030020081F00203F030020F03F0020A0D800200000FA4300247449001C0040AD06002000200040AE060020E1F303083E03002000000000FC060020C0
:40BAC00001E028F0E9FCD84890F83C00A8B9D648C06A90B1D448816B20462BF08FF8D249096B884223D30121CF4880F83C108463CE48007828F0D0FC19E0CB4890F83C0015
:40BB0000012814D1C848006B88B1C748816B20462BF074F8C449C96A884208D30021C24880F83C108463C148007828F0B5FC5FE1BD4890F88C107C30405C78BBBA48007DF3
:40BB400001282CD1B848016920462BF057F8B6494968884221D30021B3480175046128F059FC30B11FED2C0AB14800782CF0D6FF0DE028F067FC50B11FED310AAC480078F2
:40BB80002CF0CCFF0021AA48007828F085FCA6488068002801D14FF00108C1E00BE0A248016920462BF02AF89F498968884201D34FF00108B4E09C4890F88C107C30405C3C
:40BBC00001282BD1984890F8280001281AD19648416A20462BF012F893498969884210D30021914880F8281044621FED4D0A914800782CF093FF8C48C069002801D14FF005
:40BC000001088DE08848416A20462AF0F7FF8649C969884201D34FF0010881E0824890F88C107C30405C022836D17F4890F83C00012825D17C48816B20462AF0DFFF7A4973
:40BC4000C96A88426CD30021774880F83C1084637648007828F020FC28F0F4FB50B100217248007828F018FC1FED6D0A6F4800782CF054FF6C48006B90BB4FF001084FE00A
:40BC80006948816B20462AF0B9FF6749096B884246D34FF0010843E0634890F88C107C30405C03283CD1604890F8500001282CD15D48C16C20462AF0A1FF5B49096C884273
:40BCC0002ED30021584880F85010C46428F0A2FB38B11FED870A574800782CF01FFF0EE01EE028F0AFFB50B11FED8D0A524800782CF014FF00215048007828F0CDFB4A48C0
:40BD0000406C68B94FF001080AE04748C16C20462AF074FF4449496C884201D34FF00108B8F1010F63D14FF000083F4890F88C00401CC1B23C4880F88C1090F88C1090F84B
:40BD40008B00814203DB0021374880F88C10364890F88C107C30405C022809D10121324880F83C1084633148007828F095FB3EE02D4890F88C107C30405C01280DD10121ED
:40BD8000294880F828104462D0ED080AB0EE600A284800782CF0C2FE29E0234890F88C107C30405C032809D101211F4880F85010C4642148007828F06FFB18E001211A48D4
:40BDC0000175046128F026FB48B11748D0ED030AB0EE600A164800782CF0A0FE07E028F031FB20B101211248007828F055FB00BFBEE42DE9F04106460C4617469846069DF9
:40BE00002078642803DD6420FFF736FC09E020780A2803DA0A20FFF72FFC02E02078FFF72BFCBDE8F08100005814002005070020AE060020AD060020FC0600200000000049
:40BE40000000000000000000000000000000000000000000000000000000000000000000000000000000000000000000526176656E20496E647573747269657320496E6342
:40BE80000000000000000000000000004175672D31382D323031380000000000322E352E302E323700000000000000005374656572696E6720436F6E74726F6C20556E69BF
:40BEC0007400000000000000000000003037373031373135303200000000000000000000000000000000000000000000FFFFFFFFFFFFFFFFFFFFFFFFFFFFFFFFFFFFFFFFE4
:40BF0000FFFFFFFFFFFFFFFFFFFFFFFFFFFFFFFFFFFFFFFFFFFFFFFFFFFFFFFFFFFFFFFFFFFFFFFFFFFFFFFFFFFFFFFFFFFFFFFFFFFFFFFFFFFFFFFFFFFFFFFFFFFFFFFF41
:40BF4000FFFFFFFFFFFFFFFFFFFFFFFFFFFFFFFFFFFFFFFFFFFFFFFFFFFFFFFFFFFFFFFFFFFFFFFFFFFFFFFFFFFFFFFFFFFFFFFFFFFFFFFFFFFFFFFFFFFFFFFFFFFFFFFF01
:40BF8000FFFFFFFFFFFFFFFFFFFFFFFFFFFFFFFFFFFFFFFFFFFFFFFFFFFFFFFFFFFFFFFFFFFFFFFFFFFFFFFFFFFFFFFFFFFFFFFFFFFFFFFFFFFFFFFFFFFFFFFFFFFFFFFFC1
:40BFC000FFFFFFFFFFFFFFFFFFFFFFFFFFFFFFFFFFFFFFFFFFFFFFFFFFFFFFFFFFFFFFFFFFFFFFFFFFFFFFFFFFFFFFFF00C00008FFFF030800800008FBBF00080EA6D59435
:40C0000001B500BF01226946FE48006800F5D9700DF02AFB20B99DF80000FB4981F8B20100BF022017F084FC012009F016FD08BD01B500BF01226946F248006800F2B310D5
:40C040000DF012FB20B99DF80000EF4981F8B30100BF022017F06CFC012009F0FEFC08BD70B52DED028B05460E460024012D07D1E54890ED610ABDEEC00A10EE104A12E051
:40C08000032D07D1E04890ED630ABDEEC00A10EE104A08E0022D06D1DB4890ED620ABDEEC00A10EE104AD84890F8B201032809D1D648844202DC4042844201DA00242CE05D
:40C0C00001242AE0D04890F8B20108280AD142F21070844202DC4042844201DA00241CE001241AE0204634F0D4FA41EC180B9FEDC80B53EC102B34F031FC0BD3204634F0BF
:40C10000C8FA41EC180B9FEDC40B53EC102B34F0EBFA01D2002400E001241CB10120BDEC028B70BD0020FAE701460420704731B52DED020B044600BF04226946B148006853
:40C1400000F5C2700DF090FA20B99DED000AAE4880ED610A00BF0BF0D6F810B109F087FC08E00BF009F910B117F095FE02E0012017F0FEFC1C2022F007FB01203EBD31B57B
:40C180002DED020B2DED088B044694B300209FEDA40A16F01BFB10EE105A284634F0D6FD41EC1B0BB0EE4B0AF0EE6B0A31F0A8F9B0EE40AAF0EE60AA51EC1A0B33F08AFFFE
:40C1C00008EE100A904890EDE20A30EE480AF0EE408A90EDE20A30EE080AB0EE409A9DED080AB4EEC90AF1EE10FA03DD8DED089A09E009E09DED080AB4EEE80AF1EE10FAE4
:40C2000001D2CDED088A0FE000BF042208A97D48006800F562700DF027FA20B99DED080A794880EDE20A00BF00BF042208A97548006800F5C6700DF017FA20B99DED080A91
:40C24000714880ED630A00BF0BF05DF810B109F00EFC08E00BF090F810B117F01CFE02E0022017F085FC1C2022F08EFA0120BDEC088B3EBD31B52DED020B044600BF042215
:40C2800069466048006800F5C4700DF0EDF920B99DED000A5C4880ED620A00BF0BF033F810B109F0E4FB08E00BF066F810B117F0F2FD02E0032017F05BFC1C2022F064FA44
:40C2C00001203EBD0146002009292BD2DFE801F02A1F20051D1E2A2A13009FED521AC0EE010A9FED511A70EE810AFCEEE00A10EE902A90B218E0DFED4C0A70EE200AFCEED9
:40C30000E00A10EE902A90B20EE000BF00BF00BFDFED460A60EE200AFCEEE00A10EE902A90B201E0002000BF00BF704701460020092923D2DFE801F022171805151622224B
:40C340000F00DFED380A80EE201AFDEEC10A10EE902A10B214E0FCEEC00A10EE902A10B20EE000BF00BF00BFDFED300A60EE200AFDEEE00A10EE902A10B201E0002000BFEE
:40C3800000BF7047DFED2A0AB0EE600A28B92949D1ED360AB0EE600A06E0012804D12549D1ED590AB0EE600A704770B52DED0A8BB0EE408A9FED200AC8EE000A10EE905ADA
:40C3C000114890ED610AF0EE408A90ED630AB0EE409A0020FFF7D6FFF0EE409A284634F0B5FC41EC1A0B38EEE90A78EEC90A80EE201A11EE106A304634F0A8FC41EC1C0BB5
:40C400001CE00000A4030020081F0020001A0B009A999999999913409A9999999999B93F35FA0E3D0000AF4300401C4500007A4400000000700D00200000C842B0EE4C0AEE
:40C44000F0EE6C0A31F05CF8B0EE40BAF0EE60BA53EC1A2B51EC1B0B34F046F901D2012000E0002004462046BDEC0A8B70BD70B52DED0A8BB0EE408A1FED110AC8EE000AE7
:40C4800010EE905AFE4890ED620AF0EE408A90ED630AB0EE409A0020FFF774FFF0EE409A284634F053FC41EC1A0B38EEE90A78EEC90A80EE201A11EE106A304634F046FC98
:40C4C00041EC1C0BB0EE4C0AF0EE6C0A31F018F8B0EE40BAF0EE60BA53EC1A2B51EC1B0B34F002F901D2012000E0002004462046BDEC0A8B70BD70B52DED0C8BF0EE408A4C
:40C500001FED330AC8EE800A10EE904ADC4890ED620AF0EE409A90ED610AB0EE40AA90ED630AB0EE408A0020FFF72CFFB0EE409A204634F00BFC41EC1B0B39EE480A7AEE95
:40C54000480A80EE201A11EE106A304634F0FEFB41EC1D0BB0EE4D0AF0EE6D0A30F0D0FFB0EE40CAF0EE60CA53EC1B2B51EC1C0B34F0BAF824D2204634F0E8FB41EC1B0B02
:40C5800039EE480A79EEC80A80EE201A11EE106A304634F0DBFB41EC1D0BB0EE4D0AF0EE6D0A30F0ADFFB0EE40CAF0EE60CA53EC1B2B51EC1C0B34F097F801D2012000E0AD
:40C5C000002005462846BDEC0C8B70BDAD4890F85000032801D0012070470020FCE710B50124FFF7F3FF28B9A649C86A64212AF0D4FA00B10024204610BDA24890F828006E
:40C60000032801D0012070470020FCE710B50124FFF7F3FF28B99B49486864212AF0BDFA00B10024204610BD10B5FFF7EFFF10B1FFF7D5FF08B9022411E0914890ED6A0AA8
:40C64000B5EEC00AF1EE10FA08D090ED6B0AB5EEC00AF1EE10FA01D0012400E00024204610BD18B9874991ED080A04E0012802D1844991ED120A704710B5002182480078C0
:40C680002CF03AFA0021814800782CF035FA7C4890F8B201032802D0082820D10FE000209FED7B0AFFF743FD00201FED9F0AFFF766FD00209FED770AFFF7DCFD1FE00020C1
:40C6C0009FED750AFFF733FD00201FEDA70AFFF756FD00209FED710AFFF7CCFD0FE00020B7EE000AFFF723FD0020B0EE040AFFF746FD0020B1EE000AFFF7BCFD00BF00BF2E
:40C7000010BD01B55E4890F8410001280FD000BF012269466248006800F2B5100CF0A4FF20B99DF80000564981F8B50100BF1C2022F02AF808BD10B52DED028B044694ED9F
:40C74000030AD4ED040A30EE600A84ED060A94ED030A84ED040A2AF01AFA2060D4E90001401AA06094ED020AB8EE400A5FEDD10A80EE201AB0EE418A20686060B5EEC08A17
:40C78000F1EE10FA0EDD94ED060AC0EE080AC4ED050AD4ED050AB0EE600A042104F11C0018F0EEFABDEC028B10BD10B52DED020B00BF042269463A48006800F5D4700CF0F4
:40C7C00053FF20B99DED000A2D4880ED6A0A00BF1CBD10B52DED020B00BF042269463048006800F5D6700CF03FFF20B99DED000A234880ED6B0A00BF1CBD10B52DED020B79
:40C8000000BF042269462648006800F5CE700CF02BFF20B99DED000A194880ED670A00BF1CBD10B52DED020B00BF042269461C48006800F5D2700CF017FF20B99DED000AEF
:40C840000F4880ED690A00BF1CBD0E4981F8500070470C4981F82800704710B5094890F86D01012828D0064890F84B00054981F86C01084690F86C11543018F071FA11E0A8
:40C88000081F0020700D0020D8060020D706002090ED24C990ED244900803BC500803B45A4030020FC4890F86C11E03018F058FA0120F94981F86D01F84890F8B201092855
:40C8C0007DD2DFE800F09005336581828B916600F348007827F0A6FF00EE100AB8EE400ADFEDF00A20EE200AEB4880ED040A90ED040AF6EE000AB4EEE00AF1EE10FA03D2AA
:40C900000020FFF7A6FF10E0E34890ED040ADFEDE60AB4EEE00AF1EE10FA03DD0120FFF798FF02E00320FFF794FF66E0DC48007827F078FF00EE100AB8EE400ADFEDD90A32
:40C9400020EE200ADFEDD90A80EE201AD24880ED041A90ED040ADFEDD60AB4EEE00AF1EE10FA03D20020FFF774FF10E0CA4890ED040ADFEDD00AB4EEE00AF1EE10FA03DDF1
:40C980000120FFF766FF02E00320FFF762FF34E000BFC34800782CF08FF800EE100AB8EEC00ABD48D0ED000A30EE200A80ED040AFDF794FD20B10020FFF74BFF03E011E015
:40C9C0000320FFF746FF18E000BF9FEDBB0AB24880ED040A0020FFF73CFF0EE00320FFF738FF0AE000BF00BF9FEDB30AAA4880ED040A0020FFF72DFF00BF00BFA64890F879
:40CA00006C11D0ED040AB0EE600A543018F054F9A148001DFFF78FFEA04890F8B301092870D2DFE800F08005337065667B727100A248007827F0F6FE00EE100AB8EE400A40
:40CA4000DFED980A20EE200A934880ED0E0A90ED0E0AF6EE000AB4EEE00AF1EE10FA03D20020FFF7F2FE10E08B4890ED0E0ADFED8E0AB4EEE00AF1EE10FA03DD0120FFF7B5
:40CA8000E4FE02E00320FFF7E0FE55E08B48007827F0C8FE00EE100AB8EE400ADFED810A20EE200ADFED810A80EE201A7A4880ED0E1A90ED0E0ADFED7E0AB4EEE00AF1EE2D
:40CAC00010FA03D20020FFF7C0FE10E0724890ED0E0ADFED780AB4EEE00AF1EE10FA03DD0120FFF7B2FE02E00320FFF7AEFE23E000BF9FED710A684880ED0E0A0020FFF71F
:40CB0000A4FE19E00EE000BF00BF9FED6B0A624880ED0E0A0320FFF798FE0DE00320FFF794FE09E000BF9FED640A5B4880ED0E0A0020FFF78AFE00BF00BF574890F86C11ED
:40CB4000D0ED0E0AB0EE600AE03018F0B5F852482C30FFF7F0FD10BD504890ED610AD0ED630A30EE600AB5EEC00AF1EE10FA01DD012070470020FCE730B589B027F075FC86
:40CB800040B10021084616F0E0FF0121002016F0DCFF1AE0414890F8B201032804D03F4890F8B201082808D10021032016F0CDFF0121032016F0C9FF07E00021032016F02B
:40CBC000C4FF0121002016F0C0FF344890F8B25190F8B341092D5ED2DFE805F0A2051729A4A578A32A000020009001900290034603222B4903900846007827F024FD0321E7
:40CC00002748007828F0CDF89FE0002000900190029003460322224903900846007827F012FD00211E48007828F0BBF88DE000BF002000900190029003460222184903905C
:40CC40000846007827F0FFFC02211548007828F0A8F827F0DFFB68B11948DFED170A9FED190A04230022184900900D4800782BF027FC0FE027F0E6FB60B11148DFED0E0AAB
:40CC80009FED100A0423002219070090044800782BF016FC59E043E0700D0020081F0020D80600203333533A666646400CAC233FCDCCCC3C33339F4000000000D706002064
:40CCC000A0D80020809FD54A00040140002000900190029003460222F74903900846007827F0B1FC0621F448007828F05AF8002000900190022314220121029004A82BF020
:40CD0000F7FC04A85FED140A9FEDEC0A032300224FF080410090E84800782BF0D1FB14E000BF00BF00BF002000900190029003460322E14903900846007827F084FC012153
:40CD4000DD48007828F02DF800BF00BF092C7BD2DFE804F0880517298A8B5D892A00002000900190029003460322D54903900846007827F068FC0321D148007828F011F823
:40CD800085E0002000900190029003460322CC4903900846007827F056FC0021C848007827F0FFFF73E000BF002000900190029003460222C24903900846007827F043FC2C
:40CDC0000221BF48007827F0ECFF27F023FB68B1BC485FED470A1FED450A04230122BA490090B74800782BF06BFB0FE027F02AFB60B1B4485FED500A1FED4E0A04230122E4
:40CE000091070090AE4800782BF05AFB3FE0002000900190029003460222A94903900846007827F010FC0621A548007827F0B9FF002000900190034614220121029004A8A4
:40CE40002BF056FC04A800E00CE05FED650A1FED630A0223012291070090994800782BF02FFB14E000BF00BF00BF002000900190029003460322924903900846007827F0CE
:40CE8000E2FB01218E48007827F08BFF00BF00BF09B030BD10B58D4988684FF4967129F07CFE10BD8A4890ED000A7047894991F84110012901D1012007E0864991F8B5114D
:40CEC00009B1012100E000210846704710B52DED068BB0EE408A8048007838B91FED8A0A7E4880ED000A01207B490870FFF7DEFF002868D009F032F8002864D0FFF7D2FF94
:40CF000010EE104A204633F021FF41EC1A0BB0EE4A0AF0EE6A0A30F0F3FAB0EE409AF0EE609A9FED6F0B53EC102B51EC190B33F0DBFB48D2FFF7AEFFE8BB20F0D4FEDFED15
:40CF40006A0AB4EEE00AF1EE10FA3CDBFFF76CFB012838D15F4890F830000A2833D05D4890F8B201092827D2DFE800F02610110512132626060000BF584890ED000ADFED58
:40CF80005B0A08EE200A80ED000A1BE000BF00BF00BF5048D0ED630A9FED541A48EE410AB0EE600A0120FFF7EAF81FEDBD0A4B4880ED000A06E006E01FEDC10A474880ED83
:40CFC000000A00BF00BFBDEC068B10BD434890F8280008B9012070470020FCE73F4890F82800012800D170470020FCE73B4890F8500008B9012070470020FCE7374890F8E2
:40D000005000012800D170470020FCE700B50021FFF7DCFF08B13D2103E0FFF7DFFF00B13C21084600BD10B516F036FE0446204610BD10B52DED028B0AF065F920B108F055
:40D0400092FDB0EE408A16E016F02EFD2148D0ED640A30EE600ADFED260A20EE200AD0ED650A90ED641A70EEC10A80EE201A9FED210A31EE008AB0EE480ABDEC028B10BDF7
:40D0800001B59DF80000202801DD2020009000BF01226946184800684B300CF0E5FA20B99DF800000B4981F84B0000BF00200B4981F86D0108BD0000D8060020A037A04C5A
:40D0C000D7060020A0D80020000401401043002038000020081F002040000020700D0020000000A046DF813F2FDDE43E0AD7A33B000048430000C8C2A403002010B54FF4F1
:40D10000B8711A482FF09DF810BD19490870704717480078704710B52DED028BB0EE408A1448007830B9144800210160416001201049087020F0D3FDF0EE408AF0EE680AEA
:40D14000B0EE480A16F082FB0C4880ED000A282109480A4A92ED000A17F012FEBDEC028B10BD064890ED000A70470000700D0020300000204100002038000020340000205A
:40D1800010B50446204622F0F5FD10BD07B586B00020049000210898017006980078692881F03A82DFE810F069006B00E70007013501380AAB00380743074E076301C901C4
:40D1C0002F02A402F9024E039B03F003550445047C00A50417058505CB051A069806F008B20659077E096507AB07BA07EF07FD070B084C085808680872088208380A380A51
:40D20000380A9208A308C60871077D0787079F079307380A380A380A380A380A380A380A380A380A380A380ABC04380A380A380AF4081C0939096109380A380A380A380A9E
:40D24000380A380A380A380A380A380A380A380A380A380A380A380A380A380A380A8E09BF09F009380A380A380A020A380A380A380A380A380A140A260A01F0D1B9FE484D
:40D2800090F841000390069890ED010ABCEEC00A10EE100AC0B20290039916F056FCECE70698007A032803D006210898017025E0069890ED010AF7EE000AB4EE600AF1EE42
:40D2C00010FA02D114F0E4FD18E0069890ED010AF0EE000AB4EE600AF1EE10FA02D114F0BFFD0BE0069890ED010AF0EE080AB4EE600AF1EE10FA01D114F0B8FBBDE706981D
:40D30000007A032809D1069890ED010A8DED030A9DED030A0EF07BF82AE00698007A012811D1D548B0F8BE110A22079802FB001000EE100AB8EEC00A8DED030A9DED030A8A
:40D340000EF065F814E00698007A022810D1CA48B0F8BE110A22079802FB101000EE100AB8EEC00A8DED030A9DED030A0EF04FF80120049081E708F0F1FDC0B90698007A5B
:40D38000032811D1069890ED010A8DED030A9DED030A09F0CBFBB948D0F81801014603908020DFF8DCC200DF0120049002E001210898017061E713F0EDFE30BB0698007AAA
:40D3C00003281ED1069890ED010ABCEEC00A10EE100A80B2039009F09AFB09F01BFB80B90821A848DFF8A0C200DF012809D0A748406840F00101A5484160A248DFF890C229
:40D4000000DF132021F0C0F902E001210898017033E713F0BFFE30BB09F0FCFA18B30698007A03281BD1069890ED010ABCEEC00A10EE100AC0B2039009F043FB082191485D
:40D44000DFF844C200DF012809D09048406840F001008E4948608B48DFF834C200DF132021F092F902E001210898017005E70698007A032817D1804890F8420003907E4859
:40D4800090F841000290069890ED010ABCEEC00A10EE100AC0B20190DDE9021210F043FE0899087046E00698007A01281FD1724890F841105C3000EB41006F4991F84210F3
:40D4C000415C0122079802FB0010C0B201906A4890F842000390684890F8410002900146039A019810F01FFE0899087022E00698007A02281ED1604890F841105C3000EBC5
:40D5000041015C3890F84200095C0122079802FB1010C0B20190584890F842000390564890F8410002900146039A019810F0FBFD08990870012004909FE60698007A032803
:40D5400017D14D4890F8420003904B4890F841000290069890ED010ABCEEC00A10EE100AC0B20190DDE9021210F01BFE0899087046E00698007A01281FD13F4890F841106B
:40D58000603000EB4101603890F84200095C0122079802FB0010C0B20190374890F842000390354890F8410002900146039A019810F0F7FD0899087022E00698007A022893
:40D5C0001ED12D4890F84110603000EB41002A4991F84210415C0122079802FB1010C0B20190254890F842000390234890F8410002900146039A019810F0D3FD089908706F
:40D600000120049039E60698007A032817D11A4890F842000390184890F841000290069890ED010ABCEEC00A10EE100AC0B20190DDE9021210F0F3FD0899087055E0069806
:40D64000007A01282ED10C4890F84110643000EB4100094991F84210415C0122079802FB0010C0B20190044890F842000390024890F8410002900DE0081F0020F03F0020AE
:40D6800081F30308D42F002049F80308E42F002065F703080146039A019810F0C0FD0899087022E00698007A02281ED1FE4890F84110643000EB4100FB4991F84210415CC1
:40D6C0000122079802FB1010C0B20190F64890F842000390F44890F8410002900146039A019810F09CFD0899087001200490C4E50698007A032810D1EB4890F842000390D5
:40D70000069890ED010A8DED020A03989DED020A10F0F7FE089908703CE00698007A01281AD1E14890F842107C3000EB8100D0ED000A9DED070AB8EEC00A30EEC00A8DED67
:40D74000020AD94890F8420003909DED020A10F0D8FE089908701DE00698007A022819D1D14890F842107C3000EB8100D0ED000A9DED070AB8EEC00A30EE800A8DED020A66
:40D78000C94890F8420003909DED020A10F0B9FE08990870012004906FE50698007A032810D1C14890F842000390069890ED010A8DED020A03989DED020A10F0D4FD0899B3
:40D7C00008703CE00698007A01281AD1B64890F842106C3000EB8100D0ED000A9DED070AB8EEC00A30EEC00A8DED020AAE4890F8420003909DED020A10F0B5FD0899087095
:40D800001DE00698007A022819D1A74890F842106C3000EB8100D0ED000A9DED070AB8EEC00A30EE800A8DED020A9F4890F8420003909DED020A10F096FD08990870012047
:40D8400004901AE50698007A032812D1964890F842000390069890ED010ABCEEC00A10EE100AC0B20290039910F017FD0899087032E00698007A012815D18B4890F842104F
:40D880006830415C0122079802FB0010C0B20290854890F8420001460390029810F0FDFC0899087018E00698007A022814D17E4890F842106830415C0122079802FB101070
:40D8C000C0B20290784890F8420001460390029810F0E3FC0899087001200490CDE40698007A032810D1704890F842000390069890ED010A8DED020A03989DED020A10F0B2
:40D900005BFE089908703CE00698007A01281AD1654890F84210843000EB8100D0ED000A9DED070AB8EEC00A30EE800A8DED020A5D4890F8420003909DED020A10F03CFEB4
:40D94000089908701DE00698007A022819D1564890F84210843000EB8100D0ED000A9DED070AB8EEC00A30EEC00A8DED020A4E4890F8420003909DED020A10F01DFE089948
:40D9800008700120049078E40698007A032810D1454890F842000390069890ED010A8DED020A03989DED020A10F052FD089908703CE00698007A01281AD13B4890F84210E6
:40D9C000743000EB8100D0ED000A9DED070AB8EEC00A30EE800A8DED020A334890F8420003909DED020A10F033FD089908701DE00698007A022819D12B4890F84210743046
:40DA000000EB8100D0ED000A9DED070AB8EEC00A30EEC00A8DED020A234890F8420003909DED020A10F014FD089908700120049023E40698007A03280AD1069890ED010AB2
:40DA4000BCEEC00A10EE100AC0B20390FCF7F2FB13E40698007A032812D1134890F842000390069890ED010ABCEEC00A10EE100AC0B20290039910F043FC0899087035E0A1
:40DA80000698007A012818D1074890F842106A30415C0122079802FB0010C0B20290024890F84200014601E0081F00200390029810F026FC0899087018E00698007A0228E4
:40DAC00014D1FB4890F842106A30415C0122079802FB1010C0B20290F54890F8420001460390029810F00CFC089908700120049004E40698007A032803D006210898017083
:40DB00000DE0069890ED010A8DED030A9DED030A0A2007F0F3FC10B901210898017029E40698007A032814D1069890ED010ABCEEC00A10EE100A80B200EE100AB8EE400A97
:40DB40008DED030A9DED030A0DF061FC089908703EE00698007A01281BD10EF09FF9F0EE400AD348B0F8BE0100EE100AB8EE401A9DED070AF8EE401AB0EE410A00EEA10A24
:40DB80008DED030A9DED030A0DF041FC089908701EE00698007A02281AD10EF07FF9F0EE400AC348B0F8BE0100EE100AB8EE401A9DED070AF8EE401AB0EE410A00EEE10A14
:40DBC0008DED030A9DED030A0DF021FC08990870012004901CE40698007A032815D1B44890F842000390B24890F841000290069890ED010A8DED010ADDE902019DED010A3F
:40DC000010F03FFA0899087050E00698007A012824D1A74890F842000290A54890F84100019002990EF01AFFDDED070AF8EE600A9FEDA01A01EE200A8DED030A9C4890F86B
:40DC4000420002909A4890F84100019002999DED030A10F016FA0899087027E00698007A022823D1924890F842000290904890F84100019002990EF0F1FEDDED070AF8EE4B
:40DC8000600A9FED8C1A01EE600A8DED030A884890F842000290864890F84100019002999DED030A10F0EDF9089908700120049042E40698007A03280BD1069890ED010A43
:40DCC0008DED030A9DED030A10F0FFFC0899087032E00698007A012815D17548D0ED7E0A9DED070AB8EE401ADFED731AB0EE600A01EE810A8DED030A9DED030A10F0E5FC42
:40DD00000899087018E00698007A022814D16848D0ED7E0A9DED070AB8EE401ADFED661AB0EE600A01EEC10A8DED030A9DED030A10F0CBFC089908700120049022E20698B8
:40DD4000007A032814D1069890ED010ABCEEC00A10EE100A80B200EE100AB8EE400A8DED030A9DED030AFCF782FA0899087032E00698007A012815D14D48D0ED280A07983B
:40DD800000EB8000400000EE100AB8EEC00A30EE800A8DED030A9DED030AFCF768FA0899087018E00698007A022814D14048D0ED280A079800EB8000400000EE100AB8EE7E
:40DDC000C00A30EEC00A8DED030A9DED030AFCF74EFA0899087001200490D3E10698007A03282DD1069890ED010ADFED340AB4EEE00AF1EE10FA06DD022108980170642015
:40DE0000FDF73AFC62E0069890ED010AF2EE040AB4EEE00AF1EE10FA06D20321089801700A20FDF729FC51E0069890ED010ABCEEC00A10EE100AC0B20390FDF71DFC45E083
:40DE40000698007A01281BD1194890F8401007984000C0F1650081420BDA154890F840100222079802FB0010C0B20390FDF704FC2CE00221089801706420FDF7FDFB25E0EC
:40DE80000698007A022821D1094890F84010079840000930814213DD054890F840100222079802FB1010C0B20390FDF7E5FB0DE0081F00200AD7233CCDCCCC3D0000C8423C
:40DEC0000321089801700A20FDF7D6FB1920FFF757F901200490A3E30698007A032803D006210898017010E0069890ED010ABCEEC00A10EE100AC0B21FED100A039007F032
:40DF0000FDFA10B901210898017089E30698007A032803D00621089801707CE0069890ED010AF8EE000AB4EE600AF1EE10FA13D1FB4890F842107C3000EB810090ED000A2D
:40DF40008DED030A9DED030A082007F0D7FA00BB0121089801705EE0069890ED010AFFEE000AB4EE600AF1EE10FA13D1EC4890F842106C3000EB810090ED000A8DED030A4D
:40DF80009DED030A082007F0B9FA10B901210898017040E0069890ED010AF7EE000AB4EE600AF1EE10FA13D1DD4890F84210743000EB810090ED000A8DED030A9DED030A3A
:40DFC000082007F09BFA00BB01210898017022E0069890ED010AF0EE000AB4EE600AF1EE10FA13D1CE4890F84210843000EB810090ED000A8DED030A9DED030A082007F0C2
:40E000007DFA10B901210898017004E09FEDC50A002007F073FA03E30020FEF7B3F98DED030A00209DED030AFEF781F8F8E20020FEF7A8F98DED030A00209DED030AFEF794
:40E040009EF8EDE20020FEF79DF98DED030A00209DED030AFEF70EF9E2E2069890ED010ABCEEC00A10EE100AC0B203900DF078FDD6E2069890ED010ABCEEC00A10EE100AFF
:40E08000C0B20390FEF73DFBCAE2069890ED010ABCEEC00A10EE100AC0B2039010F083FCBEE2069890ED010A8DED030A9DED030A10F08FFCB4E2069890ED010ABCEEC00AAD
:40E0C00010EE100AC0B203900EF043FCA8E2069890ED010ABCEEC00A10EE100A80B203900EF021FA9CE2069890ED010ABCEEC00A10EE100A80B203900EF02AFA90E2069885
:40E1000090ED010ABCEEC00A10EE100AC0B203900FF0F8F92020FFF733F881E20698007A032803D00621089801702BE0069890ED010AF7EE000AB4EE600AF1EE10FA05D1D9
:40E14000B7EE000A072007F0D9F91BE0069890ED010AF0EE000AB4EE600AF1EE10FA05D19FED700A002007F0C9F90BE0069890ED010AF0EE080AB4EE600AF1EE10FA01D185
:40E1800000F030FC4CE2069890ED010ABCEEC00A10EE100A80B201460390022015F0E8FA3EE2069890ED010ABCEEC00A10EE100A80B201460390012015F0DAFA30E20698C6
:40E1C000007A03283BD1069890ED010AB5EEC00AF1EE10FA0BD1524890F842000390504890F841000290039908F07FFE27E0069890ED010AF7EE000AB4EE600AF1EE10FA0A
:40E2000007D1474890F842000121039008F0D4FD15E0069890ED010AF0EE080AB4EE600AF1EE10FA0BD13E4890F8420003903C4890F8410001220290039908F03CFDEFE1D1
:40E24000069890ED010ABCEEC00A10EE100AC0B2039008F0FCFCE3E10698007A03280AD1069890ED010ABCEEC00A10EE100AC0B20390FCF7FBF8D3E112F08CFF28B90698B8
:40E28000007A032801D108F083FCC9E10698007A03280AD1069890ED010ABCEEC00A10EE100AC0B20390FDF7ABFEB9E10698007A03280AD1069890ED010ABCEEC00A10EE04
:40E2C000100AC0B20390FDF7B3FEA9E10698007A03280BD1069890ED010ABCEEC00A10EE100AC0B2012103900EF047F998E10698007A032813D1069890ED010ADFED0A0AF4
:40E30000B4EE600AF1EE10FA09D10CF037F901200CF012F8002005490872054908707FE1081F00200000000000007E43E42F0020C80400200698007A03280BD1069890ED4C
:40E34000010ABDEEC00A10EE100A00B20390FAF787FB18E00698007A012808D1F748B0F8AA00401C00B20390FAF77AFB0BE00698007A022807D1F148B0F8AA00401E00B203
:40E380000390FAF76DFB4BE11B20FEF7F9FE47E10698007A03281AD1E84890F842106C3000EB810090ED000A8DED050A9DED050AB5EEC00AF1EE10FA03D19FEDE10A8DEDF2
:40E3C000050A9DED050A082007F098F807E00698007A20B91FED2D0A082007F08FF81FE10698007A03280FD1D44890F842107C3000EB810090ED000A8DED030A9DED030A2F
:40E40000082007F07BF807E00698007A20B91FED3B0A082007F072F802E10698007A03281AD1C64890F84210743000EB810090ED000A8DED050A9DED050AB5EEC00AF1EE9A
:40E4400010FA03D19FEDBF0A8DED050A9DED050A082007F053F807E00698007A20B91FED4F0A082007F04AF8DAE00698007A03280FD1B24890F84210843000EB810090EDF1
:40E48000000A8DED030A9DED030A082007F036F807E00698007A20B91FED5E0A082007F02DF8BDE00698007A03280AD1069890ED010ABCEEC00A10EE100AC0B2039008F0ED
:40E4C000A7FBADE00698007A03280ED1069890ED010ABCEEC00A10EE100A80B20121039015F082FD089908701CE00698007A01280AD115F0CCFC401C80B20121039015F068
:40E5000073FD089908700DE00698007A022809D115F0BDFC401E80B20121039015F064FD089908707CE00698007A03280ED1069890ED010ABCEEC00A10EE100A80B2012143
:40E54000039015F069FD089908701CE00698007A01280AD115F097FC401C80B20121039015F05AFD089908700DE00698007A022809D115F088FC401E80B20121039015F040
:40E580004BFD089908704BE00698007A03280CD1069890ED010ABCEEC00A10EE100A80B2039015F051FD0899087039E00698007A03280CD1069890ED010ABCEEC00A10EEFB
:40E5C000100A80B2039015F056FD0899087027E00698007A03280CD1069890ED010ABCEEC00A10EE100A80B2039015F05FFD0899087015E00698007A03280CD1069890ED83
:40E60000010ABCEEC00A10EE100A80B2039015F068FD0899087003E007210898017000BF00BF049809B000BD86B04FF6FF7438214548DFF818C100DF0221454880F80811AB
:40E640000C228421434830F045FD002874D103213F4880F8081100BF224605A93A48DFF8F8C000DF012857D000208DF800008DF80D0001208DF80C0000208DF80E000598E3
:40E680000078002839D004AA01210598FEF77EFD05469DF8100068B100250599087821F0C3FE06460598837A427A9DF81010304621F0C0FE07F052FC08B1002504E0059876
:40E6C000007A032800D100250DB39DF80D00F0B90598007AD8B1059A07CA8DE8070001208DF80D008DF80C004FF47A649DF80E00401CC0B28DF80E0009E006F036FF30B18A
:40E700001348D0F890110120DFF850C000DF11480599F9F7F5FD9FE79DF8000000289BDD9DF80E00002850DD9DF80E00032817D102208DF80C0022E04AE00000081F0020C6
:40E74000CDCCCCBDCDCCCC3D780F002009F50308F03F0020F40E002099F6030881F303089DF80E00052803D106208DF80C0006E09DF80E00072802D110208DF80C009DF85F
:40E780000E00FF2805DA9DF80E00401CC0B28DF80E009DF80C1004AA6846FEF7F7FC9DF8100078B100208DF80E000599087821F03BFE06460598837A427A9DF81010304696
:40E7C00021F038FE4FF4FA6446E74FF6FF7443E70521334880F808110020DFF8C8C000DF00BFFEE72DE9F0472DED028B0546B0EE408A0E46174698464FF001092A48DFF826
:40E80000ACC000DFD0B900BF254890F8090140F00201234880F80911B0F814014FF6FF71884207DA1E48B0F81401401C81B21C48A0F8141100BF4FF000092CE01C48F9F7BF
:40E840004FFD04466CB1257084ED018A2672677284F80A800A2221461348DFF858C000DF19E000BF0E4890F8090140F004010C4880F80911B0F814014FF6FF71884207DA49
:40E880000748B0F81401401C81B20548A0F8141100BF4FF000094846BDEC028BBDE8F087F03F002005FE0308780F002001F50308F40E0020F5F5030831B52DED020B044659
:40E8C000FE4890EDD40ADDED000AB4EEE00AF1EE10FA00D3ACB100BF04226946F848006800F554700AF0C0FE20B99DED000AF34880EDD40A00BFF348C16B0220DFF8C8C3B4
:40E9000000DF3EBD31B52DED020B0446EB4890EDD30ADDED000AB4EEE00AF1EE10FA00DCACB100BF04226946E548006800F553700AF09AFE20B99DED000AE04880EDD30A45
:40E9400000BFE048C16B0220DFF87CC300DF3EBD31B52DED020B0446D84890ED2F0ADDED000AB4EEE00AF1EE10FA00D3A4B100BF04226946D2480068BC300AF075FE20B98C
:40E980009DED000ACD4880ED2F0A00BFCD48C16B0220DFF834C300DF3EBD31B52DED020B0446C64890ED2E0ADDED000AB4EEE00AF1EE10FA00DCA4B100BF04226946C0480E
:40E9C0000068B8300AF050FE20B99DED000ABB4880ED2E0A00BFBB48C16B0220DFF8E8C200DF3EBD10B54FF4C471B8482DF029FCB24890F82800B54981F8840128F0C7F803
:40EA0000B2498860012081F88001002081F881019FEDAF0A084680ED390A002005F08FFB01209FEDAB0AFFF7B8FF01209FEDA80AFFF78EFF01209FEDA60AFFF763FF012014
:40EA40009FEDA30AFFF738FF10BD10B5002425F0E1FC40B39F4800680078012800D128E09C4800680078022801D1142421E0994800680078052801D128241AE09548006888
:40EA80000078032801D13C2413E0924800680078062801D150240CE08E4800680078082807D1642405E025F0CDFC10B1874890F88541204610BD10B5844890F881018649F0
:40EAC0000978884203D0FFF7C0FF8449087010BD70B52DED028B044612F05CFB00287DD1002596E07548C03000EB8400D0ED000AB0EE600A28460FF024FE7048C03000EBA4
:40EB00008400D0ED000AB0EE600A28460FF02BFC6A48C83000EB8400D0ED000AB0EE600A28460FF032FE6548C83000EB8400D0ED000AB0EE600A28460FF08AFC5F48D030EC
:40EB400000EB8400D0ED000AB0EE600A28460FF040FE5A48D03000EB8400D0ED000AB0EE600A28460FF0CDFC5448D83000EB8400D0ED000AB0EE600A28460FF05DFE4F4855
:40EB8000D83000EB8400D0ED000AB0EE600A28460FF012FD4949E031085D29460FF070FE4649E231085D29460FF089FE25F032FC08B34249E0310A5D891C095D501800EB54
:40EBC000D071491000EE101AB8EEC00AB0EE408ABCEEC80A10EE101AC8B200E01DE021460FF05BFBBCEEC80A10EE101AC8B221460FF086FB0BE03149E031085D21460FF08E
:40EC00004CFB2E49E231085D21460FF079FB681CC5B2022DFFF666AFA3E02848C03000EB8400D0ED000AB0EE600A20460FF089FD2248C03000EB8400D0ED000AB0EE600AEC
:40EC400020460FF090FB1D48C83000EB8400D0ED000AB0EE600A20460FF097FD1748C83000EB8400D0ED000AB0EE600A20460FF0EFFB1248D03000EB8400D0ED000AB0EEFE
:40EC8000600A20460FF0A5FD0C48D03000EB8400D0ED000AB0EE600A20460FF032FC0748D83000EB8400D0ED000AB0EE600A20460FF0C2FD0148D83012E00000081F00207B
:40ECC000A4030020F03F002081F30308B00F002000000000080300202F0300202E03002000EB8400D0ED000AB0EE600A20460FF063FCFE49085D21460FF0C2FDFB49891C16
:40ED0000085D21460FF0DBFD25F084FBF0B1F7490A5D891C095D501800EBD071491000EE101AB8EEC00AB0EE408ABCEEC80A10EE101AC8B221460FF0B0FABCEEC80A10EEC4
:40ED4000101AC8B221460FF0DBFA0AE0E749085D21460FF0A2FAE549891C085D21460FF0CFFABDEC028B70BD01B500BF01226946DF48006800F5E9700AF076FC28B99DF863
:40ED80000000DA49E03981F8D20100BF08BD10B5032005F0D4F91FED320A002006F0AEFB0120FFF7E1FFD149E03991F84200FFF78FFE17201FF0E8FC10BD01B5B8B00020E9
:40EDC0003590349033903290319030902F902E901FED410A389880ED530A1FED430A389880ED560A1FED460A389880ED540A1FED480A389880ED580A1FED4B0A389880ED8E
:40EE0000550A1FED4D0A389880ED590A01203790FEE3379831F054FC9FEDB60B53EC102BCDE926019DED260B51EC100B31F040FACDE92C0137983690389890ED6A0B8DEDA1
:40EE4000200B9DED2C0B53EC102B9DED200B51EC100B31F085FCCDE92401389890ED680B8DED1A0B9DED2C0B53EC102B9DED1A0B51EC100B31F074FCCDE91C019DED2C0BDC
:40EE800053EC102B9DED1C0B51EC100B31F068FCCDE92001389890ED660B8DED140B9DED2C0B53EC102B9DED140B51EC100B31F057FCCDE916019DED2C0B53EC102B9DEDDA
:40EEC000160B51EC100B31F04BFCCDE918019DED2C0B53EC102B9DED180B51EC100B31F03FFCCDE91C01389890ED640B8DED0E0B9DED2C0B53EC102B9DED0E0B51EC100B6E
:40EF000031F02EFCCDE910019DED2C0B53EC102B9DED100B51EC100B31F022FCCDE912019DED2C0B53EC102B9DED120B51EC100B31F016FCCDE914019DED2C0B53EC102B0C
:40EF40009DED140B51EC100B31F00AFCCDE91801389890ED620B8DED080B9DED2C0B53EC102B9DED080B51EC100B31F0F9FBCDE90A019DED2C0B53EC102B9DED0A0B51EC36
:40EF8000100B31F0EDFBCDE90C019DED2C0B53EC102B9DED0C0B51EC100B31F0E1FBCDE90E019DED2C0B53EC102B9DED0E0B51EC100B31F0D5FBCDE910019DED2C0B53EC86
:40EFC000102B9DED100B51EC100B31F0C9FBCDE91401389890ED600B8DED020B9DED2C0B53EC102B9DED020B51EC100B31F0B8FBCDE904019DED2C0B53EC102B9DED040B5D
:40F0000051EC100B31F0ACFBCDE906019DED2C0B53EC102B9DED060B51EC100B31F0A0FBCDE908019DED2C0B53EC102B9DED080B51EC100B31F094FBCDE90A019DED2C0BE8
:40F0400053EC102B9DED0A0B51EC100B31F088FBCDE90C019DED2C0B53EC102B9DED0C0B51EC100B31F07CFBCDE91001389890ED5E0B8DED000B9DED2C0B53EC102B9DED25
:40F08000000B51EC100B31F06BFBCDE902019DED2C0B53EC102B9DED020B51EC100B31F05FFBCDE904019DED2C0B53EC102B9DED040B51EC100B31F053FBCDE906019DED6B
:40F0C0002C0B53EC102B9DED060B51EC100B31F047FBCDE908019DED2C0B53EC102B9DED080B51EC100B31F03BFB07E0E81F0020A40300200000000000002440CDE90A01C9
:40F100009DED2C0B53EC102B9DED0A0B51EC100B31F026FBCDE90C019DED2C0B53EC102B9DED0C0B51EC100B31F01AFBCDE90E019DED100B53EC102B9DED0E0B51EC100B4F
:40F1400030F0FAFFCDE912019DED140B53EC102B9DED120B51EC100B30F0EEFFCDE916019DED180B53EC102B9DED160B51EC100B30F0E2FFCDE91A019DED1C0B53EC102B8A
:40F180009DED1A0B51EC100B30F0D6FFCDE91E019DED200B53EC102B9DED1E0B51EC100B30F0CAFFCDE922019DED240B53EC102B9DED220B51EC100B30F0BEFFCDE9260186
:40F1C000389890ED6C0B8DED240B9DED240B53EC102B9DED260B51EC100B30F0ADFFCDE92A01389890ED7A0B8DED200B9DED2C0B53EC102B9DED200B51EC100B31F0B0FA25
:40F20000CDE92401389890ED780B8DED1A0B9DED2C0B53EC102B9DED1A0B51EC100B31F09FFACDE91C019DED2C0B53EC102B9DED1C0B51EC100B31F093FACDE9200138981C
:40F2400090ED760B8DED140B9DED2C0B53EC102B9DED140B51EC100B31F082FACDE916019DED2C0B53EC102B9DED160B51EC100B31F076FACDE918019DED2C0B53EC102B78
:40F280009DED180B51EC100B31F06AFACDE91C01389890ED740B8DED0E0B9DED2C0B53EC102B9DED0E0B51EC100B31F059FACDE910019DED2C0B53EC102B9DED100B51EC04
:40F2C000100B31F04DFACDE912019DED2C0B53EC102B9DED120B51EC100B31F041FACDE914019DED2C0B53EC102B9DED140B51EC100B31F035FACDE91801389890ED720B3C
:40F300008DED080B9DED2C0B53EC102B9DED080B51EC100B31F024FACDE90A019DED2C0B53EC102B9DED0A0B51EC100B31F018FACDE90C019DED2C0B53EC102B9DED0C0B0C
:40F3400051EC100B31F00CFACDE90E019DED2C0B53EC102B9DED0E0B51EC100B31F000FACDE910019DED2C0B53EC102B9DED100B51EC100B31F0F4F9CDE91401389890EDD3
:40F38000700B8DED020B9DED2C0B53EC102B9DED020B51EC100B31F0E3F9CDE904019DED2C0B53EC102B9DED040B51EC100B31F0D7F9CDE906019DED2C0B53EC102B9DEDCA
:40F3C000060B51EC100B31F0CBF9CDE908019DED2C0B53EC102B9DED080B51EC100B31F0BFF9CDE90A019DED2C0B53EC102B9DED0A0B51EC100B31F0B3F9CDE90C019DEDEA
:40F400002C0B53EC102B9DED0C0B51EC100B31F0A7F9CDE91001389890ED6E0B8DED000B9DED2C0B53EC102B9DED000B51EC100B31F096F9CDE902019DED2C0B53EC102B83
:40F440009DED020B51EC100B31F08AF9CDE904019DED2C0B53EC102B9DED040B51EC100B31F07EF9CDE906019DED2C0B53EC102B9DED060B51EC100B31F072F9CDE9080144
:40F480009DED2C0B53EC102B9DED080B51EC100B31F066F9CDE90A019DED2C0B53EC102B9DED0A0B51EC100B31F05AF9CDE90C019DED2C0B53EC102B9DED0C0B51EC100B3E
:40F4C00031F04EF9CDE90E019DED100B53EC102B9DED0E0B51EC100B30F02EFECDE912019DED140B53EC102B9DED120B51EC100B30F022FECDE916019DED180B53EC102B5A
:40F500009DED160B51EC100B30F016FECDE91A019DED1C0B53EC102B9DED1A0B51EC100B30F00AFECDE91E019DED200B53EC102B9DED1E0B51EC100B30F0FEFDCDE9220166
:40F540009DED240B53EC102B9DED220B51EC100B30F0F2FDCDE92601389890ED7C0B8DED240B9DED240B53EC102B9DED260B51EC100B30F0E1FDCDE928016421369890FBDF
:40F58000F1F201FB120008BB9DED2A0B51EC100B30F0A0FD01466422369890FBF2F2521E389800F5027040F822109DED280B51EC100B30F08FFD01466422369890FBF2F2DD
:40F5C000521E389800F50C7040F82210389890ED000AB1EE400A8DED250A259831F0B6FBCDE926019DED2A0B53EC102B9DED260B51EC100B31F0B2F92AD23598401C80B22C
:40F6000035909DED350AB8EE400ADFEDFE0A00E028E2B4EEE00AF1EE10FA1BDD389890ED530AB5EEC00AF1EE10FA13D19DED2C0B51EC100B30F04EFD00EE100AB1EE400AC8
:40F64000F3EE040A30EE200A389880ED530A01E000203590389890ED000AB1EE400A8DED250A259831F072FBCDE926019DED2A0B53EC102B9DED260B51EC100B31F06EF90E
:40F6800026D23498401C80B234909DED340AB8EE400ADFEDDC0AB4EEE00AF1EE10FA19DD9DED2C0B51EC100B30F014FD00EE100AF1EE400A9DED340AB8EE400AB2EE041A6E
:40F6C000C0EE011A30EEA10A389880ED520A01E000203490389890ED010AB1EE400A8DED250A259831F032FBCDE926019DED2A0B53EC102B9DED260B51EC100B31F02EF9B4
:40F7000028D23198401C80B231909DED310AB8EE400AF1EE040AB4EEE00AF1EE10FA1BDD389890ED540AB5EEC00AF1EE10FA13D19DED2C0B51EC100B30F0CCFC00EE100ABA
:40F74000B1EE400AF6EE000A30EE200A389880ED540A01E000203190389890ED030AB1EE400A8DED250A259831F0F0FACDE926019DED2A0B53EC102B9DED260B51EC100B30
:40F7800031F0ECF828D22F98401C80B22F909DED2F0AB8EE400AF1EE040AB4EEE00AF1EE10FA1BDD389890ED550AB5EEC00AF1EE10FA13D19DED2C0B51EC100B30F08AFC84
:40F7C00000EE100AB1EE400AF6EE000A30EE200A389880ED550A01E000202F9038980068259031F0B3FACDE926019DED280B53EC102B9DED260B51EC100B30F075FF26D218
:40F800003398401C80B233909DED330AB8EE400ADFED7C0AB4EEE00AF1EE10FA19DD389890ED560AB5EEC00AF1EE10FA11D19DED2C0B51EC100B30F04DFC00EE100AF3EEE8
:40F84000040A30EE600A389880ED560A01E00020339038980068259031F078FACDE926019DED280B53EC102B9DED260B51EC100B30F03AFF24D23298401C80B232909DEDF7
:40F88000320AB8EE400ADFED5F0AB4EEE00AF1EE10FA17DD9DED2C0B51EC100B30F01AFC00EE900A9DED320AB8EE400AB2EE041AC0EE011A30EEE10A389880ED570A01E0E2
:40F8C0000020329038984068259031F03FFACDE926019DED280B53EC102B9DED260B51EC100B30F001FF26D23098401C80B230909DED300AB8EE400AF1EE040AB4EEE00A1D
:40F90000F1EE10FA19DD389890ED580AB5EEC00AF1EE10FA11D19DED2C0B51EC100B30F0D9FB00EE100AF6EE000A30EE600A389880ED580A01E0002030903898C068259069
:40F9400031F004FACDE926019DED280B53EC102B9DED260B51EC100B30F0C6FE26D22E98401C80B22E909DED2E0AB8EE400AF1EE040AB4EEE00AF1EE10FA19DD389890EDFC
:40F98000590AB5EEC00AF1EE10FA11D19DED2C0B51EC100B30F09EFB00EE100AF6EE000A30EE600A389880ED590A01E000202E90389890ED5C0AB1EE400A8DED250A2598FB
:40F9C00031F0C4F9CDE926019DED2A0B53EC102B9DED260B51EC100B30F0C0FF19D29DED2A0B51EC100B30F075FB3899C1F870019DED2C0B51EC100B30F06CFB00EE100AEC
:40FA000002E0000000004843B1EE400A389880ED5A0A3898D0F87401259031F097F9CDE926019DED280B53EC102B9DED260B51EC100B30F059FE11D29DED280B51EC100BC6
:40FA400030F048FB3899C1F874019DED2C0B51EC100B30F03FFB3899C1F86C013798401C80B237903798B0F57A7F7FF7D2A9389890ED540AB5EEC00AF1EE10FA0BD038988C
:40FA800090ED540A80ED5A0A389890ED010AB1EE400A80ED5C0A389890ED580AB5EEC00AF1EE10FA09D0389890ED580A80ED5B0A389890ED010A80ED5D0A389890ED530A51
:40FAC000B5EEC00AF1EE10FA61D0389890ED560AB5EEC00AF1EE10FA59D0389890ED5A0AD0ED530AB7EE001A70EEC10AB4EEE00AF1EE10FA4BDC389890ED5B0AD0ED560A35
:40FB0000B7EE001A70EE810AB4EEE00AF1EE10FA3DD3389890ED530AD0ED520A30EE600A8DED230A239831F011F9CDE924019DED240B2DF0E5FC8DED260B9FEDFD0B53ECB0
:40FB4000102B9DED260B51EC100B30F007FF1ED3389890ED560AD0ED570A30EE600A8DED230A239831F0F2F8CDE924019DED240B2DF0C6FC8DED260B9FEDED0B53EC102B44
:40FB80009DED260B51EC100B30F0E8FE03D22320E94981F87E01389890ED550AB5EEC00AF1EE10FA04D19FEDE50A389880ED550A389890ED590AB5EEC00AF1EE10FA04D121
:40FBC0009FEDDF0A389880ED590A39B000BD70B52DED088B064600246FE09FEDDA0BB0EE408AF0EE608A9FEDD70BB0EE409AF0EE609A002551E006F1400000EB850090EDE0
:40FC0000000A10EE101A084631F0A0F841EC1B0B04EB440000EBC400CC4901EBC00000EBC50090ED001BB0EE410AF0EE610A53EC102B51EC1B0B30F093FD53EC182B30F0EC
:40FC40007BFA41EC180B06F16C0000EB850090ED000A10EE101A084631F078F841EC1B0B04EB440000EBC400B84901EBC00000EBC50090ED001BB0EE410AF0EE610A53ECC3
:40FC8000102B51EC1B0B30F06BFD53EC192B30F053FA41EC190B681CC5B20B2DABDB06F5BC7000EBC40080ED008B06F5DC7000EBC40080ED009B601CC4B2082C8DDBBDEC21
:40FCC000088B70BDA24A92F82810022914D19FEDA10A80ED000A9FEDA00A80ED010A9FED9F0A80ED020A9FED9E0A80ED030A9FED9D0A80ED040A6FE00D2914D19FED950A8B
:40FD000080ED000A9FED940A80ED010A9FED930A80ED020A9FED920A80ED030A9FED910A80ED040A58E00C2914D19FED8A0A80ED000A9FED890A80ED010A9FED880A80EDB9
:40FD4000020A9FED870A80ED030A9FED860A80ED040A41E0032914D19FED7E0A80ED000A9FED7D0A80ED010A9FED7C0A80ED020A9FED7B0A80ED030A9FED7A0A80ED040A60
:40FD80002AE0012914D19FED730A80ED000A9FED720A80ED010A9FED710A80ED020A9FED720A80ED030A9FED710A80ED040A13E09FED680A80ED000A9FED670A80ED010AC9
:40FDC0009FED660A80ED020A9FED670A80ED030A9FED660A80ED040A704770B52DED028B04466348FFF76EFF6148FFF7F0FE6048FEF7E3FF5E48D0ED550AB0EE600A204689
:40FE00000EF07FFB5A48D0ED550AB0EE600A20460EF0DFFC5648D0ED590AB0EE600A20460EF0CAFB5248D0ED590AB0EE600A20460EF002FD4E4890ED000AFFEE000A20EE0F
:40FE4000200AB0EE408A90ED5A0AD0ED530A30EE600AD0ED5C0A70EEC80A80EE801A80ED7E1AD0ED7E0A90ED531AB0EE480A00EEC10A80ED7F0A90ED000AB0EE408A90EDD3
:40FE80005B0AD0ED560A30EE600AD0ED5D0A70EEC80A80EE801A80ED801AD0ED800A90ED561AB0EE480A00EEC10A80ED810A90ED040AD0ED7E0A80EE201AB0EE418A9FED93
:40FEC000200A28EE000AB0EE408A9FED2A0AB4EEC08AF1EE10FA04DD9FED260AB0EE408A0AE0B7EE000AB4EEC08AF1EE10FA03D2B7EE000AB0EE408AB6EE000A38EE000A7E
:40FF0000BCEEC00A10EE100AC5B2214628460EF0C4F9214628460EF0B3FC154890ED040AD0ED800A80EE201AB0EE418A24E00000000000000000F03FB00F00200000C8C2D0
:40FF40000000C842000000000000000048000020081F002035FA0E3DC2B8323E00000000C2B8B23E8FDAA53B920A063F88C3643B3811002000007F431FED0F0A28EE000A76
:40FF8000B0EE408A1FED050AB4EEC08AF1EE10FA04DD1FED080AB0EE408A0AE0B7EE000AB4EEC08AF1EE10FA03D2B7EE000AB0EE408AB6EE000A38EE000ABCEEC00A10EED8
:40FFC000100AC5B2214628460EF09AF9214628460EF075FCBDEC028B70BD70B502460C4600201FED222AF0EE420A1FED242AB0EE421A1FED262AB0EE420A1FED282AF0EE2C
:020000040801F1
:40000000421A64B902F1400102F16C031FED2C2AB0EE420A9FEDF92AF0EE421A1CE0012C0CD102F1980102F1C403B0EE002AB0EE420AB7EE002AF0EE421A0DE0022C0BD17E
:4000400002F1F00102F58E73B3EE042AB0EE420AB2EE042AF0EE421AB5EEC00AF1EE10FA7EDD1FED422A81ED002A1FED442A83ED002A1FED462A82ED052A012082E002EE81
:40008000100AB8EE422AF2EE042A22EE222A02F1140505EB800585ED002A451ED84E06EB850595ED002AB5EEC02AF1EE10FA06DD1FED562A01EB800585ED002A09E0451E9F
:4000C000CF4E06EB850595ED002A01EB800585ED002A451ECA4E2C3606EB850595ED002AB5EEC02AF1EE10FA06D21FED642A03EB800585ED002A0AE0451EC14E2C3606EB05
:40010000850595ED002A03EB800585ED002A01EB800595ED002A451E01EB8505D5ED002A32EE622AF0EE420A03EB800595ED002A451E03EB8505D5ED002A32EE622AB0EE92
:40014000421AB1EE402AF4EEC20AF1EE10FA12D3F4EEE10AF1EE10FA0DDCB4EEC01A00E013E0F1EE10FA06DCB1EE612AB4EEC21AF1EE10FA04D22325A14E243E86F87E5198
:40018000451CE8B20B28FFF67AAF70BD10B500219C48FFF722FF01219A48FFF71EFF02219848FFF71AFF10BD10B5974890F82840042C17D006DC012C0DD0022C08D0032C23
:4001C00017D104E00C2C05D00D2C12D101E000BF00BF00BF00BF9FED8D0A8948243880ED390A0DE09FED8A0A8548243880ED390A06E01FEDA60A8248243880ED390A00BF10
:4002000000BF13F0FBFBB5EEC00AF1EE10FA09DD7B48243890ED390AFFEE000A20EE200A80ED390A10BD73B52DED020B04460D460A2C21D200BF05EB85027649096801F5CE
:40024000177101EBC20101EB84000422694609F00BFA50B99DED000A05EB85016E4800EBC10000EB840080ED000A00BF6B48C16B0220DFF8ACC100DF7FBD10B5FAF757FD80
:4002800010BD73B52DED020B04460D460A2C21D200BF05EB85025F49096801F59A7101EBC20101EB84000422694609F0DDF950B99DED000A05EB85015A4800EBC10000EBFD
:4002C000840080ED000A00BF5448C16B0220DFF850C100DF7FBD73B52DED020B04460D460A2C22D200BF05EB85024A49096801F5037101EBC20101EB84000422694609F0B0
:40030000B3F958B99DED000A05EB85014248503800EBC10000EB840080ED000A00BF3F48C16B0220DFF8F8C000DF7FBD10B5FAF7FEFC10BD73B52DED020B04460D460A2C75
:4003400021D200BF05EB850232490968E43101EBC20101EB84000422694609F085F958B99DED000A05EB85012E48503800EBC10000EB840080ED000A00BF2848C16B0220C0
:40038000DFF89CC000DF7FBD1F4A92F82810042917D006DC01290DD0022908D0032917D104E00C2905D00D2912D101E000BF00BF00BF00BF9FED150A114A243A82ED390AB6
:4003C0000DE09FED130A0E4A243A82ED390A06E09FED150A0A4A243A82ED390A00BF00BF032809D1064A243A92ED390AFFEE000A20EE200A82ED390A70470000920A863E1F
:40040000D40F002038110020081F002000008C4200004842A403002064210020F03F002081F303083C20002000000000FE4A92F82810062905D19FEDFD0AFD4A82ED390A60
:400440000CE0042905D11FED0E0AF94A82ED390A04E01FED120AF64A82ED390A062808D1F34A92ED390AFFEE000A20EE200A82ED390A7047B5EEC00AF1EE10FA01D201208E
:4004800070470020FCE7B5EEC00AF1EE10FA01DD012070470020FCE72DE9F04106460C4615460427E04890F828802868A0B926F06EFB28600020DF4908709FEDDF0A13F088
:4004C000BBFB20B1BFEE000ADC4880ED000A13F095FADB4880ED000AB8F1040F1FD009DCB8F1010F11D0B8F1020F0BD0B8F1030F1FD106E0B8F10C0F06D0B8F10D0F18D15F
:4005000001E000BF00BF00BF00BFCC4890ED000A5FED420A20EE200A84ED000A13E0C74890ED000A5FED460A20EE200A84ED000A09E0C24890ED000A5FED450A20EE200AD3
:4005400084ED000A00BF00BF41F28831286826F024FB20B1212030700127002595E040F6C411286826F019FBE0B1B2480078C8B99FEDB40A13F060FB20B99FEDB20A13F048
:4005800000FB78B10120AB490870AC4890ED000AFFEE000A20EE200A80ED000A26F0F7FA286072E0D4ED000AB0EE600AFFF76BFF68B113F023FAA248D0ED000A30EE600AE3
:4005C000DFEDA00AB4EEE00AF1EE10FA14DCD4ED000AB0EE600AFFF74DFFA8B113F00EFA9748D0ED000A30EE600ADFED970AB4EEE00AF1EE10FA07D203271FED750A84ED98
:40060000000A0020286040E0D4ED000AB0EE600AFFF739FF68B113F0F1F98948D0ED000A30EE600ADFED880AB4EEE00AF1EE10FA14D3D4ED000AB0EE600AFFF71BFF20B351
:4006400013F0DCF97E48D0ED000A30EE600ADFED7D0AB4EEE00AF1EE10FA16DD724890F89C0018B90120F9F7E5FD07E06E4890F89C00012802D10020F9F7DCFD03271FED54
:40068000960A84ED000A002028603846BDE8F08110B52DED048B0424654890F880010A287DD2DFE800F00506FD477CFC487CFBFA00BF5F4890F8810120B1102821D011283C
:4006C00035D110E011205A4981F8810113F096F9574880ED080AB6EE000A80ED390A00205349086024E0524A02F1E40101F19A00FFF7D2FE032803D110204D4981F8810179
:4007000016E006204A4981F88001022081F881010A2081F887010020086013F06FF9444880ED080AB6EE000A80ED390A00E000BF00BF1CE300BF3E4890F88101801E0B28EF
:4007400070D2DFE800F0066FB6FC5EDE6F6F6F6F8F003748006870B926F019FA34490860084690F885010A2805DD084690F88501C01F81F885012E4991F88001FFF756FE3F
:400780002B4908684FF47A6126F007FAB0B113F035F92748D0ED080A30EEC00A00E0F7E3B0EEC00ADFED290AB4EEE00AF1EE10FA04D221201E4981F87E0121E09FED210AA4
:4007C00013F03AFA20B11A4890F88001032809D09FED1C0A13F0D5F990B1154890F8800106280DD1B6EE000A114880ED390A06200F4981F881010C2081F88301002008606B
:40080000B4E2B6EE000A0A4880ED390A006818B926F0BDF90649086005490868C82126F0BCF915E0A1E20000081F002000002042B00F002031030020C2B8323E34030020AF
:4008400038030020C2B8B23DC2B8B2BD35FA0E3D38B1FE4890F88301FC4981F881010020086083E2F94991F88001FFF78DFDF748006818B926F08BF9F4490860F3490868BA
:400880004FF4FA7126F089F990B1B6EE000AEF4880ED390A0620ED4903E0CEE3E4E367E267E281F8810100200860042081F883015CE213F0A3F8F0EE409A4FF6FF71E448BA
:4008C00014F05EFAE148006818B926F060F9DF490860DE4908684FF4FA7126F05EF978B1DA4890ED510A80ED080A0720D74981F881010020086001F580700021416481648C
:4009000034E2D248006818B926F041F9CF490860CE4890F8870100EB8000400000EE100AB8EEC00AC94880ED390A90F8800103280AD1C64890ED390AFFEE000A00E044E09C
:4009400020EE200A80ED390A1FED420A13F074F920B1BE4890F88001062809D01FED470A13F00FF9B0B1B94890F88001032811D10220B64981F8810101F580700021416438
:40098000816413F03BF8B14880ED080A0020AF49086019E0AD4908684FF4FA7126F0FDF890B1B6EE000AA94880ED390A0620A74981F88101086826F012F9A449C8610020A4
:4009C0000860052081F88301D0E113F017F8F0EE409A4FF6FF719E4814F0D2F99B48006818B926F0D4F899490860984908684FF4FA7126F0D2F800287DD0944890ED510A38
:400A0000D0ED080A30EE608AB0EEC80AF0EE409A13F0B7F820B18D4890F8800103281FD01FED780A13F0ADF820B1884890F88001032815D0B0EEC80AF0EE409A13F0FCF82D
:400A400020B1824890F88001062809D01FED830A13F0F2F898B17D4890F8800106280ED102207A4981F88101084690ED510A80ED080A00F580700021416481640DE00720F8
:400A8000724981F88101084690ED510A80ED080A00F580700021416481646C4890F88701401E6A4981F88701084690F8800103285AD1084690ED070AF8EE400A9FED651AB1
:400AC00080EE810AC8EE000A90F88711243000EB8100C0ED000A604A92F842105B4A92F8870192F88731243202EB8302D2ED000AB0EE600A00E037E1FFF71CFC534890F865
:400B00008711243000EB8100D0ED000AB0EE600A0020FDF742FFFFF709FC4C4890F887117C3000EB810080ED000A4B4A92F84210464A92F8870192F887317C3202EB830286
:400B4000D2ED000AB0EE600AFFF7C5FB3F4890F887117C3000EB8100D0ED000AB0EE600A0020FDF7CFFE57E0384890ED070AF8EE400A9FED381A80EE810AC8EE000A90F8EB
:400B80008711503000EB8100C0ED000A324A92F842102E4A92F8870192F88731503202EB8302D2ED000AB0EE600AFFF76AFB274890F88711503000EB8100D0ED000AB0EED6
:400BC000600A0020FDF7C4FEFFF757FB1F4890F88711A83000EB810080ED000A1E4A92F842101A4A92F8870192F88731A83202EB8302D2ED000AB0EE600AFFF714FB1348B2
:400C000090F88711A83000EB8100D0ED000AB0EE600A0020FDF776FE0C4890F88701002813D10A4890F88001062817D10320074981F88001022081F88101B6EE000A084692
:400C400080ED390A0A2081F887018AE0B00F0020F410002000007A44081F0020B7EE000AF94880ED370A0920F849087026E0F6485030F64991F9001000EB810090ED000A17
:400C8000DFEDF30AB4EEE00AF1EE10FA10D2EF4890F9000000EE100AB8EEC00AF2EE040A20EE200AE84880ED370AFF20E7490870E6480078401E40B2E4490870E34890F9C2
:400CC00000000028D3DAB7EE000ADF4880ED360A0920DE49087026E0DB482430DB4991F9001000EB810090ED000ADFEDDA0AB4EEE00AF1EE10FA10DDD44890F9000000EE01
:400D0000100AB8EEC00AFAEE040A20EE200ACE4880ED360AFF20CD490870CC480078401E40B2CA490870C94890F900000028D3DAC54890ED370A80ED380A0520C24981F892
:400D400080010D2081F88101B6EE000A084680ED390A002081F887019FEDBF0A084680ED350A0020B849086000E000BF00BF99E100BFB54890F8810106281CD00D2802D066
:400D80000E287DD131E0FFF70FFA9FEDB10A12F028FF78B1B6EE000AAB4880ED390A0620A94981F881010E2081F8830125F0EFFEA54908603FE1B6EE000AA34880ED390AB6
:400DC000014608684FF4FA7125F0E7FE60B19E4890F883019C4981F881010020086012F00DFE994880ED080A25E1974890F88001052807D112F002FE9348D0ED080A70EEBF
:400E0000608A06E012F0FAFD8F48D0ED080A70EEC08A8D48006818B925F0B9FE8A4908609FED8E0AF4EEC08AF1EE10FA7EDD864890ED350AD0ED390A30EE200A80ED350A74
:400E400090F88701401C804981F88701B6EE000A084680ED390A0D2081F88101086825F0BEFE00EE100AB8EE400A5FED860A80EE209A754890F88001052818D1724800E0B5
:400E8000D8E090ED380A30EE090AF1EE040A30EE600A80ED380A90ED380AB5EEC00AF1EE10FA1AD29FED6C0A80ED380A15E0664890ED380A30EE490AF1EE040A30EE200AAC
:400EC00080ED380A90ED380AB5EEC00AF1EE10FA03DD9FED610A80ED380A5B4890F88701032839DB5848D0ED350A90F8870100EE100AB8EE400A80EE801A534880ED351AB3
:400F000090F88001052828D1554991F842004E49D1ED350AB0EE600A0DF037FC9FED4E0A494880ED350AB6EE000A00E031E080ED390A0020444981F88701022081F8800113
:400F40000D2081F8810125F022FE3F490860084690ED360A80ED380A6BE0414991F842003949D1ED350AB0EE600A0DF0EAFB9FED3A0A354880ED350AB6EE000A80ED390A0A
:400F80000820314981F880010F2081F8810150E087E02D4890ED390AB0EEC00ADFED310AB4EEE00AF1EE10FA07DA0146086825F016FE4EF66021884207D92120224981F866
:400FC0007E01092081F8800133E01F4890F88001022817D11C49086825F001FE00EE100AB8EE400AFFEE000A60EE200A1FEDE71A80EE810A1448D0ED380A30EE200A80ED54
:40100000390A16E01049086825F0E9FD00EE100AB8EE400AF7EE000A60EE200A1FEDF31A80EE810A0848D0ED380A30EE200A80ED390A00E000BF00BF34E002249FED060AC7
:40104000014880ED390A2DE0B00F00203003002035FA0E3D35FA0EBD0000000035FA8E3C081F002000008C42FFF790F8FE4890F87E0120B10920FC4981F8800110E0FB497E
:4010800091F84200FEF7A9FE1020F74981F8810103241FED0F0A084680ED390AFDF777FE00E000BF00BFF04890F88201EE4991F88111884214D0EC4890F88501401CEA4939
:4010C00081F88501084690F88501642802DD642081F88501E44890F88101E34981F88201E14890ED390AB5EEC00AF1EE10FA08D0D0ED390AB0EE600A01210846F9F73AF997
:4011000008E0D948D0ED390AB0EE600A00210120F9F730F92046BDEC048B10BD002070471FED330AD04880ED5B0A1FED350A80ED5D0A1FED370A80ED550A1FED390A80EDDA
:40114000530A1FED3B0A80ED590A1FED3D0A80ED570A704770B52DED048B0446F0EE408AB0EE609AF0EE419A0D46C04890F8300070280CD1F7EE000A80EEA80ADFEDBC0ADF
:4011800089EE201A20EE010A20EE298A60E0B74890F830000A280CD1F0EE000A80EEA80ADFEDB30A89EE201A20EE010A20EE298A4EE0A81E0C283DD2DFE800F02D3C063CE9
:4011C00013203C3C3C3C2F2EF0EE080A80EEA80ADFEDA70A89EE201A20EE010A20EE298A35E0DFEDA40A80EEA80ADFEDA10A89EE201A20EE010A20EE298A28E0DFED9E0A2A
:4012000080EEA80ADFED9A0A89EE201A20EE010A20EE298A1BE000BF00BFDFED980A80EEA80ADFED930A89EE201A20EE010A20EE298A0CE0DFED920A80EEA80ADFED8C0AC2
:4012400089EE201A20EE010A20EE298A00BF00BFB2EE040AB4EEC08AF1EE10FA04D2B2EE040AB0EE408A0AE09FED860AB4EEC08AF1EE10FA03DD9FED830AB0EE408A012C8D
:401280000AD17A4A92F84210BCEEC80A10EE102AD0B20DF0F5FA09E0744A92F84210BCEEC80A10EE102AD0B20DF009FBBDEC048B70BD00B52DED028B95B06B4890ED390A5E
:4012C0008DED140A25F063FC0E9004200C9012F014FB654880ED3B0AC068634948610846006988616848007827F0E6FB5E49C86025F04DFC5C490861084680690B9025F0B5
:401300006EFC4FF47A71B1FBF0F00F905648C06855494969401A00EE100AB8EEC00AF7EE000A20EE200A9FED591AC0EE010A9DED0F0AB8EEC00A20EE800A8DED130A0521BB
:4013400053489DED130A13F01BFD0521504808309DED140A13F014FD1CF0C1FC8DED0B0A1E214B4818389DED0B0A13F009FD494890ED000A8DED0B0A1E21454820389DEDE7
:401380000B0A13F0FDFC434890ED000A364880ED3A0A414800780EF079FB8DED0B0A05213B4808389DED0B0A13F0EAFC3B4800780EF029FD8DED050A05982FF0C7FCCDE98B
:4013C00006019DED060B2CF09BF88DED080B9DED080B51EC100B2EF07DFE05210B902C4810389DED0B0A13F0CBFC2048B0F8BE014FF4967190FBF1F000EE100AB8EEC00A9E
:401400008DED0D0A194890F82800062850D0174890F8280007284BD0134890F88001042804D0114890F88001072841D10E4890ED5D0ADFED1B0AB4EEE00AF1EE10FA38DDA7
:4014400090ED5B1A9DED0D0AF2EE040AF1EE041A41EEC00AB4EEE01AF1EE10FA28D20920014981F880011DE0B00F0020081F002000007A44CDCC4C406666A6408FC2753E4D
:401480009A99193F00007F43D806002052EC2F451C1100201043002093060020E406002000004842242081F87E01002081F881016EE0FE4890ED5D0ADFEDFD0AB4EEE00AF4
:4014C000F1EE10FA19D290ED5B1A9DED0D0AFAEE040AF1EE041A41EE800AB4EEE01AF1EE10FA55DD0920F14981F88001242081F87E01002081F881014AE0EC48D0F87401D3
:4015000007902FF023FCCDE908019DED080B2BF0F7FF8DED0A0B9FEDE70B53EC102B9DED0A0B51EC100B2FF01BF831D1DDED0D0AB1EE040AB1EE041A01EE200A8DED070AC8
:4015400007982FF003FCCDE90A01D848D0F86C0105902FF0FBFBCDE906019DED060B2BF0CFFF8DED080B9DED0A0B53EC102B9DED080B51EC100B2FF0F1F909D20920CB49F1
:4015800081F88001242081F87E01002081F88101C64890F88101062813D1C448806801460B900E9825F02AFBC0494968884241F2A783BE4890F88301BC4981F8810101F016
:4015C0009FBBBA4890F880010A2881F09783DFE810F030000A0040002804950B34020807950B8B0B760BB14890F87F0180B1AF4890F87F01AD4981F88001062081F881017E
:40160000002081F88301192048600E9888600EE00020A64981F88001062081F88101002081F883014FF47A7048600E98886001F066BB02209D4981F88001062081F8810151
:40164000002081F883014FF47A7048600E988860EDE7964890F88001944981F87F01084690F8810108287CD003DC38B1052879D15AE1092877D00B28F9D10BE006208B49B1
:4016800081F881010B2081F88301192048600E988860D0E18548806801460B900E9825F0ADFA41F28831884207D909207F4981F88001262081F87E0170E0804890F8280067
:4016C00006280ED07D4890F82800072809D0774890ED3B0ADFED7A0AB4EEE00AF1EE10FA13DC764890F82800062804D0734890F8280007280FD16D4890ED3B0ADFED710A84
:40170000B4EEE00AF1EE10FA05DDBBEE0E0A674880ED390A42E0694890F8280006280ED0664890F82800072809D0604890ED3B0ADFED650AB4EEE00AF1EE10FA17D35F4892
:4017400090F82800062804D05C4890F82800072813D1564890ED3B0ADFED5C0AB4EEE00A02E034E060E11AE0F1EE10FA05D2B3EE0E0A4E4880ED390A10E006204B4981F81F
:401780008101092081F883014FF47A7048600E9888609FED4F0A084680ED390A4BE10620424981F88101082081F88301192048600E988860BAEE000A084680ED390A454892
:4017C000007827F079F93949C1F82C0133E13B4890F82800062804D0384890F82800072810D13248C0683149D1F82C11401A00EE100AB8EEC00ADFED380AB4EEE00AF1EE8A
:4018000010FA31D32D4890F830000A2800D010E02648C0682549D1F82C11401A00EE100AB8EEC00ADFED2D0AB4EEE00AF1EE10FA1AD3224890F82800062851D01F4890F8E2
:40184000280007284CD01948C0681849D1F82C11401A00EE100AB8EEC00ADFED1F0AB4EEE00AF1EE10FA3BD2144890F842000B909DED140A0CF065FF06200C4981F881017D
:40188000052081F883014FF47A7048600E9888609DED140A084680ED390A0E48007827F00BF90249C1F82C013DE00000B00F0020000048C20000000000002040081F002036
:4018C000CDCCCC3CCDCC4C3DCDCCCCBCCDCC4CBD00000000D80600206CE7DBC57390EAC4F74890ED390A5FED0E0AB4EEE00AF1EE10FA0BD81FED0A0A80ED390A0920F049D3
:4019000081F88001272081F87E010CE09DED140ADFEDEC0A30EE600A8DED140A9DED140AE74880ED390A86E0E548D0ED390A9FEDE61A80EE810A8DED010A01982FF006FA1C
:40194000CDE902019DED020B2BF0DAFD8DED060BDB48D0F8640103902FF0F8F9CDE904019DED060B53EC102B9DED040B51EC100B2EF0F6FE9FEDD50B53EC102BCDE908012F
:401980009DED080B51EC100B2EF092FCCDE90A019DED0A0B51EC100B2EF09CFBC849C1F8FC00084690ED570ADFEDCA0A80EE201A80ED431AC84890F830000A2804D1B3EEA5
:4019C000090A8DED100A03E0B1EE040A8DED100A9DED100ADFEDC10A80EE201A9FEDC00A21EE000ABDEEC00AB8EEC00AB44880ED470AB0F87C0140F00400B149A1F87C01C2
:401A0000052081F88001062081F88101002081F883014FF47A7048600E9888601FED540A084680ED390A06E00020A549A1F87C0181F8800100BF00BFF9E5A14890F880012C
:401A40009F4981F87F01084690F8810108287CD003DC38B1052879D15AE1092877D00B28F9D10BE00620964981F881010B2081F88301192048600E988860D0E190488068CF
:401A800001460B900E9825F0B9F841F28831884207D909208A4981F88001282081F87E0170E08D4890F8280006280ED08A4890F82800072809D0824890ED3B0A5FED800A3F
:401AC000B4EEE00AF1EE10FA13DC834890F82800062804D0804890F8280007280FD1784890ED3B0A5FED890AB4EEE00AF1EE10FA05DDBBEE0E0A724880ED390A42E07648BB
:401B000090F8280006280ED0734890F82800072809D06B4890ED3B0A5FED950AB4EEE00AF1EE10FA17D36C4890F82800062804D0694890F82800072813D1614890ED3B0A72
:401B40005FED9E0AB4EEE00A02E034E060E11AE0F1EE10FA05D2B3EE0E0A594880ED390A10E00620564981F88101092081F883014FF47A7048600E9888601FEDAB0A0846A2
:401B800080ED390A4BE106204D4981F88101082081F88301192048600E988860B2EE000A084680ED390A4F48007826F085FF4449C1F82C0133E1484890F82800062804D0E4
:401BC000454890F82800072810D13D48C0683C49D1F82C11401A00EE100AB8EEC00ADFED420AB4EEE00AF1EE10FA31DC3A4890F830000A2800D010E03148C0683049D1F8E5
:401C00002C11401A00EE100AB8EEC00ADFED370AB4EEE00AF1EE10FA1ADC2F4890F82800062836D02C4890F82800072831D02448C0682349D1F82C11401A00EE100AB8EE60
:401C4000C00ADFED290AB4EEE00AF1EE10FA20DD214890F842000B909DED140A0CF095FD0620174981F88101052081F883014FF47A7048600E9888609DED140A084680EDBC
:401C8000390A1848007826F017FF0D49C1F82C013DE00B4890ED390ADFED150AB4EEE00AF1EE10FA26DB1FEDF60A80ED390A0920034981F88001292081F87E0127E000009D
:401CC000B00F0020CDCCCC3D0000C8420000000000408F4000007A44081F0020000070428DED2448D80600206CE7DB457390EA44000048429DED140A5FED0E0A30EE200A2D
:401D00008DED140A9DED140AFE4880ED390A86E0FC48D0ED390A1FED141A80EE810A8DED010A01982FF012F8CDE902019DED020B2BF0E6FB8DED060BF248D0F86401039078
:401D40002FF004F8CDE904019DED060B53EC102B9DED040B51EC100B2EF002FD1FED250B53EC102BCDE908019DED080B51EC100B2EF09EFACDE90A019DED0A0B51EC100B92
:401D80002EF0A8F9DF49C1F80401084690ED570A5FED300A80EE201A80ED451ADA4890F830000A2804D1B3EE090A8DED100A03E0B1EE040A8DED100A9DED100A5FED390AD8
:401DC00080EE201A1FED3A0A21EE000ABDEEC00AB8EEC00ACB4880ED490AB0F87C0140F02000C849A1F87C01032081F88001062081F88101002081F883014FF47A7048604E
:401E00000E9888609FEDC10A084680ED390A06E00020BC49A1F87C0181F8800100BF00BF05E4B84890F88001B64981F87F01084690F8810130B105287ED007287DD00A28DA
:401E40007CD10BE00620AF4981F881010A2081F88301192048600E988860C0E2A948806801460B900E9824F0C9FE42F21071884207D90920A34981F88001262081F87E01F1
:401E8000BCE0A14890F8280006280ED09E4890F82800072809D09B4890ED3B0A5FED770AB4EEE00AF1EE10FA13DC974890F82800062804D0944890F8280007282AD191484D
:401EC00090ED3B0ADFED920AB4EEE00AF1EE10FA20DD8D4890F82800062804D08A4890F8280007280BD100BF874890ED300AF0EE040A30EE600A834880ED390A7EE08248D6
:401F000090ED300AF2EE0E0A30EE600A7D4880ED390A73E07C4890F82800062812D07A4890F8280007280DD07648D0ED3B0A9FED790AF4EEC00A02E061E0F3E148E2F1EE25
:401F400010FA13D3704890F82800062804D06E4890F8280007282AD16A4890ED3B0A5FEDA70AB4EEE00AF1EE10FA20D2664890F82800062804D0644890F8280007280BD1D8
:401F800000BF614890ED320AF0EE040A30EE200A5C4880ED390A31E05B4890ED320AF2EE0E0A30EE200A574880ED390A26E00620544981F88101052081F8830140F6B83078
:401FC00048600E988860504890F8280007280AD14D48D0ED320A9FED500A20EE800A084680ED390A04E09FED490A464880ED390A00204449C1F82C01C1F83801EFE1414870
:40200000D0F82C01D0BB4548007826F055FD3D49C1F82C01084690ED530A80ED4C0A90ED550A80ED4D0A062081F88101072081F88301354890F82800072803D14FF47A701A
:40204000486003E04FF47A702E4948602D490E9888602D4890F82800062804D02A4890F8280007280BD1284890ED300AF2EE0E0A30EE600A234880ED390A52E10AE02248E8
:4020800090ED300A5FEDE60A30EE600A1D4880ED390A46E11B48D0F8380100287DD11F48007826F009FD1749C1F83801084690ED530A80ED4F0A90ED550A80ED500AD0F8E9
:4020C0003801D1F82C11401A0B9013F0C5F800EE100AF8EE400A9FED120A20EE800ADFED100A80EE201A074880ED481AD0F838010449D1F82C11401A00EE100AB8EEC00AA2
:4021000010E00000B00F0020081F002000000000CDCC4C3ECDCC4C3D9A99193FD806002000007A44DFEDFE0AB4EEE00AF1EE10FA7DD2FC4890F82800062804D0F94890F8A6
:402140002800072804D19FEDF80A8DED130A04E0F64890ED550A8DED130AF24890F82800072839D1F14890F884010B90ED4890ED0F0A8DED0A0AED4890ED4F0A8DED090A84
:402180000B989DED0A1ADDED130A9DED090A10F09AFCE64880ED3E0A00E0C2E090F884010B90E04890ED0F0A8DED0A0ADF4890ED4C0A8DED090A0B989DED0A1ADDED130A9C
:4021C0009DED090A10F07FFCD848D0ED3E0A30EEC00A80ED3E0A38E0D44890F884010B90D04890ED0F0A8DED0A0AD04890ED4F0A8DED090A0B989DED0A1ADDED130A9DEDB0
:40220000090A10F060FCC94880ED3E0A90F884010B90C44890ED0F0A8DED0A0AC34890ED4C0A8DED090A0B989DED0A1A00E06CE0DDED130A9DED090A10F045FCBB48D0ED24
:402240003E0A30EEC00A80ED3E0AB84890F884010B90B64890ED400AB1EE400A8DED0A0A90ED3E0A8DED090A0B999DED0A1A5FED540A9DED090A0120FEF76CFFAB4890EDB9
:402280003E0AF7EE000A80EE201A1FED600A31EE408AA74800780DF0F9FB5FED5F0A80EE201AA24890ED400AB1EE400AC0EE010A9C4890ED300A9FED9F1A10EE810AC8EEB9
:4022C000000A9A48C0ED3C0AB0F87C0140F008009649A1F87C010846B0F87C0140F01000A1F87C01062081F8800181F88101002081F883014FF47A7048600E9888601FED3D
:402300007D0A084680ED390A0BE01FED800A874880ED390A0920854981F880012B2081F87E015CE00620814981F88101052081F883010A2048600E9888600846D0ED390AED
:402340009FED7C1A80EE810A8DED010A01982EF0FDFCCDE902019DED020B2BF0D1F88DED060B7248D0F8640103902EF0EFFCCDE904019DED060B53EC102B9DED040B51EC25
:40238000100B2EF0EDF99FED6C0B53EC102BCDE908019DED080B51EC100B2DF089FFCDE90A019DED0A0B51EC100B2DF093FE5F49C1F80001084690ED570A5FEDA70A80EEC9
:4023C000201A80ED441ABAEE000A80ED390A06E000205649A1F87C0181F8800100BF00BFFEE3524890F88001504981F87F01084690F8810130B105287ED007287DD00A28CB
:402400007CD10BE00620494981F881010A2081F88301192048600E988860F1E34348806801460B900E9824F0E9FB42F21071884207D909203D4981F88001282081F87E010C
:40244000D3E0384890F8280006280ED0354890F82800072809D0354890ED3B0ADFED380AB4EEE00AF1EE10FA13D32E4890F82800062804D02B4890F8280007282AD12B48A8
:4024800090ED3B0ADFED2F0AB4EEE00AF1EE10FA20D2244890F82800062804D0214890F8280007280BD100BF1E4890ED320AF0EE040A30EE200A1D4880ED390A95E01948AF
:4024C00090ED320AF2EE0E0A30EE200A174880ED390A8AE0134890F82800062812D0114890F8280007280DD0104890ED3B0ADFED160AB4EEE00A02E078E082E3D1E3F1EE76
:4025000010FA2ADC074890F82800062804D0054890F82800072841D1044890ED3B0A15E0FF4680C6081F002039B40040B00F0020930600200000C8420000000000408F4099
:40254000CDCCCCBDCDCC4CBECDCC4CBD5FED040AB4EEE00AF1EE10FA20DDFE4890F82800062804D0FB4890F8280007280BD100BFF84890ED300AF0EE040A30EE600AF648CA
:4025800080ED390A31E0F34890ED300AF2EE0E0A30EE600AF04880ED390A26E00620EE4981F88101052081F8830140F6B83048600E988860E74890F8280007280AD1E54816
:4025C00090ED300ADFEDE50A20EE200A084680ED390A04E09FEDE20ADF4880ED390A0020DD49C1F82C01C1F8380166E3DA48D0F82C01D0BBDB48007826F05EFAD649C1F816
:402600002C01084690ED530A80ED4C0A90ED550A80ED4D0A062081F88101072081F88301CC4890F82800072803D14FF47A70486003E04FF47A70C8494860C7490E9888609A
:40264000C44890F82800062804D0C24890F8280007280BD1BF4890ED320AF2EE0E0A30EE200ABD4880ED390ACAE20AE0B94890ED320ADFEDBD0A30EE200AB74880ED390A48
:40268000BEE2B548D0F838010028EDD1B548007826F012FAB049C1F83801084690ED530A80ED4F0A90ED550A80ED500AD0F83801D1F82C11401A0B9012F0CEFD4FF47A718C
:4026C000B0FBF1F000EE100AB8EE400ADFEDA70A20EE200AA04880ED4A0AD0F838019E49D1F82C11401A00EE100AB8EEC00ADFEDA00AB4EEE00AF1EE10FA7DDD954890F88E
:402700002800062804D0934890F82800072804D11FED7B0A8DED130A04E08F4890ED550A8DED130A8B4890F82800072837D18A4890F884010B90874890ED0F0A8DED0A0A63
:40274000854890ED4F0A8DED090A0B989DED0A1ADDED130A9DED090A10F0B5F97E4880ED3E0A90F884010B907A4890ED0F0A8DED0A0A794890ED4C0A8DED090A0B989DED4F
:402780000A1ADDED130A9DED090A10F09CF97248D0ED3E0A30EEC00A80ED3E0A38E06E4890F884010B906B4890ED0F0A8DED0A0A694890ED4F0A8DED090A0B989DED0A1ACE
:4027C000DDED130A9DED090A10F07DF9624880ED3E0A90F884010B905E4890ED0F0A8DED0A0A5D4890ED4C0A8DED090A0B989DED0A1ADDED130A00E0F6E19DED090A10F07D
:4028000062F95548D0ED3E0A30EEC00A80ED3E0A514890F884010B904F4890ED420A8DED0A0A90ED3E0A8DED090A0B999DED0A1ADFED4E0A9DED090A0220FEF78BFC46483E
:4028400090ED3E0AF7EE000A80EE201A9FED440A31EE408A474800780DF018F9DFED430A80EE201A3C4890ED420AC0EE010A394890ED320A1FEDD11A10EE810AC8EE000AE3
:402880003548C0ED3D0AB0F87C0140F040003249A1F87C010846B0F87C0140F08000A1F87C010846D0ED3F0A90ED410A30EE800A80ED3F0A90ED3F0AF0EE000A80EE201A78
:4028C00080ED3F1AD0ED400A90ED420A30EE800A80ED400A90ED400AF0EE000A80EE201A80ED401AD0ED430A90ED450A30EE800A80ED430A90ED430AF0EE000A80EE201A33
:4029000080ED431A90ED440AD0ED460A30EE200A80ED440A90ED440AF0EE000A80EE201A80ED441A90ED470AD0ED490A30EE200A80ED470A90ED470AF0EE000A80EE201A8A
:4029400080ED471A90ED470ADFED0B0A20EE200A14E00000081F0020B00F00209A99193F00000000D80600200000484200007A44FF468046930600205F43BA3980ED470AA0
:4029800090ED480AD0ED4A0A30EE200A80ED480A90ED480AF0EE000A80EE201A80ED481A90ED480A5FED0C0A20EE200A80ED480A90ED440AD0ED430A70EE600A90ED400A76
:4029C00090ED3F1A30EE411A80EE810A8DED0B0A9DED0B0A08F0D2FDFE4890ED440AFE48D0ED700AFB4890ED401A00EEC10A8DED0B0A9DED0B0A08F097FDF64890ED480A72
:402A0000D0ED470A70EE600A90ED400A90ED3F1A30EE411A80EE810A8DED0B0A9DED0B0A08F068FDEB4890ED480AEB48D0ED720AE84890ED401A00EEC10A8DED0B0A9DEDDF
:402A40000B0A08F03DFDE54800780DF01FF85FED390A80EE201AE04890ED700A21EE000AD0ED710AB2EE001A71EE600A80EE801A9FEDDB0A21EE000A8DED130A90F8280053
:402A8000062804D19FEDD70A8DED110A0DE0D24890F830000A2804D19FEDD20A8DED110A03E09FEDD10A8DED110ACA48D0ED3C0A9DED110A80EE201AC74890ED300A31EE28
:402AC000400A8DED120A9DED130ADFEDC50AB4EEE00AF1EE10FA10DD9DED120ADFEDC00AB4EEE00AF1EE10FA07DD90F842009FEDBF0A0B900BF06DFE1DE09DED130ADDED2F
:402B0000120AB4EEE00AF1EE10FA0ADDB24890F842000B909DED120AB1EE400A0BF059FE09E0AD4890F842000B909DED130AB1EE400A0BF04EFEA748D0ED3D0A9DED110A2B
:402B400080EE201AA44890ED320A31EE000A8DED120A9DED130ADFEDA20AB4EEE00AF1EE10FA10DD9DED120ADFED9D0AB4EEE00AF1EE10FA07DD90F842009FED990A0B90C2
:402B80000BF05AFE19E09DED130ADDED120AB4EEE00AF1EE10FA08DD8F4890F842000B909DED120A0BF048FE07E08B4890F842000B909DED130A0BF03FFE0820854981F852
:402BC0008001062081F88101002081F883014FF47A7048600E9888601FED9F0A084600E08DE080ED390A0BE01FEDA30A794880ED390A0920774981F880012B2081F87E0178
:402C00005BE00620734981F88101052081F883010A2048600E9888600846D0ED390A9FED701A80EE810A8DED030A03982EF08EF8CDE904019DED040B2AF062FC8DED080B7E
:402C40006448D0ED590A1FEDB71A80EE810A8DED050A05982EF07AF8CDE906019DED080B53EC102B9DED060B51EC100B2DF078FDCDE90A019DED0A0B51EC100B2DF02AFAAA
:402C80005449C1F80801084690ED570A5FEDC90A80EE201A80ED461AB2EE000A80ED390A0BE000204B49A1F87C0181F880011FEDD40A084680ED390A00BF00BF1FE0022065
:402CC0000C900620434981F88101002081F88301192048600E9888601FEDDF0A084680ED390AFEF71DFA0AE003200C901FEDE40A384880ED390AFCF74AF800E000BF00BF9A
:402D0000344890ED390AB5EEC00AF1EE10FA0AD090ED390A8DED0B0A012108469DED0B0AF7F728FB0AE02B4890ED390A8DED0B0A002101209DED0B0AF7F71CFB0C9815B0BD
:402D4000BDEC028B00BD10B50124224890F87E01B8B921F05FFB18B1FEF7ABFA04460EE021F070FB58B11C4890F82800072803D1FEF7D4F9044602E0FDF78AFC0446FBF74E
:402D80009AFE204601F0DBF9124890F87E0120B1104991F87E0101F0A9FE204610BD10B50C4890F880010A2849D2DFE800F0494A300548310648484B00BF0220054981F802
:402DC00081010020086010F019FE024880ED080A0EE00000B00F0020081F0020930600200000C8423333B33F3333B33E0000C8C290F88701401C8E4981F88701084690F8BF
:402E000087010A2802DD0A2081F887011DE000BF0D20874981F8810123F0B9FE844908609FED840A084680ED350A002081F88701084690F88501C01E81F8850105E000BF09
:402E400000BF00BFFBF7CEFD00BF00BF7A480021416481640020764981F87E01B6EE000A084680ED390A10BD10B521F0D3FA10B301F038FE2B2802D1FBF7B4FD1DE06C48D5
:402E800090F87F016A4981F88001062081F88101002081F883014FF47A70486023F077FE634988609FED630A084680ED390A002081F87E0101E0FFF772FF10BDB7EE000A5B
:402EC00070475B4890F87E01704710B55B48FCF7F9FE5A48FCF77BFE5848FBF76EFF10BD10B55648FCF7EEFE5448FCF770FE5348FBF763FF10BD4E4890F8800170474C48A9
:402F000090F88101704710B50424494890F88001012804D10620464981F8800186E04FF4FA714748008823F038FE00287ED023F02EFE434908803E4890F88001801E072803
:402F400072D2DFE800F0450571440471700000BF374890F88101801E0B2835D2DFE800F00634151F0B1A3434343410000620304981F8810129E00C202D4981F8810124E0E4
:402F800004202B4981F881011FE00720284981F881011AE00520264981F8810115E0244890F88001062807D10320214981F88001022081F8810106E005201D4981F88001E4
:402FC0000D2081F8810100E000BF00BF2DE000BF174890F88101062804D00D2807D00E281ED109E00D20124981F8810119E00E200F4981F8810114E00D4890F8800105287E
:4030000009D102200A4981F88001062081F8810105E00BE008E00820054981F8800100E000BF00BF01E000E000BF00BF204610BDB00F002000000000B01000203811002006
:403040003C03002070B541201CE0C41700EBD4646511CD4C54F82540C51700EBD5656D11A0EB45160125B5402C40C51700EBD5656D11A0EB45160125B540AC4200D103E023
:40308000411EC8B20028E0DC00BF70BD30B5C31700EBD3635C11BC4B183353F824300246C41700EBD4646411A0EB44150124AC4023430146C41700EBD4646511B24C18340E
:4030C00044F8253030BD13B50C4600BFAF49096801F5B07108190122694606F0C5FA18B99DF80010AA48015500BF1CBD13B50C4600BFA649096801F25F210819012269465C
:4031000006F0B2FA20B99DF80010A148FF30015500BF1CBD70B504469E480470E21704EBD2625311984A52F823202146E31704EBD3635B11A4EB43150123AB409A43204686
:40314000E31704EBD3635D118F4B43F82520E21704EBD26253118C4A0C3252F82320E31704EBD3635B11A4EB43150123AB409A43E31704EBD3635D11834B0C3343F82520CF
:40318000E21704EBD26253117F4A183252F82320E31704EBD3635B11A4EB43150123AB409A43E31704EBD3635D11774B183343F825200020FFF79AFF70BD30B50146CB178D
:4031C00001EBD3635C11704B53F82430CC1701EBD4646411A1EB44150124AC4023400BB1012030BD0020FCE76B49087070476A480078704770B52DED048B04460025422CD5
:4032000070D2DFE804F02122272C2D2E2F37424D586069737F88A3A8BBFEFDFCFBFAF9F8F7F6F5F4F3F2F1F0EFEEEDECEBEAE9E8E7E6E5E4E3E2E1E0DFDEDDDCDBDAD9D83D
:40324000D7D6D5D4D3D2D194F2E20DF0A3FF80F00105EDE221F0D6F880F00105E8E2E7E2E6E2E5E2F9F7BAFE08B1012000E000200546DDE20EF03FFE30B1F9F7A7FE08B1C9
:40328000012000E000200546D2E20EF034FE30B1F9F7B4FE08B1012000E000200546C7E20EF029FE30B1F9F7A1FE08B1012000E000200546BCE210F0EFFC012800D100E050
:4032C00000200546B4E210F0E7FC032801D1012000E000200546ABE2304890F83800012801D101E0A3E200200546A1E20EF003FE38B12A4890F8380008B9012000E0002071
:40330000054695E2254890F89000012800D100E0002005468CE20EF0EEFD38B11F4890F8900008B9012000E00020054680E21B4890F83800022804D0184890F890000228F0
:4033400001D1012000E00020054671E209F0E2FA80F001056CE21248007D60B90A48001F006900F48030B0F5803F04D002F0F6FD08B1012000E00020054659E20948007D6A
:4033800008B901203FE03DE0E8160020AC0300200825002048030020490300202C27002028280020402800203DE212E200E2F3E1EAE1DDE1D1E1C5E1BCE1B3E1A7E19EE191
:4033C00092E189E180E177E16EE165E15CE153E14AE141E138E12FE126E121E115E103E1DAE0CDE0C0E0B3E0A6E099E08CE082E077E06CE054E047E03AE029E01CE00FE065
:4034000006E002E00020054612E2F74805780FE2F7F773F808B1012000E00020054607E20DF04CFCB0EE408A9FEDF01ADFEDF00A0DF0C3FB0546FBE10DF040FCB0EE408AC5
:403440009FEDEC1ADFEDEC0A0DF0B7FB0546EFE103F052F8B0F57B4F07DB03F04DF84FF6FF71884201DA012000E000200546DFE103F003F828B1E1488078FE2801D00120E2
:4034800000E000200546D3E1DC488078FE2806D0F9F700FD18B101250020D9490872C7E1D6488078FE2805D0D648007810B103F0FAFD20B101251A20FFF796FE06E0FFF7CC
:4034C00096FE1A2802D10020FFF78EFEB0E1CE48007800F0B40008B1012000E000200546A6E1C948007800F0480008B1012000E0002005469CE1C5480088102801D00120F0
:4035000000E00020054693E10DF027FCB0EE408A9FEDB61ADFEDB80A0DF04FFB054687E10DF023FCB0EE408A9FEDB01ADFEDB20A0DF043FB05467BE10DF01FFCB0EE408A9C
:403540009FEDAA1ADFEDAC0A0DF037FB05466FE10DF0DCFBB0EE408A9FEDA41ADFEDA60A0DF02BFB054663E10CF045FCB0EE408A9FED9E1ADFEDA00A0DF01FFB054657E102
:403580000DF0CCFBB0EE408A9FED981ADFED9A0A0DF013FB05464BE120F03CFF18B3F7F7C6FBB0EE408AF7F797FB38EE400A10EE106A30462DF0CAFB41EC190BB0EE490A80
:4035C000F0EE690A29F09CFFB0EE408AF0EE608A9FED8F0B53EC102B51EC180B2DF0BEF900D2012500BF23E1F7F7A1FBDFED8A0AB4EEE00AF1EE10FA04DDF6F7E3F908B145
:40360000012000E00020054612E102F0A7FC20B903F0ECF908B9012000E00020054607E108F036FA054603E10EF065FC18B103F01FFE80F00105FBE0F6F76AFF08B10120C0
:4036400000E000200546F3E0F6F76FFF08B1012000E000200546EBE0F7F70FF808B1012000E000200546E3E0F7F745F808B1012000E000200546DBE0F7F777F808B10120C2
:4036800000E000200546D3E0F7F7A9F808B1012000E000200546CBE0F7F7DFF808B1012000E000200546C3E0F7F711F908B1012000E000200546BBE0F7F743F908B1012064
:4036C00000E000200546B3E0F7F779F908B1012000E000200546ABE0F7F7ABF908B1012000E000200546A3E00EF005FC30B1F7F70BFA08B1012000E00020054698E0F7F744
:403700001FFA08B1012000E00020054690E00EF0F2FB30B1F7F72FFA08B1012000E00020054685E0F7F746FA08B1012000E0002005467DE0F7F75AFA08B1012000E00020A2
:40374000054675E00EF0D7FB30B1F7F76BFA08B1012000E0002005466AE00EF0CCFB30B1F7F77CFA08B1012000E0002005465FE00DF08FFB06460DF00FFC06430EB10120C4
:4037800000E00020054653E00DF03EFC08B1012000E0002005464BE00EF0ADFB38B108F0F6FB012803D103F0D4FC00B901253FE0F6F744FE28B9F7F7F4FA10B9F7F70BFB25
:4037C00020B103F0C6FC08B9012000E0002005462EE00DF0BFFC20B91048007821F05EFAF0B101201DE000008D03002000FF7F4700A0254600007A4600000000D8C7002080
:40380000E42F0020C8040020A103002046070020000000000070A7400000FA45130700200020054604E003F010F9054600E000BF00BF05B100BF3DB9FE480078002807DD3F
:40384000FC480078844203D10120BDEC048B70BD0020FAE74FF00008C1464FF0010A4FF0500B0321F44880F8B81000248FE0F348005D04EB840101EBC401F14A02EB81019F
:4038800089680870ED48FF30005D00287DD0E21704EBD2625311EB4A52F82320E31704EBD3635B11A4EB431C012303FA0CF31A43E31704EBD3634FEA631CE24B43F82C20A6
:4038C000E21704EBD2625311DE4A0C3252F82320E31704EBD3635B11A4EB431C012303FA0CF31A43E31704EBD3634FEA631CD54B0C3343F82C2004EB840000EBC400D04967
:4039000001EB8000007BE0B1E21704EBD2625311CC4A183252F823202146E31704EBD3635B11A4EB431C012303FA0CF31A432046E31704EBD3634FEA631CC24B183343F875
:403940002C2023F024F9C04941F8240000BFE21704EBD2625311BB4A243252F823202146E31704EBD3635B11A4EB431C012303FA0CF39A432046E31704EBD3634FEA631C24
:40398000B04B243343F82C2000BF601CC4B2422CFFF66DAF4FF47A60DFF8B0C200DFA648D0F8DC100120DFF8A8C200DF4FF47A60DFF898C200DF00BF002259460320DFF82F
:4039C00094C200DF0646022E21D1DFF88CC200DF074607F00200D0B1002416E0002004EB840101EBC401964A02EB81018968087004EB840101EBC40102EB8101896808783D
:403A00002146FFF760FB601CC4B2422CE6DB0024AAE22046FFF7EEFB05462046FFF7CDFBA8427DD0002D7CD1A946E31704EBD3634FEA631C834B0C3353F82C304FEAE47C85
:403A400004EBDC6C4FEA6C1CA4EB4C1E4FF0010C0CFA0EFC03EA0C034FEAE47C04EBDC6C4FEA6C1CA4EB4C1E4FF0010C0CFA0EFC634501D04FF0010904EB840000EBC40033
:403A80006F4901EB800090F8330000F0010008B14FF0010904EB840000EBC400684901EB800090F8330000F0020020B108F0EEFD08B14FF0010904EB840000EBC4006049C7
:403AC00001EB800090F8330000F0040038B107F0E7FF10B920F0C9FC08B14FF0010904EB840000EBC400564901EB800090F8330000F0080020B1BAF1000F01D04FF00109C0
:403B000004EB840000EBC4004D4901EB800090F8330000F0100038B15048005D012801E010E010E000D18146B9F1010F0AD100204A4908554FF001082046FFF7EBFA3620C2
:403B4000F9F71EFB03E1E31704EBD3634FEA631C3C4B53F82C304FEAE47C04EBDC6C4FEA6C1CA4EB4C1E4FF0010C0CFA0EFC03EA0C034FEAE47C04EBDC6C4FEA6C1CA4EB51
:403B80004C1E4FF0010C0CFA0EFC6345DAD000203249085500BF02F0E1F9E8B1E21704EBD2625311274A243252F823202146E31704EBD3635B11A4EB431C012303FA0CF3FD
:403BC0001A432046E31704EBD3634FEA631C1D4B243343F82C201CE0E21704EBD2625311184A243252F823202146E31704EBD3635B11A4EB431C012303FA0CF39A432046E1
:403C0000E31704EBD3634FEA631C0E4B243343F82C20E21704EBD26253110A4A52F82320E31704EBD3635B11A4EB431C012303FA0CF315E04A030020F03F0020082500207E
:403C4000340F0408E8160020DC15002021F3030881F30308E1F3030829F303089A1500201A43E31704EBD3634FEA631CFE4B43F82C2022F08CFFFD4941F8240004EB84009C
:403C800000EBC400FA4901EB800080680078401C04EB840101EBC401F54A02EB81018968087004EB840000EBC400114601EB8000806800787E2808DD7E2004EB840101EBE0
:403CC000C40102EB81018968087000BF00BF02F045F901281DD1E21704EBD2625311E24A243252F823202146E31704EBD3635B11A4EB431C012303FA0CF31A432046E31716
:403D000004EBD3634FEA631CD74B243343F82C201CE0E21704EBD2625311D34A243252F823202146E31704EBD3635B11A4EB431C012303FA0CF39A432046E31704EBD363C8
:403D40004FEA631CC84B243343F82C2000BF002D7DD0E21704EBD2625311C34A0C3252F82320E31704EBD3635B11A4EB431C012303FA0CF31A40002A53D104EB840000EB6A
:403D8000C400BB4901EB8000406AE8BBE21704EBD2625311B44A0C3252F82320E31704EBD3635B11A4EB431C012303FA0CF31A43E31704EBD3634FEA631CAB4B0C3343F8FC
:403DC0002C204FF0010804EB840000EBC40001EB8000806800787E2811DA04EB840000EBC40001EB800080680078401C04EB840101EBC4019E4A02EB81018968087021461A
:403E00000120FFF773F900E00CE004EB840101EBC401974A02EB8101896808782146FFF752F95BE004EB840202EBC402904B03EB8202516A8D4A52F8240022F0AEFEE8B39C
:403E4000E21704EBD2625311874A0C3200E083E052F82320E31704EBD3635B11A4EB431C012303FA0CF31A43E31704EBD3634FEA631C7D4B0C3343F82C204FF0010804EB51
:403E8000840000EBC4007A4901EB8000806800787E2811DA04EB840000EBC40001EB800080680078401C04EB840101EBC401704A02EB810189680870214600E00EE0012058
:403EC000FFF714F904EB840101EBC401684A02EB8101896808782146FFF7F5F804EB840202EBC402624B03EB8202127BA2B3E21704EBD26253115C4A183252F82320E3179E
:403F000004EBD3635B11A4EB431C012303FA0CF31A400ABB02F022F810B901F026FBE0B104EB840000EBC400514901EB8000806A68B104EB840202EBC4020B4603EB820235
:403F4000916A4A4A52F8240022F027FE20B12046FFF79CF84FF0010804E02046FFF796F84FF00108601CC4B2422CFFF652ADB8F1010F0BD13F48D0F8DC100120DFF8F8C01A
:403F800000DF4FF000083620F9F7FAF84FF0000AFFF758F804460FE5002107E0324850F8210008B101207047481CC1B20329F5DB0020F8E7002108E02B48183050F821005B
:403FC00008B101207047481CC1B20329F4DB0020F8E770B541201DE0C41700EBD4646511214C183454F82540C51700EBD5656D11A0EB45160125B5402C40C51700EBD56511
:404000006D11A0EB45160125B540AC4200D103E0411EC8B20028DFDC00BF70BD70B5002401F09CFFF8B1412437E0E31704EBD3635D110D4B0C3353F82530E51704EBD565D4
:404040006D11A4EB45160125B5402B40E51704EBD5656D11A4EB45160125B540AB421AD104EB84030AE01BE0E8160020DC150020340F0408F03F002081F3030803EBC40376
:40408000294D05EB830393F83330102B03D1274B1B5D03B903E0601EC4B2002CC5DC00BF204670BD0121214A1154704701460020FF2906DA1D4A525C0AB1012200E000226E
:4040C0001046704700B5002304E01846FFF7EAFF581CC3B2422BF8DB00BD0EB5144A07CA8DE807001BF079FD1DF020FB0C226946FF201BF03EFD0EBD014601EB810000EB11
:40410000C100094A52F820007047014601EB810000EBC100044A02EB80000079704770470449087070470000340F04089A1500209C1C04084A030020FE48007B7047FD49BF
:404140000873704710B52DED088BF0EE409AF0EE608A04469FEDF80AF0EE40AA9FEDF70AC0EE290AB0EE608AB1EE000A28EE800AC0EE080AB0EE60AA9FEDEF0AB0EE40BAB7
:40418000204622F02CFDBCEEC80A10EE101AB0FBF1F201FB120000EE100AB8EE400AB0EE409AB5EE000A28EE000AB4EEC90AF1EE10FA15D8B6EE080A28EE000AB4EEC90A4B
:4041C000F1EE10FA0CDDBFEE000A2AEE000AB0EE40AAB0EE000A28EE800AB0EE40BA0EE0B6EE080A28EE000AB4EEC90AF1EE10FA05D8B9EE000A28EE800AB0EE40BAB0EE26
:404200004B0A0AEE090AF0EE40AAB0EE6A0ABDEC088B10BD70B52DED068B04460D46284622F0DDFC00EE100AB8EE400AB0EE408A9FEDC20AC8EE000AB0EE608A94ED000AEA
:40424000D4ED020A00EE880ADFEDBD0A68EE200A20EE200A10EE101A08462CF077FD41EC1A0BB0EE4A0AF0EE6A0A2AF009F8B0EE409AF0EE609A51EC190B2BF02BFF08EE03
:40428000100A94ED040A20EE080AB0EE408AB0EE480ABDEC068B70BD2DE9F0412DED028B05460F4690460024002600BF32E0322108FB01F000EE100AB8EEC00ADFED9F0AC3
:4042C00080EE201A05F1300000EB840090ED000A30EE410A05F1300000EB840080ED000A08FB01F000EE100AB8EEC00ADFED930A80EE201A05F1700000EB840090ED000AAC
:4043000030EE410A05F1700000EB840080ED000A601CC4B2082CCADB0024D8E007F1300000EB840090ED000A07F1700000EB8400D0ED000A30EE600AF0EE000A20EE200ABD
:40434000B0EE408A05F1300000EB840090ED000A07F1300000EB8400D0ED000A30EE600A05F1900000EB860080ED000A05F1900000EB860090ED000AC0EE080A9FED710A20
:4043800020EE800A05F1CC0000EB860080ED000A05F1500000EB840090ED000A05F1100000EB8400D0ED000A30EE600A07F1500000EB8400D0ED000A07F1100000EB8400C6
:4043C00090ED001A70EEC10A80EE201A05F5847000EB860080ED001AB7EE000AC0EE080A05F5A27000EB8600C0ED000A701CC6B20F2E6ADA07F17000611C00EB810090ED79
:40440000000A07F1300000EB8400D0ED000A30EE600AF0EE000A20EE200AB0EE408A05F1700000EB810090ED000A07F1700000EB8100D0ED000A30EE600A05F1900000EB17
:40444000860080ED000A05F1900000EB860090ED000AC0EE080A9FED3B0A20EE800A05F1CC0000EB860080ED000A05F1500000EB810090ED000A05F1100000EB8400D0ED83
:40448000000A30EE600A07F1500000EB8100D0ED000A07F1100000EB840090ED001A70EEC10A80EE201A05F5847000EB860080ED001AB7EE000AC0EE080A05F5A27000EBC4
:4044C0008600C0ED000A701CC6B2601CC4B2082CFFF624AF1C4B0F221C4901F13C0012F0B0FD1B4B0F2219493C3901F1780012F0A8FD154890ED010A0E4880ED1D0A12480B
:4045000090ED000A0B4880ED230A114890ED010ADFED100A30EEC00AD0ED000A80EE201A044880ED261A0F210848783812F06FFD004811E02C1700200000000000007A44F8
:40454000DB0FC9400000B44350030020DC180020580300200000344380ED200ABDEC028BBDE8F08170B52DED028B0446B0EE408A0D46207800F0100000280AD094ED020AFD
:4045800084ED030A84ED028AA078082802D10420208086E0207800F00100D8B394ED020AD4ED030AB4EEE00AF1EE10FA20DD94ED020AFD48817804F1500000EB810080ED71
:4045C000000AFA49486822F00AFB00EE100AB8EE400A5FED260A80EE201AF348817804F1700000EB810080ED001A0020E07002E0E078401CE070E0782179884251DD208817
:4046000040F002002080208820F0010020800020E07046E0FFE7207800F00200F0B394ED020AD4ED030AB4EEE00AF1EE10FA1ED294ED020AA17804F1100000EB810080ED62
:40464000000ADA49486822F0CAFA00EE100AB8EE400A5FED460A80EE201AA17804F1300000EB810080ED001A0020E07002E0E078401CE070E0782179884212DD208840F041
:4046800001002080208820F002002080A078401CA0700020E0700DB1207900E001E0401E2071BDEC028B70BD10B52DED028BF0EE408AB0EE608ABD49486822F090FAB0F50E
:4046C0007A7F0BD90121B0EE480AB948FFF74AFF0021B0EE680AB448FFF744FFB448008804280DD1B0480088042809D10222AE49AF48FFF7D1FD2020AD490880AA49088002
:40470000BDEC028B10BD10B52DED0C8B044602F0FAFD60B1F8F78DFCB0EE408AD4ED098AB1EE00AAF1EE00AAB0EE009A2BE00FF0E4F8B0EE408A9F4991F8280091ED0F0A00
:40474000F0EE400AB0EE480A0EF0EEFFDFED9A0A20EE200AB0EE408A964991F8280091ED0F1AF0EE410A94ED091AB0EE410A0EF0DBFFDFED910A60EE208AB0EE00AAF0EEDC
:4047800000AAB7EE009A4020005D40B994ED0B0A38EEC00A84ED0E0A0121402001551AEE100A2CF0D3FA41EC1B0B94ED0B0A30EE480A10EE101A08462CF0C8FA41EC1D0B66
:4047C000B0EE4D0AF0EE6D0A28F09AFEB0EE40CAF0EE60CA53EC1B2B51EC1C0B2CF0BEF80ED24C20005D58B9606822F0F8F900EE100AB8EE400A84ED110A01214C20015567
:404800001AEE900A2CF0A2FA41EC1B0B38EEC80A10EE101A08462CF099FA41EC1D0BB0EE4D0AF0EE6D0A28F06BFEB0EE40CAF0EE60CA53EC1B2B51EC1C0B2BF055FF0ED2A6
:404840005820005D58B9606822F0C9F900EE100AB8EE400A84ED140A01215820015519EE100A2CF073FA41EC1D0B38EEC80A10EE101A08462CF06AFA41EC1C0BB0EE4C0A0A
:40488000F0EE6C0A28F03CFEB0EE40BAF0EE60BA53EC1D2B51EC1B0B2CF060F80DD8002164200155607B454951F8200000EE100AB8EE400A84ED170A31E019EE100A2CF0DA
:4048C00045FA41EC1B0B38EEC80A10EE101A08462CF03CFA41EC1D0BB0EE4D0AF0EE6D0A28F00EFEB0EE40CAF0EE60CA53EC1B2B51EC1C0B2BF0F8FE11D26420005D70B90C
:40490000012164200155606822F069F900EE100AB8EE400A84ED170A22F039F9A06078EEC89A94ED0E0AB5EEC00AF1EE10FA0BD2B4EEE88AF1EE10FA06D294ED1B0AB4EEC0
:40494000E90AF1EE10FA12D394ED0E0AB5EEC00AF1EE10FA25DDB4EEE88AF1EE10FA20DD94ED1B0AB4EEE90AF1EE10FA19DDC4ED1B9A94ED1B0A10EE101A08462CF0E6F9F4
:4049800041EC1C0BB0EE4C0AF0EE6C0A28F0B8FDB0EE40BAF0EE60BA51EC1B0B2BF09AFBA066BDEC0C8B10BD541900202C170020D4170020081F0020E02E6542A81C040811
:4049C00000200022002100BF33E0FA4B03EB820393ED000AB5EEC00AF1EE10FA01D14B1C99B2F44B403303EB820393ED000AB5EEC00AF1EE10FA01D14B1C99B2EE4B03EBB6
:404A0000820393ED000AB5EEC00AF1EE10FA01D14B1C99B2E84B403303EB820393ED000AB5EEC00AF1EE10FA01D14B1C99B2531CDAB2082AC9DB00224FE0E04B93ED1D0A1C
:404A4000DFEDDF0AB4EEE00AF1EE10FA06DC93ED1D0AB5EEC00AF1EE10FA01D24B1C99B2D64B93ED230ADFEDD60AB4EEE00AF1EE10FA08DC93ED230ADFEDD20AB4EEE00AF4
:404A8000F1EE10FA01D24B1C99B2CC4B93ED260ADFEDCB0AB4EEE00AF1EE10FA06DC93ED260AB5EEC00AF1EE10FA01D24B1C99B2C24B93ED200ADFEDC20AB4EEE00AF1EE84
:404AC00010FA06DC93ED200AB5EEC00AF1EE10FA01D24B1C99B2531CDAB20F2AADDB01B901207047B54890F8A4007047B34981F8A4007047B148407B0C281FD0AF48407BBE
:404B00000B281BD0AD48407B072817D0AB48407B082813D0A948407B0A280FD0A748407B04280BD0A548407B052807D0A348407B0F2803D0A148407B102801D10120704780
:404B40000020FCE79D48407B082817D09B48407B042813D09948407B05280FD09748407B0A280BD09548407B0B2807D09348407B0F2803D09148407B102801D101207047C7
:404B80000020FCE78D48407B08280FD08B48407B0A280BD08948407B0B2807D08748407B102803D08548407B0F2801D1012070470020FCE78148407B082803D07F48407B18
:404BC0000A2801D1012070470020FCE770B5002426F0DEFF002872D101F04FFC18B10720FFF784FF80E007F095FE30B9FFF7E2FF18B90220FFF77AFF76E019F090F8B5EEF4
:404C0000C00AF1EE10FA06D2FFF7BCFF18B90920FFF76CFF68E019F082F8DFED6B0AB4EEE00AF1EE10FA02D2FFF78CFF60B16348407B0F280CD119F076F8DFED630AB4EE2A
:404C4000E00AF1EE10FA03D20420FFF74FFF4BE019F065F8DFED5D0AB4EEE00AF1EE10FA06DDFFF76FFF18B90520FFF73FFF3BE05748007D18B90120FFF738FF34E0F5F724
:404C8000DDFB50B102F065FA38B94C48407B0F2803D10D20FFF72AFF26E006F0D4FF28B106F0D1FF0546FFF721FF1DE0F8F7AEF930B1F8F7ABF90546FFF718FF14E01AE017
:404CC00006F0E6FE38B13D48407B0B2803D02420FFF70CFF08E0FFF76DF928B1FFF70AFF10B90A20FFF702FFFFF7FCFE18B10120FFF725FA0124204670BDC9B1DFED350A34
:404D0000C0ED000ADFED340AC0ED010A334AD2ED060AB8EE601ADFED321AC1EE210A9FED311AC1EE201AC0ED021A80ED040A1CE0DFED2D0AC0ED000ADFED2C0AC0ED010A28
:404D4000264AD2ED0D0AB8EE601ADFED251AC1EE210ADFED271A81EEA01AF6EE000A61EE200AC0ED020A80ED040A704710B501219FED200A11481030FFF7BFFF4FF4C07102
:404D80000C48303827F05DFA4FF4C0710A48303827F057FA0A20074930390871064930390871112003493039088003493039088010BD000004180020841900202C170020D2
:404DC00000409C4500409CC52FDDE43E2FDDE43F40280020CDCCCC3D14AE473FA81C040800007A447A142E3FCDCC4C3E0000204233331F4235FA0E3D2DED028B84B04FF4B5
:404E00007A66A821F94827F01CFA1421F84827F018FA00BF002231460320DFF8D8C300DF0546022D70D1DFF8D0C300DF0446022C6BD1EF480078002867D0ED480078112845
:404E400063DC0120ED490870E9480078E749487321F09DFEE5494860E54890ED010A084680ED090A407BE64908700020DF498860084600218166C1660167C16501664166E0
:404E80008163C163016441648164C1640165416581650020D54981F8A4000846407BD94951F82000D14908600846407B11287DD2DFE800F08F4B4E4F505109434849478A65
:404EC000412C3A4C4D00C948002141678167C1678030C160016141618161C1610162016041608160FFF742FF04208DF8040003208DF8050005208DF80600022201A9FF203B
:404F00001AF037FE042665E097E067E000219FEDBE0AB6481030FFF7F0FE9FEDBC0AB34880ED090A042655E09FEDB80AAF4880ED090A04264EE0C8264CE0FDF795FFC82695
:404F400048E000BF00BF042644E000BF00BF00BF00BF00BF00BF02F0D6F950B1F8F769F8B0EE408AA14880ED0B8A012180F8341018E00EF0C2FCB0EE408AA54991F82800C5
:404F800091ED0F0AF0EE400AB0EE480A0EF0CCFBDFEDA00A20EE200A944880ED0B0A012180F8341004208DF8040000E011E003208DF8050005208DF80600032201A9FF20CA
:404FC0001AF0D7FD042605E04FF4C87606F050FF00E000BF00BF042084490873012C2CD1002082494873002101209FED880AF5F7C1F90020814908709FED840A7C4880EDB1
:40500000010A9FED820A794880ED090A4FF47A665720F8F7B5F85820F8F7B2F8FFF78CF8042802D10020FFF78AF80C2019F0ACFB002201A9FF201AF09CFD6C48407B0028B3
:405040007DD06A4A1168506821F0A7FDF8B9FFF773F804280BD06548407B072817D06348407B0B2813D06148407B0C280FD0FFF7ADFD60B95D4890F8640001286DD15B496A
:40508000886840F6C41121F088FD002865D05748407B022807D05548407B012803D05348407B032819D1514890F8640030B94F4890ED000AB8EE400A80ED170A4B4890F8C3
:4050C000580030B9494890ED000AB8EE400A80ED140A5820F8F754F81FE04448407B06281BD1FFF76DFC80B99FED4B0A3F4880ED1D0A9FED490A80ED230A9FED470A80ED72
:40510000260A9FED450A80ED200A002043490880434908805720F8F733F80C2019F034FB002032494873FFF707F8042802D10020FFF705F8002101209FED340A00E00CE05B
:40514000F5F718F900202D4908709FED300A284880ED010A4FF47A665CE62448407B11287DD2DFE800F0090A329EF4F2F1F0EFEEEDECEBEAE90B0C00ABE100BF00BF02F07A
:40518000FBF888B10EF0A9FF00EE100AB8EE400A164880ED090AD0ED090AB0EE600A0121032008F0DEFE0CE09FED180A0F4880ED090AD0ED090AB0EE600A0121032008F0D0
:4051C0009FFD0A48FFF79FFA83E102F09CF858B39FED140A054880ED090AD0ED090AB0EE600A0121032008F05FFE56E02C17002018170020E1F3030829F303084C030020F7
:4052000068030020A81C04080000A04200000000081F0020E02E6542003C1C46D41700205419002000008CC2FFE71FF01EF9E8B1FE4890ED640ADFEDFE0A20EE200ADFED03
:40524000FD0A20EE200AB0EE408A014691F8280091ED0F0AF0EE400AB0EE480A00E01EE10DF000FDF44880ED090A0DE0EF4991F8280091ED0F0AF0EE400A9FEDF00A0DF033
:40528000F1FCED4880ED090AEB48D0ED090AB0EE600A0121032008F033FDE748FFF733FA17E102F030F868B19FEDE10AE24880ED090AD0ED090AB0EE600A0121032008F021
:4052C000F3FD35E01FF0D1F8D8B1D84890ED650ADFEDD70A20EE200ADFEDD60A20EE200AB0EE408A014691F8280091ED0F0AF0EE400AB0EE480A0DF0B5FCCF4880ED090A1F
:405300000DE0CA4991F8280091ED0F0AF0EE400A9FEDCB0A0DF0A6FCC74880ED090AC648D0ED090AB0EE600A0121032008F0E8FCC148FFF7E8F9CCE071E05FE09AE093E05E
:4053400086E090E085E080E01FE00FE0FFE7B74890F84210D03000EB8100D0ED000AB0EE600A01210846F5F705F8B2E0AF4890F84210D83000EB8100D0ED000AB0EE600AAB
:4053800001210846F4F7F6FFA3E0AB4841681030FEF740FFA84880ED090AA44991F8280091ED0F1AF0EE410AA34991ED091AB0EE410A0DF057FCF0EE408A0121032008F081
:4053C0009FFC9D4890F82900B8B100209A4981F829000EF00FFBF0EE408A032199480FF0CFFC984890ED001AF0EE410A924890ED091AB0EE410AFFF757F96AE08E484168DD
:405400001030FEF707FF8C4880ED090AD0ED090AB0EE600A01210846F4F7ACFF59E0864948688949D1ED000A884991ED000AFEF789FE814880ED090AD0ED090AB0EE600AB7
:4054400001210846F4F796FF43E0FDF77CFC40E000BF7948D0ED090AB0EE600A01210846F4F788FF35E034E006F008FC8046FEF766FE2EE0704A083202F11C0101F180008D
:40548000FBF70AF88046FEF75AFE6B48D0ED090AB0EE600A01210846F4F76CFF19E00020654948730873002101201FEDA80AF4F761FF0020664908701FEDAC0A654880ED29
:4054C000010A002201A9FF201AF053FB4FF47A6600BF00BFFEF730FE04287FF43DAE4FF4FA71384621F059FB00283FF435AE21F04EFB07460C2019F047F98BE470B52DED77
:40550000028B0446B0EE408A0025B5EEC08AF1EE10FA0AD04CB1112C07DC4E4890ED010AB4EE480AF1EE10FA0DD14B48D0F890110120DFF828C100DF1FEDCC0A454880EDC9
:40554000010A00250DE00CB142480470414880ED018A4148D0F890110220DFF800C100DF01252846BDEC028B70BD3948007870470120314981F8290070477A2303702E4B23
:40558000D3ED0E0A9FED360AB2EE041A00EE810ABDEEC00A10EE103A1AB24270130A8370254B93ED110ABCEEC00A10EE103A99B2C1700B0A0371204B93ED140ABCEEC00A7C
:4055C00010EE103A99B241710B0A83711A4B93ED170ABCEEC00A10EE103A99B2C1710B0A0372154BD3ED1A0A9FED1D0AB2EE041A00EE810ABDEEC00A10EE103A1AB2427229
:40560000130A837270477B2303700B4BD3ED1D0A9FED141A9FED120A00EE810ABDEEC00A10EE103A19B241700B0A1DE0081F002000008C420AD7233C2C170020C2B8B2BE8B
:40564000C2B8B23E60030020700300206C0300204C03002018170020F03F002081F30308000000470000C8428370604BD3ED230A1FED041A1FED060A00EE810ABDEEC00A7F
:4056800010EE103A19B2C1700B0A0371574BD3ED260A1FED0C1A1FED0E0A00EE810ABDEEC00A10EE103A19B241710B0A83714F4B93ED200ADFED4E0A20EE200ABCEEC00A65
:4056C00010EE103A9AB2C271130A0372704710B500244648407B112812D2DFE800F01213161718191A091D1E1C0D111B11141500FDF701FC044611E006F0B4FB04460DE01C
:4057000000BF00BF00BF00BF00BF00BF00BF00BF00BF00BF00BF00BF00BF00BF00BF204610BD10B500243148407B112812D2DFE800F01213161718191A091D1E1C0D111BDE
:4057400011141500FDF7DBFB044611E006F08AFB04460DE000BF00BF00BF00BF00BF00BF00BF00BF00BF00BF00BF00BF00BF00BF00BF204610BD1D48407B70471B4890F812
:405780006400704710B500241848407B112815D2DFE800F0161718191A1B1C091F201E15141D140D0E00F9F750F9044613E000BFFFF7E4FF642110FB01F40CE000BF00BF6C
:4057C00000BF00BF00BF00BF00BF00BF00BF00BF00BF00BF00BF00BF204610BD002003490873704703480078704700002C17002000007A446803002010B5F7F7BDF928200D
:40580000F7F7BEFC2920F7F7BBFC01F07CFD70B1DFF874C300DF0446042121F0F1FADFF868C300DF0446022121F0EAFA0DE0DFF858C300DF0446042121F0FFFADFF848C393
:4058400000DF0446022121F0F8FA10BD10B5CF48C16B012021F00EFBCC48C16B0120DFF830C300DF10BD10B52DED0C8BB0EE408AC84890ED630AB0EE409AB4EEC98AF1EECE
:4058800010FA02DDF7F768F938B9B4EEC98AF1EE10FA2CD2F7F760F948BBBE4890ED6A0A10EE101A08462BF051FA41EC1B0B38EE490A10EE101A08462BF048FA41EC1D0BD2
:4058C000B0EE4D0AF0EE6D0A27F01AFEB0EE40CAF0EE60CA53EC1B2B51EC1C0B2AF040FF41EC1A0B2AF0F6FB08EE900A3BE0B4EEC98AF1EE10FA02DDF7F72EF938B1B4EED8
:40590000C98AF1EE10FA2CD2F7F726F948B3A14890ED6B0A10EE101A08462BF017FA41EC1B0B38EE490A10EE101A08462BF00EFA41EC1D0BB0EE4D0AF0EE6D0A27F0E0FDB0
:40594000B0EE40CAF0EE60CA53EC1B2B51EC1C0B2AF006FF41EC1A0B2AF0BCFB08EE900A01E0DFED8D8A9FED8D0AF4EEC08AF1EE10FA03DD9FED890AF0EE408A9FED880AFB
:40598000F4EEC08AF1EE10FA03D29FED850AF0EE408AB0EE680ABDEC0C8B10BD10B52DED028B21F0F4F87F4908600020F6F7EAFCB0EE408AFFF757FF7A4880ED030AF6F7B4
:4059C000BAFEBDEC028B10BD2821764826F039FC01216E4880F82012DFF8ACC100DF06460122042121F0DDF9DFF89CC100DF06461922022121F0D5F9DFF88CC100DF06468F
:405A000031460120DFF888C100DF03215F4880F8201200BF00224FF6FF710720DFF888C100DF85B2012DF5D0022DF3D1DFF87CC100DF044604F0040008B1F6F70EFF04F0A5
:405A4000020018B1FFF7AAFFFFF700FF04F001000028DFD0FFF7D0FEDCE710B504464B48D0F81C122046DFF828C100DF10BD10B52DED088B474890ED630AD0ED610A30EED9
:405A8000600ADFED470A80EE801A11EE104A20462BF05CF941EC1B0BB0EE4B0AF0EE6B0A27F02EFDB0EE40AAF0EE60AA51EC1A0B2AF004FB41EC190B2AF00CFB08EE900A60
:405AC000344890ED620AD0ED630A30EE600ADFED330A80EE801A11EE104A20462BF036F941EC1A0BB0EE4A0AF0EE6A0A27F008FDB0EE409AF0EE609A51EC190B2AF0EAFA14
:405B000008EE100A0020F6F7FCFD224890F830000A280CD11F4890F8B201032807D19FED240AB0EE408AB1EE480AF0EE408AB0EE680AF6F73AFEB0EE480AF6F74AFEBDECBB
:405B4000088B10BD70B505460C46F6F795FD2846F6F756FA2046F6F76BFAFFF788FF0120FFF77BFF70BD0F48D0ED030AB0EE600A70470C4890F82400032801D00120704732
:405B80000020FCE702207047C1FF0308F03F002081F30308081F0020000000000000C8420000C8C2D41A0020E1F3030829F30308D051863970B50023012113E0CC1701EB75
:405BC000D4646511FE4C54F82540CD1701EBD5656D11A1EB45160125B5402C4004B10B46481CC1B24029E9DB184670BD70B504460D46E21704EBD2625311F14A52F8232067
:405C00002146E31704EBD3635B11A4EB43160123B3401A432046E31704EBD3635E11E84B43F826202846FDF7DFFA002C37D00821E448DFF894C300DF012813D0E148203811
:405C4000817F807F401CDF4A203A907710464454807F1E2802DB002011468877D948DFF86CC300DF0821DA48DFF85CC300DF012815D020F08CFFD74901EBC4014860D54854
:405C800010F83400FF2806DAD24810F83400401CD04901F83400CE48DFF830C300DF70BDCD490870704710B5CC480079052876D2DFE800F003152563B700FEF77BF910B971
:405CC0000220C6490871C648007838B10120C5490870FFF7E5FF0020C1490870E6E0FEF769F910B90220BD490871BD48007828B10120BC4908700020B9490870D6E0FEF7A8
:405D000059F918B10020B549087135E0B448007838B30120B3490870FEF74CF950B1FEF758F9044621460920FFF760FF0120FFF7B7FF21E005F0ACFE38B127210320FFF741
:405D400055FF0120FFF7ACFF16E0A748007800F0080038B918213120FFF748FF0120FFF79FFF09E003209D49087120F010FF9F4908600020FDF738FA98E099480078002832
:405D800044D005F085FE58B127210320FFF72EFF0120FFF785FF01209249087040E084E0FEF708F968B10120FFF77AFF01208D490870FEF70EF9044621460920FFF716FF3E
:405DC0002EE04FF47A718948006820F0E6FE90B18548007800F0020010BB0120FFF760FF18213120FFF702FF01207E49087000207A49087114E07C48007800F00B0078B1F0
:405E000004207649087106F065FC09E018210220FFF7ECFE01207349087002206F49087144E06F48007850B918210220FFF7DEFE01206C49087002206849087123E005F0C8
:405E400027FE68B127210320FFF7D0FE0220634908710120FFF724FF01206249087012E0FEF7A8F878B100205C4908710120FFF717FFFEF7AEF8044621460920FFF7B6FEB6
:405E80000120584908705548007904280CD006F020FC08F0BBFD38B1FFF767FB20B99FED540A0F20FFF72AFB00E000BF00BF4B4800794A49487110BD4148001F00210160CD
:405EC00041608160C16070474A490870704710B5494991F8300001F00CF930B1002213466421464812F03DFF11E0434991F8300001F021F928B9404991F8300001F023F962
:405F000028B10022134631213C4812F02AFF10BD10B50024384991F8300001F0EAF858B9354991F8300001F006F928B9324991F8300001F008F900B10124204610BD2D488C
:405F40000078704710B504462D480078844204D02B480470112018F017FC10BD1F490979042901D1012100E000210846704700EE900AB8EE601ADFED230AF5EE001A51EE6E
:405F8000210AB0EE600ADFED200A80EE201AB0EE410A70471D480078704710B52DED028BFFF7F8FF022807D0FFF7F4FF032803D0FFF7F0FF05283CD10BF088FF40B328E0FF
:405FC000741D0020601D002049F8030865F70308FC1A0020401B0020820300207803002083030020840300208C030020880300200000C84280030020081F002018CD00200F
:40600000760300200000FB4500007A447403002006E00BF055FF022802D19FEDFE8A0AE00BF054FF10B19FEDFC8A04E09FEDFB8A01E09FEDFA8AB0EE480ABDEC028B10BD08
:4060400010B52DED028B17F04EFEB0EE408AFFF7A4FFB4EEC08AF1EE10FA03DB0120BDEC028B10BD0020FAE710B52DED048BF0EE408AB0EE609A0446F0EE689AFFF7E0FFDB
:4060800000EE100AB8EE400AB4EEC90AF1EE10FA07DDFFF7D5FF00EE100AB8EE400AB0EE409A29EE090ADFEDDE0A80EE808AECB1F4EEC88AF1EE10FA05DDF0EE489A012099
:4060C000D849087015E0B1EE480AF4EEC08AF1EE10FA07D2B1EE480AF0EE409A0120D149087006E00020CF49087002E00020CD490870B0EE690ABDEC048B10BD10B504468C
:406100000020206060606071207120F040FD206010BD2DED048B92B04FF05008002405E04FF6FF702DF81400601CC4B2022CF7DB0020FFF7C9FE00208DF80400BA49087098
:40614000FFF7AEFD0020B9490870B948DFF8E4C200DFB948DFF8DCC200DFB848DFF8D4C200DF0020B24918390875B548FFF7C6FF0321B44880F8441100BF002241460720C9
:40618000DFF8C4C200DF0746022F7AD1DFF8BCC200DF054605F00200002873D01021A448DFF8ACC200DF012809D02822A049183908A825F0EAFF9E48DFF898C200DFBDF8D9
:4061C0002060FFF7CBFE08B1012000E00020814617F089FDF0EE408A3046FFF7C8FEB0EE409A4846F0EE680AFFF73EFFB0EE408AFFF7B4FE00B38E481838007D01280BD164
:40620000DDED0A0AB0EE600A0121042007F0EFFD8146FFF797FE2FE085481838007D02280BD1DDED090AB0EE600A0121052007F03BFE8146FFF786FE1EE07D481838007D21
:4062400003280BD1DDED0B0AB0EE600A0121062007F087FE8146FFF775FE0DE074481838007D042808D101210220B0EE480A07F047FD8146FFF766FE9DF83500012802D16B
:4062800002E047E032E00020734908709DF8350040B97248007840F00800704908700020FFF7FEFC4FF6FF7086421FD06B48007800F00200D0B96948007800F00800A8B176
:4062C000002410E03DF81410711A08B20EF0BDFF022806DC6148007840F002005F49087003E0601CC4B2022CECDB00BF05F0040080B15B4801889DF80420501CC0B28DF8B8
:4063000004002DF812109DF80400022802DB00208DF804001BF022FA68B10AF03BFF50B1FFF70DFE38B9FFF7F3FD08B1FFF7CFFD0120FFF7C9FD9DF8360090B10C9820F064
:406340004EFCB0F5C87F0CD30120374908703D48D0F8B4100120DFF80CC100DF0BF0D7FD02E00020304908703F48007D01281CD19DF81C0028B900203849087020F007FCA0
:40638000824640F2E241504620F007FC60B31EF06CF848BB0120254908702A48D0F8B4100120DFF8C0C000DF1EE09DF81C0001281AD12D48007DB8B900201C490870FFF71A
:4063C0007BFD2048D0F8B4100120DFF898C000DF2248007840F001002049087001202349087020F0D4FB824618221F4902A825F0CCFEFFF758FC1D48007801287FF4BDAE09
:40640000FFF7D8FB1A490870002018490870122030E000000AD7A33C9A99193E2FDDE43ED222FB3F85030020810300208D030020241B002055F70308601D0020FC1A002052
:4064400078030020F03F0020E1F3030829F3030849F8030865F70308830300208C030020341B002081F3030810280020840300207503002018F088F97FE6FE48007870473C
:40648000FD4800787047FD480078704770B50025FB48007D012801D1002405E0F848007D08B9012400E002242543F648C472FDF781FD08B9012400E0002445EA8400C5B2DB
:4064C000F0484472F048007D08B9012406E0EE48007D012801D1002400E0022445EA0410C5B2E8488472FFF7CEFF044645EA8415E4480472284670BDE448008870472DE9E2
:40650000F04105460C4617469846069EB5F52D4F28D12821DD481830DFF874C300DF012820D0A078D949C875A07800F0030048752078617840EA0120D449088020F027FB01
:40654000D24908610120887504200875D148D0F840110220DFF840C300DFCC481830DFF83CC300DFBDE8F081F0EE400A9FEDCC0A30EEC01ADFEDCB1A81EE210A70472DE90A
:40658000F0412DED028B04460D4616461F462078AD2833D12821BD481830DFF8F4C200DF01282AD0E078B949C875E07800F0030048756078A17840EA012000EE100AB8EE86
:4065C000C00AB0EE408AB0EE480AFFF7CDFFAF4880ED020A20F0DBFAAC490861012088750875AC48D0F840110220DFF8ACC200DFA6481830DFF8A4C200DF6BE02078AE280B
:4066000034D12821A1481830DFF884C200DF012860D0E0789D49C875E07800F0030048756078A17840EA012000EE100AB8EEC00AB0EE408AB0EE480AFFF796FF934880ED24
:40664000010A20F0A4FA9149086101208875022008759048D0F840110220DFF83CC200DF8A481830DFF834C200DF33E02078AF2830D1282185481830DFF814C200DF01283E
:4066800028D0E0788149C875E07800F0030048756078A17840EA012000EE100AB8EEC00AB0EE408A794880ED038A20F070FA7749086101208875032008757648D0F840116C
:4066C0000220DFF8D4C100DF70481830DFF8CCC100DF00BFBDEC028BBDE8F0819FED721ADFED720A40EE010AF1EE001AB6EE001A00EEA11AFCEEC10A10EE901A88B2704798
:4067000010B52DED028B0DF0F8F8B0EE408A9FED680AB4EE408AF1EE10FA06D0B0EE480AFFF7DCFF5749088003E04FF6FF70554908805848D0F840110420DFF85CC100DF19
:4067400050480088BDEC028B10BD70B58CB006460025002E50D01DF088FE00284DD040F2B240012102220023CDE90532CDE90710042017210193CDE902310490972013463A
:406780000022114600900AA812F0ECF80AA9304611F0DEFD044640F292400440844204D11DB9042043490870012540F2B240012102220023CDE90532CDE90710042017213F
:4067C0000193CDE902310490972001230022114600900AA812F0C6F80AA9304611F0B8FD044640F292400440844205D1002DFCD10520304908700125DAE040F2B2400121EF
:4068000002220023CDE90532CDE9071017210193CDE902319720049300900123002211460AA812F09FF80AA9304611F091FD044640F292400440844204D11DB903201D4998
:406840000870012540F2B240012102220023CDE90532CDE9071017210193CDE902319720049300901346002211460AA812F07AF80AA921E081030020760300208203002012
:4068800040280020341B0020E82700200C1B002049F80308F03F002081F3030865F7030800401C460000C84200007A440000FB4500FF7F4774030020304611F049FD0446DD
:4068C00040F292400440844204D11DB9022068490870012540F2B240012102220023CDE90532CDE9071017210193CDE902319720049300900323002211460AA812F032F817
:406900000AA9304611F024FD044640F292400440844204D11DB9032055490870012540F2B240012102220023CDE90532CDE9071017210193CDE902319720049300900423A9
:40694000002211460AA812F00DF80AA9304611F0FFFC044640F292400440844204D11DB9022043490870012540F2B240012102220023CDE90532CDE9071017210193CDE9A8
:40698000023197201A461946049300900AA811F0E9FF0AA9304611F0DBFC044640F292400440844204D11DB9012031490870012515B15520F6F7E4FB28460CB070BD10B50C
:4069C0002C4890F8280007280DD117F08CF9DFED2A0AB4EEE00AF1EE10FA01DB012000E00020044600E00124204610BD10B517F07AF9DFED220AB4EEE00AF1EE10FA01D861
:406A0000012010BD0020FCE79FED1D0A70479FED1D0A70471648007803280FD01448007802280BD012480078012807D010480078042803D00E480078052801D10120704792
:406A40000020FCE710480079704710B500F033FC10B10E48047800E00024204610BDF0EE400A1FED701A1FED720A00EE810A704774030020081F00202FDDE43E83C00041D7
:406A8000B81E4141A2454841780300208503002010B5044600BF28222146FD48006802F0E3FD20B928222146FA4825F029FB00BF10BD10B504462822F649204625F020FB0E
:406AC00010BD01B500BF04226946F1480068283002F0CAFD18B99DF80000EE49886200BFED48C16B0220DFF8B4C300DF08BD01B500BF04226946E64800682C3002F0B4FD33
:406B000018B99DF80000E349C86200BF08BD01B500BF04226946DE480068303002F0A4FD10B9DC490098086300BF08BD10B52DED020B00BF04226946D54800683C3002F072
:406B400093FD20B99DED000AD24880ED0F0A00BF03F090FED048C16B0220DFF840C300DF0220F6F70DFB4F20F6F70AFB1CBD01B500BF01226946C6480068483002F074FD30
:406B800020B99DF80000C34981F8480000BF08BD08B5002000901DF055FCA0B10021C04800781DF079FCBF4800781EF077F828B10220FFF7DCFF0120009004E00120FFF763
:406BC000D6FF0220009000BF01226946B0480068493002F049FD20B99DF80000AD4981F8490000BFAC48016D0120DFF8B0C200DF08BD01B500BF04226946A5480068443004
:406C000002F032FD10B9A3490098486400BF08BD01B5A04890F841009DF80010884215D000BF012269469A480068413002F01CFD20B99DF80000974981F8410000BF18F0D5
:406C4000CCFF07F0F3FE1E20F6F79AFA08BD01B500BF012269468E480068423002F004FD20B99DF800008B4981F8420000BF18F0B4FF2520F6F784FA8748C16B0220DFF8D8
:406C80001CC200DF07F0D2FE08BD01B500BF0422694685480068AC3002F0E6FC18B97D480099C0F89C1400BF08BD8048006870477E490860704770B52DED028B04460D460B
:406CC00016461DF0A7FBF8B17249E0314A5D891C495D501800EBD071491000EE101AB8EEC00AB0EE408ABCEEC80A10EE101AC8B2294607F0D2FABCEEC80A10EE101AC8B2D7
:406D0000294607F0FDFA0EE01DF09CFB58B16149E031485D294607F0C0FA5E49E231485D294607F0EDFA624800EB8400D0ED000AB0EE600A2946204607F0A3F95C49083101
:406D4000085D2A46214607F0EEF959490A31085D2A46214607F025FA55490C31085D2A46214607F05CFA46B1182017F00DFD4A48016D0120DFF824C100DFBDEC028B70BD07
:406D800070B500240CE0002506E0002229462046FFF791FF681CC5B2022DF6DB601CC4B2022CF0DB182017F0EFFC3B48016D0120DFF8E8C000DF70BD70B52DED028B044653
:406DC0000D461DF027FB00B33248D03000EB840090ED000AB1EE400A2E48D83000EB8400D0ED000A30EE200AF0EE000A80EE201AB0EE418A2046B1EE480A07F082FB2046DF
:406E0000B0EE480A07F0D8FB18E01DF01BFBA8B12048D03000EB8400D0ED000AB0EE600A204607F06EFB1B48D83000EB8400D0ED000AB0EE600A204607F0BEFB1548C030AC
:406E400000EB8400D0ED000AB0EE600A204607F08AFA1048C83000EB8400D0ED000AB0EE600A204607F0F4FA75B1142017F08CFC182017F089FC142017F086FC0648016DF4
:406E80000120DFF818C000DFBDEC028B70BD0000A4030020081F0020F03F002081F30308F706002018070020A803002090030020EC20002010B5002405E000212046FFF793
:406EC0007BFF601CC4B2022CF7DB142017F05CFC182017F059FC142017F056FCFB48016D0120DFF8ECC300DF10BD70B505460C4600212046FFF760FF002221462846FFF7E3
:406F0000DAFE70BD70B52DED028B05460024B5E0F04890F84900C0EB001105F1380000EB81000E3030F9140000EE900AF8EEE00AB0EE600A204607F004FCE64890F84900E6
:406F4000C0EB001105F1380000EB8100123030F9140000EE900AF8EEE00AB0EE600A204607F013FCDB4890F84900C0EB001105F1380000EB8100163030F9140000EE900A1B
:406F8000F8EEE00AB0EE600A204607F022FCD14890F84900C0EB001105F1380000EB81001A3030F9140000EE900AF8EEE00AB0EE600A204607F040FCC64991F84910C1EB21
:406FC000011205F1380101EB82010931085D214607F056FCBF4991F84910C1EB011205F1380101EB82010B31085D214607F067FCB84890F84900C0EB001105F1380000EB42
:407000008100401C005D00EE100AB8EE400ADFEDB20A80EE201AB0EE418A2046B0EE480A07F06CFCAB4991F84910C1EB011205F1380101EB8201C91C085D214607F077FC82
:40704000A44991F84910C1EB011205F1380101EB8201491D085D214607F07DFC9D4991F84910C1EB011205F1380101EB8201C91D085D214607F083FC601CC4B2022CFFF6E0
:4070800047AF944890F84900C0EB001105F1380000EB8100D0ED080AB0EE600A07F015FBBDEC028B70BD8B4890F8280008B9012070470020FCE710B5012019F003FE014640
:4070C000864880F83910002019F0FCFD83494874012019F0F7FD04462146012011F029F9002019F0EFFD04462146002011F021F910BD01460020282901D1012200E00022C7
:40710000402901D1012300E000231A43492901D1012300E000231A434A2901D1012300E000231A434B2901D1012300E000231A4302B10120704701460020562901D0612969
:4071400000D10120704701460020592900D10120704710B500245F4890F830000A2803D11DF070F900B10124204610BD594890F82810082905D0092903D00A2901D00E2960
:4071800001D1012070470020FCE7524890F828100A2901D1012070470020FCE74D4890F82810082901D1012070470020FCE7494890F82810092901D1012070470020FCE785
:4071C000444890F828100E2901D1012070470020FCE710B504461DF035F970B11DF045F900B92CB901213E4800781DF055F904E000213B4800781DF04FF910BD354890F869
:407200003000C0EB001101EB4010364901EBC000408E70470246012109E001EB0110324B13F81000904201D1C8B27047491C1A29F3DB0020F9E7274890ED0F0A704725481A
:4072400090F84900022801D1012070470020FCE7204890F84900012800D170470020FCE71C4890F8490008B9012070470020FCE710B50024FFF7F4FF08B1012419E01DF0F2
:40728000E1F8B0B1FFF7E4FF20B1184800781DF005FD68B9FFF7D3FF58B1F3F7DBF838B9F3F7D8F828B9114800781DF0F7FC00B90124204610BD074890F8970020B105485A
:4072C00090F89700012813D101207047F03F002081F30308081F00200000C842D8CD0020F206002060200408EC1C0408180700200020EAE74C4890F82800072801D1012058
:4073000070470020FCE7484890F89700022804D0454890F89700032801D1012070470020FCE7414890F89700032801D1012070470020FCE73C4890F89700022801D1012022
:4073400070470020FCE7384890F8970008B9012070470020FCE7344890F89700012800D170470020FCE7304890F89700042801D1012070470020FCE72B4890F8970004289B
:4073800001D1012070470020FCE701B500BF0122694626480068973002F066F920B99DF80000214981F8970000BF08BD01B500BF012269461D48006800F2853002F054F985
:4073C00020B99DF80000184981F8850300BF08BD10B50024144890F8300028281DD0124890F83000402818D00F4890F83000492813D00D4890F830004A280ED00A4890F803
:4074000030004B2809D0084890F83000592804D0054890F830005C2800D101242046FFF7C5FF204610BD0000081F0020A40300201FB51DF02EF8062808D01DF02AF8072828
:4074400004D01DF026F8082841F077821DF00DF800287DD0002000900190029003460122FE4903901DF0EFF8002000900190029003460322FA49039001201DF0E4F80020DE
:4074800000900190029003460322F649039002201DF0D9F8002000900190029003460322F149039010461DF0CEF8002000900190029003460322ED49039004201DF0C3F8AC
:4074C000002000900190029003460422E849039005201DF0B8F8002002220123CDE901200093039003460322E24906201DF0ABF8002000900190029003460246DE490390B2
:4075000007201DF0A0F8002000900190029003460322DA49039008201DF095F8002000900190029003460122D549039009201DF08AF8002000900190029003460122D149C5
:4075400003900A201DF07FF800200090019000E0E0E3029003460122CB4903900B201DF072F8002001210090CDE9010103460A46C64903900C201DF066F800200090019002
:40758000029003460246C249039011201DF05BF8002000900190029003460322BD49039012201DF050F800200222CDE9000202900346B949039016201DF045F800200121EA
:4075C0000090CDE9010103460A46B449039017201DF039F8002000900190029003460222AF49039019201DF02EF800200222CDE9000202900346AB4903901A201DF023F8AE
:40760000002000900190029001230222A64903901B201DF018F8002000900190029001230222A24903901C201DF00DF800200222CDE90002029003469D4903901E201DF0D3
:4076400002F800200222CDE90002029003460246984903901F201CF0F6FF0020009001900290034603229449039021201CF0EBFF0020009001900290034603228F490390A9
:4076800022201CF0E0FF0020009001900290034603228B49039023201CF0D5FF0020009001900290034603228649039024201CF0CAFF00200090019002900346032282490A
:4076C000039025201CF0BFFF0020009001900290034603227D49039026201CF0B4FF0020009001900290034601227949039027201CF0A9FF0020009001900290034601227B
:407700007449039028201CF09EFF0020009001900290034601227049039029201CF093FF0020009001900290034602226B4903902B201CF088FF0020009001900290034615
:407740000222674903902C201CF07DFF002000900190029003460122624903902D201CF072FF0020009001900290034601225E4903902E201CF067FF00200090019002907B
:4077800003460122594903902F201CF05CFF0020009001900290034601225549039031201CF051FF0020009001900290034601225049039032201CF046FF00200121CDE94F
:4077C000000103460A46CDE902104B4936201CF03AFF002000900190029003460122474903903B201CF02FFF002000900190029003460122424903903C201CF024FF0020F9
:407800000122CDE90002029003463E4903903D201CF019FF00200122CDE9000202900346394903903E201CF00EFF002001210090CDE9010103460A463449039041201CF0F5
:4078400002FF0020009001900290034601223049039042201CF0F7FE00205BE0BB060020D8060020D70600201C0700201D070020DB060020DC06002028070020D90600204A
:40788000EF060020EE060020ED06002010070020A4060020E106002097060020AE060020980600209D0600201E0700201F0700209C060020A10600209106002093060020EE
:4078C000E4060020E5060020E6060020E7060020E9060020E8060020EA060020EB060020EC060020DD060020DF060020DE060020F0060020F1060020F2060020F40600209F
:40790000F5060020F6060020F7060020F8060020C206002000900190029003460122FE49039043201CF08FFE002000900190029003460122F949039044201CF084FE0020D2
:4079400001210090CDE9010103460A46F449039048201CF078FE002001210090CDE9010103460A46EF4903904B201CF06CFE002001210090CDE9010103460A46EA49039092
:407980004D201CF060FE002000900190029003460322E64903904F201CF055FE012000220092CDE9012013460246E149039050201CF049FE002001210090CDE9010103467F
:4079C0000A46DC49039051201CF03DFE002000900190029003460122D749039052201CF032FE002000900190029003460322D349039054201CF027FE0020009001900290BF
:407A000003460322CE49039055201CF01CFE002000900190029003460322CA49039056201CF011FE002000900190029003460322C549039057201CF006FE00200222CDE9B8
:407A40000002029003460246C049039057201CF0FAFD002000900190029003460322BC49039058201CF0EFFD002000900190029003460322B749039059201CF0E4FD002028
:407A800000900190029003460322B34903905A201CF0D9FD002000900190029003460322AE4903905B201CF0CEFD002001210090CDE9010103460A46A94903905C201CF06D
:407AC000C2FD002000900190029003460122A54903905D201CF0B7FD002000900190029003460122A04903905E201CF0ACFD0020009001900290034601229C4903905F20A6
:407B00001CF0A1FD00200222CDE900020290034601229749039061201CF095FD00200222CDE900020290034601229249039062201CF089FD00200090019002900346012254
:407B40008D49039064201CF07EFD0020009001900290034601228949039065201CF073FD002001210090CDE9010103460A468449039067201CF067FD002001210090CDE9EA
:407B8000010103460A467F49039069201CF05BFD00200222CDE900020290034602467A4903906A201CF04FFD01200021009101910B460246CDE9021074496B201CF043FD31
:407BC00000200222CDE9000202900346704903906D201CF038FD00200222CDE90002029003466C4903906E201CF02DFD00200222CDE9000202900346674903906F201CF0FC
:407C000022FD002001210090CDE9010103460A466249039073201CF016FD00200222CDE900020290034602465D49039079201CF00AFD00200090019002900346022259492C
:407C400003907A201CF0FFFC002000900190029003460122544903907B201CF0F4FC002000900190029003460122504903907C201CF0E9FC00200090019002900346012293
:407C80004B4903907D201CF0DEFC002001210090CDE9010103460A46464903907E201CF0D2FC002000900190029003460122424903907F201CF0C7FC002001210090CDE90A
:407CC0000101034602223D49039082201CF0BBFC002001210090CDE90101034602223849039083201CF0AFFC002001210090CDE90101034602223349039084201CF0A3FCDD
:407D000001200021009101910B460222CDE902102D495BE0DAE00000F9060020FA06002020070020210700200F070020DA060020FB060020FC060020FD0600202507002080
:407D4000260700202707002029070020A90600200207002003070020040700209F06002005070020070700200807002006070020E3060020E2060020090700200A070020DE
:407D80000C0700200E070020CF060020BC060020220700202307002024070020110700201307002014070020B5060020B6060020150700201607002012070020BF060020AB
:407DC000C0060020C10600201807002086201CF03AFC01200021009101910B460222CDE90210FE4987201CF02EFC01200021009101910B460246CDE90210F94988201CF00D
:407E000022FC002000900190029003460322F54903908E201CF017FC002000900190029003460322F04903908F201CF00CFC002000900190029003460322EC4903908F20BD
:407E40001CF001FC012008F0C6FE0021E84800781CF022FB0021E74800781CF01DFB0021E54800781CF018FB0021E44800781CF013FB01200021009101910B460222CDE9EA
:407E80000210DF4986201CF0DEFB01200021009101910B460222CDE90210DA4987201CF0D2FB0121D84800781CF07BFF0121D74800781CF076FF0121D54800781CF071FF0B
:407EC0000121D44800781CF06CFFE1E3002000900190029003460122CF4903901CF0B3FB002000900190029003460322C649039001201CF0A8FB002000900190029003461E
:407F00000322C249039002201CF09DFB002000900190029003460322C049039010461CF092FB002000900190029003460322BC49039004201CF087FB00200090019002908E
:407F400003460422B749039005201CF07CFB002002220123CDE901200093039003460322B14906201CF06FFB002000900190029003460322A749039007201CF064FB002078
:407F800000900190029003460322A149039008201CF059FB002000900190029003460122A249039009201CF04EFB0020009001900290034601229E4903900A201CF043FB33
:407FC000002000900190029003460122994903900B201CF038FB002001210090CDE9010103460A46944903900C201CF02CFB00200090019002900346032290490390112093
:408000001CF021FB0020009001900290034603228B49039012201CF016FB00200222CDE90002029003468749039016201CF00BFB002001210090CDE9010103460A466E49C5
:40804000039017201CF0FFFA0020009001900290034602227C49039019201CF0F4FA00200222CDE9000202900346784903901A201CF0E9FA002000900190029001230222F7
:40808000734903901B201CF0DEFA0020009001900290012302226F4903901C201CF0D3FA00200222CDE90002029003466A4903901E201CF0C8FA00200222CDE90002029020
:4080C00003460246654903901F201CF0BCFA00200222CDE900020290034602466049039020201CF0B0FA0020009001900290034603225C49039021201CF0A5FA0020009047
:4081000001900290034603225749039022201CF09AFA0020009001900290034603225349039023201CF08FFA0020009001900290034603224E49039024201CF084FA0020F8
:40814000009001900290034603224A49039025201CF079FA0020009001900290034603224549039026201CF06EFA0020009001900290034601224149039027201CF063FACC
:408180000020009001900290034601223C49039028201CF058FA0020009001900290034601223849039029201CF04DFA002000900190029003460222334903902B201CF02D
:4081C00042FA0020009001900290034602222F4903902C201CF037FA002059E0190700201A070020C8060020C9060020C706002005070020FC060020AE060020F106002092
:40820000AB060020AA060020D8060020D7060020D9060020D6060020BB0600201C0700201D070020DB060020DC060020EF060020EE060020ED06002010070020A5060020FE
:40824000E106002097060020980600209D0600201E0700201F0700209C060020A1060020A80600209106002093060020E4060020E5060020E6060020E7060020E90600202A
:40828000E8060020EA060020EB060020EC06002000900190029003460122FE4903902D201CF0D1F9002000900190029003460122F94903902E201CF0C6F9002000900190F3
:4082C000029003460122F54903902F201CF0BBF9002000900190029003460122F049039031201CF0B0F9002000900190029003460122EC49039032201CF0A5F9002001214A
:40830000CDE9000103460A46CDE90210E64936201CF099F9002000900190029003460122E24903903B201CF08EF9002000900190029003460122DE4903903C201CF083F93A
:4083400000200122CDE9000202900346D94903903D201CF078F900200122CDE9000202900346D54903903E201CF06DF9002001210090CDE9010103460A46D0490390412011
:408380001CF061F9002000900190029003460122CB49039042201CF056F9002000900190029003460122C749039043201CF04BF9002000900190029003460122C249039042
:4083C00044201CF040F9002001210090CDE9010103460A46BD49039048201CF034F9002001210090CDE9010103460A46B84903904B201CF028F9002001210090CDE901019E
:4084000003460A46B34903904D201CF01CF9002000900190029003460322AF4903904F201CF011F9012000220092CDE9012013460246AA49039050201CF005F900200121A6
:408440000090CDE9010103460A46A549039051201CF0F9F8002000900190029003460122A049039052201CF0EEF80020009001900290034603229C49039054201CF0E3F8F9
:408480000020009001900290034603229749039055201CF0D8F80020009001900290034603229349039056201CF0CDF80020009001900290034603228E49039057201CF092
:4084C000C2F80020009001900290034603228A49039058201CF0B7F80020009001900290034603228549039059201CF0ACF8002000900190029003460322814903905A2005
:408500001CF0A1F80020009001900290034603227C4903905B201CF096F8002001210090CDE9010103460A46774903905C201CF08AF800200090019002900346012273496D
:4085400003905D201CF07FF80020009001900290034601226E4903905E201CF074F80020009001900290034601226A4903905F201CF069F800200222CDE9000202900346A1
:4085800001226549039061201CF05DF800200222CDE900020290034601226049039062201CF051F80020009001900290034601225B49039064201CF046F8002000900190E3
:4085C0000290034601225749039065201CF03BF8002001210090CDE9010103460A465249039067201CF02FF8002001210090CDE9010103460A464D49039069201CF023F87F
:4086000000200222CDE90002029003460246484903906A201CF017F801200021009101910B460246CDE9021042496B201CF00BF800200222CDE90002029003463E49039076
:408640006D201CF000F800200222CDE90002029003463A4903906E201BF0F5FF00200222CDE9000202900346354903906F201BF0EAFF002001210090CDE9010103460A4661
:408680003049039073201BF0DEFF002002225BE053E10000DD060020DF060020DE060020F0060020F1060020F2060020F4060020F5060020F6060020F7060020F8060020A3
:4086C000C2060020F9060020FA06002020070020210700200F070020DA060020FB060020FC060020FD0600202507002026070020270700202907002002070020030700209E
:40870000040700209F06002005070020070700200807002006070020E3060020E2060020090700200A0700200C0700200E070020CF060020BC06002022070020230700204F
:408740002407002011070020CDE90002029003460246FE49039079201BF075FF002000900190029003460222F94903907A201BF06AFF002000900190029003460122F54909
:4087800003907B201BF05FFF002000900190029003460122F04903907C201BF054FF002000900190029003460122EC4903907D201BF049FF002001210090CDE90101034653
:4087C0000A46E74903907E201BF03DFF002000900190029003460122E24903907F201BF032FF002001210090CDE9010103460222DD49039082201BF026FF00200121009055
:40880000CDE9010103460222D849039083201BF01AFF002001210090CDE9010103460222D349039084201BF00EFF01200021009101910B460222CDE90210CE4986201BF0CC
:4088400002FF01200021009101910B460222CDE90210C94987201BF0F6FE01200021009101910B460246CDE90210C44988201BF0EAFE002000900190029003460322C049E5
:4088800003908E201BF0DFFE002000900190029003460322BB4903908F201BF0D4FE002000900190029003460322B74903908F201BF0C9FE012008F08EF90021B3480078A2
:4088C0001BF0EAFD0021B24800781BF0E5FD0021B04800781BF0E0FD0021AF4800781BF0DBFD01200021009101910B460222CDE90210AA4986201BF0A6FE0120002100915D
:4089000001910B460222CDE90210A54987201BF09AFE0121A34800781CF043FA0121A24800781CF03EFA0121A04800781CF039FA01219F4800781CF034FA1FBD1FB500204E
:40894000009001900290034603229A49039001201BF079FE0020009001900290034603229549039002201BF06EFE0020009001900290034603229149039010461BF063FE02
:408980000020009001900290034603228C49039004201BF058FE0020009001900290034604228849039005201BF04DFE0020009001900290034603228349039006201BF097
:4089C00042FE0020009001900290034603227F49039007201BF037FE0020009001900290034603227A49039008201BF02CFE002000900190029003460222554903900920A6
:408A00001BF021FE0020009001900290034602227049039017201BF016FE0020009001900290034602466C49039019201BF00BFE00200090019002900346032267490390AD
:408A400021201BF000FE0020009001900290034603226349039022201BF0F5FD0020009001900290034602224D49039027201BF0EAFD00200090019002900346022247497B
:408A8000039028201BF0DFFD0020009001900290034602465349039029201BF0D4FD01200021009101910B460A46CDE902104E492A201BF0C8FD00200090019002900346A1
:408AC00002464A4903902B201BF0BDFD002000900190029003460122454903902D201BF0B2FD002000900190029003460246414903902E201BF0A7FD002000900190029040
:408B0000034602463C4903902F201BF09CFD0020009001900290034602463849039030201BF091FD0020009001900290034602463349039046201BF086FD00200090019090
:408B40000290034602462F4903905DE01307002014070020B5060020B6060020150700201607002012070020BF060020C0060020C106002018070020190700201A0700203A
:408B8000C8060020C9060020C706002005070020FC060020AE060020F1060020AB060020AA060020D8060020D7060020D9060020D6060020E40600209106002092060020A2
:408BC0009306002094060020E70600209506002096060020C30600209B0600209E0600209F060020AC060020A5060020A2060020CC060020CD060020CE060020CF06002018
:408C0000A0060020D106002047201BF01CFD002000900190029003460246F649039048201BF011FD002000900190029003460122F149039057201BF006FD00200090019063
:408C4000029003460222ED49039059201BF0FBFC002000900190029003460222E84903905A201BF0F0FC002000900190029003460122E44903905B201BF0E5FC0020009026
:408C80000190029003460122DF4903905C201BF0DAFC002000900190029003460122DB4903905D201BF0CFFC002000900190029003460122D64903905E201BF0C4FC00206A
:408CC00000900190029003460122D24903905F201BF0B9FC002000900190029003460122CD49039060201BF0AEFC002000900190029003460122C949039061201BF0A3FC3C
:408D0000002000900190029003460122C449039064201BF098FC002000900190029003460122C049039065201BF08DFC002000900190029003460122BB49039066201BF0D6
:408D400082FC002000900190029003460122B749039067201BF077FC002000900190029003460122B249039068201BF06CFC002000900190029003460122AE490390692084
:408D80001BF061FC002000900190029001231A46A94903906A201BF056FC002000900190029003460122A54903906C201BF04BFC002000900190029003460122A04903902F
:408DC0006D201BF040FC0020009001900290034601229C4903906E201BF035FC01200021009101910B460A46CDE9021096497C201BF029FC01200021009101910B460A469F
:408E0000CDE9021091497D201BF01DFC002001210090CDE9010103460A468D49039081201BF011FC0020009001900290034602228849039082201BF006FC002000900190F6
:408E40000290034602228449039083201BF0FBFB0020009001900290034602227F49039084201BF0F0FB0020009001900290034602227B49039086201BF0E5FB00200090E2
:408E800001900290034602227649039087201BF0DAFB0020009001900290034602467249039088201BF0CFFB0020009001900290034603226D4903908D201BF0C4FB0020F9
:408EC00000900190029003460322694903908E201BF0B9FB002000900190029003460322644903908F201BF0AEFB0121584800781BF0D2FA0121604800781BF0CDFA012174
:408F00005E4800781BF0C8FA1FBD1FB500240CE000205B4901EB041189680870584901EB0411C9680870601CC4B2902CF0DB1BF005FA1CF0A3F81FF0E5FB0121022021F09F
:408F4000A4FE0020009001900290034601224D49039016201BF077FB002001210090CDE9010103460A46484903901E201BF06BFB00200090019002900346012243490390E0
:408F80006B201BF060FB1BF084FAFF2831D00121084621F07AFE0121042021F076FE0121082021F072FE0121102021F06EFE0121202021F06AFE0121402021F066FE0121BD
:408FC000802021F062FE0121080221F05EFE1BF060FA0A2862D2DFE800F06105060708095B5C5D5E00BF00BF00BF00BFFFF7A6FC55E055E0A1060020D5060020AD060020BC
:40900000AE060020AF060020B0060020B1060020D2060020D3060020D4060020B2060020F5060020F6060020B5060020B6060020B7060020B8060020B9060020BC060020AD
:40904000BD060020BE060020A8060020A7060020C2060020BF060020C0060020C1060020D8060020D7060020C4060020C7060020C8060020C9060020C5060020C60600206E
:40908000403C0408970600209C060020BB06002000BF00BF00BFFEF7CBF900E000BF00BF1FBD10B50120FE4908701DF070FDFC494860012021F09AFC1CE0612021F038FC02
:4090C00078B145F25550F74908600120486040F6B83088604CF6CC4008600220F049087008E0EF4948681DF07AFD642802D90320EB490870EA4800780128DED010BD10B5CE
:409100000020E74908704FF4FA701DF019FDFA201DF057FDFFF7C5FFFFF7F7FE1BF07AF9C8B1E14800781BF0B9FD40B90121DF4800781BF0B1F90020DD4908700BE0DD48E1
:4091400000781BF0ABFD18B10220D949087002E00120D74908701AF0CFFBEFF7B3F800221146D548DFF854C300DF002010BD10B572B66FF0040000F054FA6FF0010000F011
:4091800050FA4FF0FF3000F04CFA042000F049FA052000F046FA062000F043FA072000F040FA082000F03DFA092000F03AFA0A2000F037FA0B2000F034FA0C2000F031FAFA
:4091C0000D2000F02EFA0E2000F02BFA0F2000F028FA102000F025FA112000F022FA122000F01FFA132000F01CFA142000F019FA152000F016FA162000F013FA172000F0F0
:4092000010FA182000F00DFA192000F00AFA1A2000F007FA1B2000F004FA1C2000F001FA1D2000F0FEF91E2000F0FBF91F2000F0F8F9202000F0F5F9212000F0F2F922206B
:4092400000F0EFF9232000F0ECF9242000F0E9F9252000F0E6F9262000F0E3F9272000F0E0F9282000F0DDF9292000F0DAF92A2000F0D7F92B2000F0D4F92C2000F0D1F980
:409280002D2000F0CEF92E2000F0CBF92F2000F0C8F9302000F0C5F9312000F0C2F9322000F0BFF9332000F0BCF9342000F0B9F9352000F0B6F9362000F0B3F9372000F099
:4092C000B0F9382000F0ADF9392000F0AAF93A2000F0A7F93B2000F0A4F93C2000F0A1F93D2000F09EF93E2000F09BF93F2000F098F9402000F095F9412000F092F9422071
:4093000000F08FF9432000F08CF9442000F089F9452000F086F9462000F083F9472000F080F9482000F07DF9492000F07AF94A2000F077F94B2000F074F94C2000F071F99F
:409340004D2000F06EF94E2000F06BF94F2000F068F9502000F065F9512000F062F96FF0040000F067F96FF0010000F063F94FF0FF3000F05FF9042000F05CF9052000F09A
:4093800059F9062000F056F9072000F053F9082000F050F9092000F04DF90A2000F04AF90B2000F047F90C2000F044F90D2000F041F90E2000F03EF90F2000F03BF9102093
:4093C00000F038F9112000F035F9122000F032F9132000F02FF9142000F02CF9152000F029F9162000F026F9172000F023F9182000F020F9192000F01DF91A2000F01AF990
:409400001B2000F017F91C2000F014F91D2000F011F91E2000F00EF91F2000F00BF9202000F008F9212000F005F9222000F002F9232000F0FFF8242000F0FCF8252000F005
:40944000F9F8262000F0F6F8272000F0F3F8282000F0F0F8292000F0EDF82A2000F0EAF82B2000F0E7F82C2000F0E4F82D2000F0E1F82E2000F0DEF82F2000F0DBF830209D
:4094800000F0D8F8312000F0D5F8322000F0D2F8332000F0CFF8342000F0CCF835200FE09803002000300040A2060020BE06002094030020CF0600206320020895FB0308D1
:4094C00000F0B8F8362000F0B5F8372000F0B2F8382000F0AFF8392000F0ACF83A2000F0A9F83B2000F0A6F83C2000F0A3F83D2000F0A0F83E2000F09DF83F2000F09AF8A8
:40950000402000F097F8412000F094F8422000F091F8432000F08EF8442000F08BF8452000F088F8462000F085F8472000F082F8482000F07FF8492000F07CF84A2000F075
:4095400079F84B2000F076F84C2000F073F84D2000F070F84E2000F06DF84F2000F06AF8502000F067F8512000F064F862B610BD38B5044660680090009D206880F3088889
:4095800000BFA84738BD00BFBFF34F8F2E48006800F4E0602D490843001D2B490860BFF34F8F00BF00BFFEE710B50021284800781AF072FF0021274800781AF06DFF01DF53
:4095C00010BD01B500BF04226946234800688C3000F04AF818B921480099C0F87C1400BF08BD01B500BF042269461B480068903000F03AF818B919480099C0F8801400BF27
:4096000008BD01B500BF0422694613480068943000F02AF818B911480099C0F8841400BF08BD00F01F02012191400D4A430942F82310704700F01F0201219140094A43097D
:4096400042F82310704700000CED00E00000FA05F60600200B070020A8030020081F002080E100E080E200E070B504460D461646324629462046EFF7CAFB70BD2DE9F34F70
:4096800082B0844600BF00210A460B460E460F46002001908046009063E09CF80000A0F13004E5179CF800002E2838D1B8F1000F0CD1F9494FF00009A2FB010A03FB01A18B
:4096C00002FB0919861949EB07071FE0B8F1010F0CD1F2494FF00009A2FB010A03FB01A102FB0919861949EB07070FE0B8F1020F0CD14FF47A714FF00009A2FB010A03FB68
:4097000001A102FB0919861949EB070708F1010000F0FF0800200090002213461BE09CF80000C0B1009810B922462B460FE0009801280CDB0A214FF0000B9146A9FB010E9B
:4097400003FB01E102FB0B19021949EB05030098401CC0B200900CF1010C0198401CC0B2019003990198884297DBB6185F413046394604B0BDE8F08F2DE9F04F8346894600
:40978000924600BF00BF51465846FFF777FF05460E4651464846FFF771FF07468846781B78EB060001DA012407E0E81B76EB080002DA4FF0FF3400E000242046BDE8F08F42
:4097C000F0B585B00546B6A2B8A101A822F0A8FB1022294601A8FFF7CFFF00283CDDB44890F82464012434E0062C0CD2DFE804F00B0C09070503AF4F08E0AF4F06E0AF4FDF
:4098000004E0AF4F02E000BFAE4F00BF00BF40F6C41000900222694607F56070FFF724FFB44204D1BDF80000A149A1F880034FF47A5000900222694607F28230FFF714FF2E
:40984000B44204D1BDF800009949A1F88203601CC4B2052CC8DD00BF05B0F0BD2DE9F04105460E4617463A4631462846EFF745FB044604B103DF2046BDE8F081F0B585B07A
:40988000054691A289A101A822F04AFB1022294601A8FFF771FF00282FDD854890F82474012427E0062C0CD2DFE804F00B0C09070503804E08E0804E06E0804E04E0804E1F
:4098C00002E000BF7F4E00BF00BF042206F5C6716846FFF7C3FF0422694606F56270FFF7C3FEBC4204D19DED000A714880EDE20A601CC4B2052CD5DD00BF05B0F0BDF0B551
:4099000085B0054673A269A101A822F009FB1022294601A8FFF730FF00282BDD644890F82464012423E0062C0CD2DFE804F00B0C090705035F4F08E05F4F06E05F4F04E090
:409940005F4F02E000BF5F4F00BF00BF002000900122694607F19700FFF786FEB44204D19DF80000524981F89700601CC4B2052CD9DD00BF05B0F0BD2DE9F04186B0054614
:4099800057A24AA102A822F0CBFA1022294602A8FFF7F2FE002836DD002001900026444890F8247400242BE0062C13D2DFE804F0130F0C090603DFF8FC800FE0DFF8F88081
:4099C0000CE0DFF8F88009E0DFF8F48006E0DFF8F48003E000BFDFF8148100BF00BF042201A908F1B400FFF73FFEBC4206D130490198C1F8B4000846C0F89860601CC4B247
:409A0000052CD1DD00BF06B0BDE8F081F0B587B0064637A225A103A822F082FA1022314603A8FFF7A9FE002869DD214890F82474002483E0062C0ED2DFE804F00E0B090757
:409A400005031C4D0AE01C4D08E01C4D06E01C4D04E01C4D02E000BF244D00BF00BF042205F1300101A8FFF7F9FE13208DF809000198FDF73EFB18B90198FDF764FB18B1B5
:409A800090208DF808003EE00198FDF754FBA8B313208DF8080036E000CA9A3B40420F00322E342E302E35330000000025730000081F0020581B00687017006888130068DA
:409AC000A00F0068B80B0068322E342E302E343400000000322E332E302E333000000000322E322E302E343600000000D0070068322E322E302E31380000000000E021E0EB
:409B0000FF208DF8080001220DF1090105F1B300FFF7AAFD012202A905F1B200FFF7A4FDBC4209D19DF80910FE4880F8B3109DF80800FC4981F8B200601CC4B2052C7FF74E
:409B400079AF00BF07B0F0BDF0B585B00546F6A2AFF2A80101A822F0E3F91022294601A8FFF70AFE00282DDDEE4890F8246401200090002423E0062C0ED2DFE804F00E0B7E
:409B800009070503EA4F0AE0EA4F08E0EA4F06E0EA4F04E0EA4F02E000BFEA4F00BF00BF0122694607F14B00FFF75EFDB44204D19DF80000DB4981F84B00601CC4B2052CAB
:409BC000D9DD00BF05B0F0BDF0B587B00546DEA2AFF2281103A822F0A3F91022294603A8FFF7CAFD002839DDCE4890F82474002431E0062C0ED2DFE804F00E0B0907050304
:409C0000CB4E0AE0CB4E08E0CB4E06E0CB4E04E0CB4E02E000BFCB4E00BF00BF012206F1280102A8FFF71AFE9DF80800042810D0B2EE040A8DED010A042201A906F5FC70C5
:409C4000FFF712FDBC4204D19DED010AB54880ED7E0A601CC4B2052CCBDD00BF07B0F0BDF0B585B00646BAA2AFF2C01101A822F057F91022314601A8FFF77EFD002843DD8D
:409C80000727B6A2AFF2DC1101A822F049F91022314601A8FFF770FD002800DD09270020009000242DE0062C0ED2DFE804F00E0B090705039E4D0AE09E4D08E09E4D06E051
:409CC0009E4D04E09E4D02E000BF9E4D00BF00BF042205F130016846FFF7C0FD009838440090009814280BD30422694605F13000FFF7BAFC9348854202D18A4900980863AA
:409D0000641C062CCFD300BF05B0F0BD2DE9F3410D468449ADEB01040846071988482618AAB239463046FFF79FFC7E48071983482618AAB239463046FFF796FC79480719A0
:409D40007D482618AAB239463046FFF78DFC7548071978482618AAB239463046FFF784FC7048071972482618AAB239463046FFF77BFCBDE8FC812DE9FE4F81468A46174667
:409D800098460020009000262D2200233846414622F03CF805462D2200233846414622F035F8934615B9BBF1000F35D0D5B1002416E0C4EB041000EB400048440290C4EB6F
:409DC000041000EB4000504401902D22DDE90110FFF74AFC0646009931430091601CC4B2AC42E6D3BBF1000F18D0C5EB051000EB400048440290C5EB051000EB40005044E5
:409E000001901FFA8BF2DDE90110FFF72DFC064600993143009101E0402000900098BDE8FE8F01B500BF012269464F4800682D30FFF71AFC20B99DF800103A4880F81D1428
:409E400000BF08BD2DE9FE4F81468A46174698460020009000262D2200233846414621F0D5FF05462D2200233846414621F0CEFF934615B9BBF1000F35D0D5B1002416E050
:409E8000C4EB041000EB400048440290C4EB041000EB4000504401902D22DDE90110FFF7DDFC0646009931430091601CC4B2AC42E6D3BBF1000F18D0C5EB051000EB400078
:409EC00048440290C5EB051000EB4000504401901FFA8BF2DDE90110FFF7C0FC064600993143009101E0402000900098BDE8FE8F3EB5002002900A200190002000904FF438
:409F00007B71084822F09DF9B021184822F099F94FF458711548B03022F093F9012201A9114825E0081F0020322E322E302E3200581B00687017006888130068A00F0068DB
:409F4000B80B0068D0070068322E322E302E3100322E312E302E373300000000322E312E302E353400000000A8030020F822002000689830FFF778FB0122FB4801689831E5
:409F800002A8FFF76BFC9DF80800401CC0B20190012201A9F44800689830FFF765FB0122F1480168983102A8FFF758FC9DF808009DF80410884207D0EC48007840F080004A
:409FC000EA49087001248CE00122E74801682E316846FFF743FC9DF8000044284CD0FF224FF47B71E24822F002F94FF47B720023DF49E048FFF7BFFE4FF47B720023DC49B6
:40A00000DD48FFF7B8FE4FF47B720023D849DB48FFF7B1FE4FF47B720023D549D848FFF7AAFE4FF47B720023D149D648FFF7A3FE4FF47B720023CE49D348FFF79CFE4FF46A
:40A040007B71CB4822F0FDF8B0220023CF494FF0D040FFF790FE4FF458720023CB49B031CB48FFF788FE4420009001226946BE4800682E30FFF7F8FAB02200234FF0D04187
:40A08000C248FFF7DFFE4FF458720023C049BF48B030FFF7D7FE0122B34801682D31BB482D30FFF7DBFBB24890F81D04672810D001246720FFF7B5FE4FF47B71AC4822F02B
:40A0C000C0F84FF47B720023A949AA48FFF753FE07E002244FF47B720023A649A448FFF7B1FE20463EBD10B5AA48EEF73FFE0446204610BD70B58CB00024002008900990BD
:40A100000A900B9004900590069007900090019002900390954908709F49087001200870FFF7E1FFFFF7E4FE9C4908709C4AAFF2846108A821F0F4FE04A81AF097FF99A14F
:40A1400004A822F0A5F808B1012000E00020054645B196A01AF076FF92A01AF073FF97A01AF056FF04A81AF065FF102204A908A8FFF702FB044689480078012806D1002021
:40A180008549087008A81AF043FFC3E0002CFCD0002005F069FB002005F0B9FB08A81AF037FF002C39DA0020FFF73BFEFF224FF47B716F4822F01BF84FF47B7200236C49CE
:40A1C0006C48FFF7D8FD4FF47B72002368496A48FFF7D1FD4FF47B72002365496748FFF7CAFD4FF47B72002361496548FFF7C3FD4FF47B7200235E496248FFF7BCFD4FF403
:40A200007B7200235A496048FFF7B5FD4FF47B71574822F016F803DF7CE06AA2AFF27471684621F07DFE102204A96846FFF7A4FA002838DD0020FFF7F4FDFF224FF47B716E
:40A240004B4821F0D4FF4FF47B72002348494948FFF791FD4FF47B72002345494648FFF78AFD4FF47B72002341494448FFF783FD4FF47B7200233E494148FFF77CFD4FF48E
:40A280007B7200233A493F48FFF775FD4FF47B72002337493C48FFF76EFD4FF47B71344821F0CFFF03DF4AA2AFF60001684621F037FE102204A96846FFF75EFA002811DD81
:40A2C000012007F04EFC01212948B130FFF71EFD1AF0A0F830B10320F1F7AAFE01213F48FFF714FD04A8FFF7BBFC04A8FFF76CFC04A8FFF729FC04A8FFF788FB04A8FFF7A0
:40A300003BFB04A8FFF7FBFA04A8FFF7B7FA04A8FFF756FA0020FCF7B8FC0020FCF7C8FCFDF756F80646FCF754FF1B4800780CB070BD19480078704701B500BF01226946FE
:40A34000094800683430FFF78FF920B99DF80010074880F8241400BF2148C16B0220DFF884C000DF08BD0000A8030020A1030020081F0020D0070068B80B0068A00F006839
:40A380008813006870170068581B0068F8220020F401006800380040A2030020A00300209CBE0008322E302E3100000030303030303030303030303000000000322E302EEA
:40A3C000302E3100322E302E302E363500000000322E312E302E333900000000BB200020F03F002081F303087CB505460E46FE4C042204F1340101A8FFF730FA012204F1AA
:40A40000B1016846FFF72AFA0198854205D19DF80000B04201D101207CBDF44C042204F1340101A8FFF71AFA012204F1B1016846FFF714FA0198854205D19DF80000B0423D
:40A4400001D10220E8E7EA4C042204F1340101A8FFF704FA012204F1B1016846FFF7FEF90198854205D19DF80000B04201D10320D2E7E04C042204F1340101A8FFF7EEF924
:40A48000012204F1B1016846FFF7E8F90198854205D19DF80000B04201D10420BCE7D64C042204F1340101A8FFF7D8F9012204F1B1016846FFF7D2F90198854205D19DF811
:40A4C0000000B04201D10520A6E70020A4E738B5C54C042204F5EC716846FFF7BFF940F2FD110098884201D0012038BDBF4C042204F5EC716846FFF7B1F940F2FD1100982F
:40A50000884201D00220F0E7B94C042204F5EC716846FFF7A3F940F2FD110098884201D00320E2E7B34C042204F5EC716846FFF795F940F2FD110098884201D00420D4E768
:40A54000AD4C042204F5EC716846FFF787F940F2FD110098884201D00520C6E70020C4E710B54FF47B71A54821F06BFE4FF47B720023A249A248FFF7FEFB10BD10B54FF4EB
:40A580007B719E4821F05DFE4FF47B7200239B499B48FFF7F0FB4FF47B72002397499248FFF7E9FB4FF47B72002394498F48FFF7E2FB4FF47B72002390498D48FFF7DBFBD4
:40A5C0004FF47B7200238D498A48FFF7D4FB4FF47B72002389498848FFF7CDFB4FF47B71864821F02EFE10BD2DE9F0410446884615461F463CB982482E183A464146304640
:40A60000FFF732F830E0012C07D177482E183A4641463046FFF728F826E0022C07D173482E183A4641463046FFF71EF81CE0032C07D16F482E183A4641463046FFF714F838
:40A6400012E0042C07D16B482E183A4641463046FFF70AF808E0052C06D167482E183A4641463046FFF700F8BDE8F0812DE9F04104460F46154698463CB961482E18424681
:40A6800031463846FFF7EAF830E0012C07D156482E18424631463846FFF7E0F826E0022C07D152482E18424631463846FFF7D6F81CE0032C07D14E482E1842463146384600
:40A6C000FFF7CCF812E0042C07D14A482E18424631463846FFF7C2F808E0052C06D146482E18424631463846FFF7B8F8BDE8F08110B5424890F82444062C2CD2DFE804F07A
:40A700002C030B131B234FF47B7200233B493648FFF731FB21E04FF47B72002337493348FFF729FB19E04FF47B72002333493048FFF721FB11E04FF47B7200232F492D482B
:40A74000FFF719FB09E04FF47B7200232B492A48FFF711FB01E000BF00BF00BF10BD70B505460E4631462846FFF73EFE0446062C6CD2DFE804F06C03152747594FF47B72F5
:40A78000002319491D48FFF75DFB4FF47B7200231A491B48FFF7EFFA0120FFF7CDFD62E04FF47B72002311491448FFF74BFB4FF47B72002311491248FFF7DDFA0220FFF715
:40A7C000BBFD50E04FF47B72002309490B48FFF739FB4FF47B72002308490948FFF7CBFA0320FFF7A9FD3EE0B80B0068A00F00688813006870170068581B0068081F00206C
:40A80000D00700684FF47B72002339493948FFF719FB4FF47B72002336493748FFF7ABFA0420FFF789FD1EE04FF47B72002333493048FFF707FB4FF47B7200232D492E4871
:40A84000FFF799FA0520FFF777FD0CE000BFFFF787FE0020FFF770FD002029494860222013F092FF00BF00BF04B103DF70BD4FF40050704710B51F4890F82404062831D26E
:40A88000DFE800F031030C151E271E4C042219493C3104F13C00FEF7E7FE25E01A4C042214493C3104F13C00FEF7DEFE1CE0174C042210493C3104F13C00FEF7D5FE13E049
:40A8C0000B4C04220B493C3104F13C00FEF7CCFE0AE00A4C042207493C3104F13C00FEF7C3FE01E000BF00BF00BF10BD0848704770170068081F0020D0070068581B0068DE
:40A90000E42F0020B80B0068A00F006888130068AFD3D73B10B51CF03AF9FE49086009F06DF8FC4880ED010A10BD10B5FA4890F84A0002281FD1F94890ED020ADFEDF80AE6
:40A94000B4EEE00AF1EE10FA0ADBFBF707FBC4B223467D22EF490C3101200CF0A9FC2EE0FBF7FCFAC4B223467D22EA490C3100200CF09EFC23E0E948D0ED010AE648B0F868
:40A98000BE0100EE100AB8EE400AF4EEC00AF1EE10FA0ADBFBF7E2FAC4B22346FA22DD490C3101200CF084FC09E0FBF7D7FAC4B22346FA22D7490C3100200CF079FC10BD3B
:40A9C00010B52DED048B19F03DFD002867D0FFF7ACFFEFF73FFD18B10020CE49087261E0CC48007A60B9CB4890F82000002859D10120C84908721CF0CAF8C649086051E0F3
:40AA0000C448007A01280CD1C249C86947F230511CF0C3F8A0B30220BE490872FFF77AFF40E0BC48007A02283CD108F0E7FFB948D0ED010A30EEC00A10EE104A204626F030
:40AA400085F941EC190BB0EE490AF0EE690A22F057FDB0EE408AF0EE608A9FEDB20B53EC102B51EC180B25F079FF0ED2A94890F82000012805D10020A649487201200872A3
:40AA800010E00120A34948720CE0A24908684FF4FA611CF082F828B1FFF73CFF02E000209C494872BDEC048B10BD9C4981F8900070479A4981F838007047F0EE400A9FED20
:40AAC0009B0A20EE800A704770B52DED0A8B0446914890F8BD010E287DD2DFE800F07C355DFB36FCF9F87C7C077C7CF7EFF7AEFC10EE105A284626F029F941EC1A0BB0EE41
:40AB00004A0AF0EE6A0A22F0FBFCB0EE409AF0EE609A51EC190B25F0DDFAA0619FED840A84ED1C0A94ED060A84ED010AEFF7D6FC18B10020FFF7BDFF02E00320FFF7B9FF04
:40AB40000320FFF7B2FF34E300BF7A4800781AF0A5F820B19FED780A84ED060A03E09FED740A84ED060A754800781AF097F820B19FED710A84ED1C0A03E09FED6D0A84EDF2
:40AB80001C0A0320FFF795FF0320FFF78EFF94ED060A84ED010A0CE36648007819F042FE00EE100AF8EE400A9FED651A9FED650A10EE810A84ED0C0AE16821611BF0E7FFA7
:40ABC000E060D4E90310091A6161D4ED0C0AB0EE600A0A2100E0DDE204F118000AF0D0F894ED060ADFED580AB4EEE00AF1EE10FA03D20020FFF75DFF0FE094ED060AF0EE0F
:40AC0000040AB4EEE00AF1EE10FA03DD0120FFF750FF02E00320FFF74CFF0320FFF745FF94ED0C0AB5EEC00AF1EE10FA02D29FED408A01E094ED068A94ED0F0A84ED100A7A
:40AC400084ED0F8A94ED050AB8EE400ADFED3A0A80EE201A11EE105A284626F077F841EC1A0B94ED0F0AD4ED100A30EE600A10EE101A084626F06AF841EC1C0BB0EE4C0AB1
:40AC8000F0EE6C0A22F03CFCB0EE40BAF0EE60BA53EC1A2B51EC1B0B25F00AFB41EC190B25F018FA60639FED220A84ED1C0AB0EE480AFFF702FF84ED010AD4ED0D0AB0EE02
:40ACC000600AFFF7FAFE84ED020A72E253E2A5E110E100E067E01748007819F0A3FD00EE100AB8EE400ADFED160A20EE200ADFED170A80EE201A84ED0C1AD4ED0C0AB0EE1B
:40AD0000600A0A2104F118000AF03AF894ED060A1EE0000008270020081F00202C27002000C0DA44000000401857B63FC0A9064600000000D606002000007A44DA060020BC
:40AD40003333533A9A99193FCDCCCCBE0CAC233FDFEDF80AB4EEE00AF1EE10FA03D20020FFF7A7FE0FE094ED060ADFEDF30AB4EEE00AF1EE10FA03DD0120FFF79AFE02E016
:40AD80000320FFF796FE0320FFF78FFE1FED180A84ED1C0AD4ED060AB0EE600AFFF78DFE84ED010A05E2E548007819F03BFD00EE100AF8EE400A1FED1E1A1FED1E0A10EE2A
:40ADC000810A84ED0C0AD4ED0C0AB0EE600A0A2104F1180009F0D4FF94ED060A5FED260AB4EEE00AF1EE10FA03D20020FFF761FE0FE094ED060AF0EE040AB4EEE00AF1EEBB
:40AE000010FA03DD0120FFF754FE02E00320FFF750FE94ED0C0AB5EEC00AF1EE10FA02D21FED3D8A01E094ED068AC548007819F0F9FC00EE100AF8EE400A1FED3F1A1FEDC4
:40AE40003F0A10EE810A84ED220AD4ED220AB0EE600A0A2104F1700009F092FF94ED1C0A5FED470AB4EEE00AF1EE10FA03D20020FFF71BFE0FE094ED1C0AF0EE040AB4EE73
:40AE8000E00AF1EE10FA03DD0120FFF70EFE02E00320FFF70AFE94ED220AB5EEC00AF1EE10FA02D25FED5E8A01E0D4ED1C8AB0EE480AFFF702FEB0EE401AB0EE680AFFF782
:40AEC000FCFD31EE400A10EE105A284625F03EFF41EC1A0BB0EE4A0AF0EE6A0A22F010FBB0EE409AF0EE609A51EC190B25F0F2F860605EE19148007819F094FC00EE100A74
:40AF0000B8EE400A5FED720A20EE200A5FED710A80EE201A84ED0C1AD4ED0C0AB0EE600A0A2104F1180009F02BFF94ED060ADFED810AB4EEE00AF1EE10FA03D20020FFF799
:40AF4000B8FD0FE094ED060ADFED7B0AB4EEE00AF1EE10FA03DD0120FFF7ABFD02E00320FFF7A7FD7648007819F05CFC00EE100AB8EE400A5FED8E0A20EE200A5FED8D0A0A
:40AF800080EE201A84ED221AD4ED220AB0EE600A0A2104F1700009F0F3FE94ED1C0ADFED650AB4EEE00AF1EE10FA03D20020FFF77CFD0FE094ED1C0ADFED5F0AB4EEE00ABB
:40AFC000F1EE10FA03DD0120FFF76FFD02E00320FFF76BFD94ED060AD4ED1C0A30EE600A10EE101A084625F0B1FE41EC1B0BB0EE4B0AF0EE6B0A22F083FAB0EE40AAF0EEDA
:40B0000060AA51EC1A0B25F065F809EE100AB0EE490AFFF752FD84ED010ACAE06421E0681BF0BBFD00287AD01BF0B1FDE06094ED0F0A84ED100A414800781DF03DFD00EE6F
:40B04000100AB8EEC00A84ED0F0A94ED0F0AD4ED100A30EE600A84ED0C0A94ED0C0ADFED390A80EE201A84ED0C1A94ED250A84ED260A354800781DF01FFD00EE100AB8EE36
:40B08000C00A84ED250A94ED250AD4ED260A30EE600A84ED220A94ED220ADFED2A0A80EE201A84ED221AD4ED0C0AB0EE600A032104F1180009F064FED4ED220AB0EE600AFE
:40B0C000032104F1700009F05BFE94ED060AD4ED1C0AB4EEE00AF1EE10FA04DD94ED060A84ED010A03E094ED1C0A84ED010AEFF7F5F918B10020FFF7DCFC14E094ED1C0A6E
:40B10000D4ED060A30EE600AF3EE090AB4EEE00AF1EE10FA04DD0220FFF7CBFC03E029E00320FFF7C6FCEFF7E6F978B10020FFF7BCFC1FE0CDCCCC3C33339F40D606002029
:40B14000D9060020CDCCCC3DDA06002094ED060AD4ED1C0A30EE600AF3EE090AB4EEE00AF1EE10FA03DD0220FFF79FFC02E00320FFF79BFC1DE09FEDF90A84ED0C0A9FED01
:40B18000F70A84ED010A0320FFF793FC0320FFF78CFC0EE09FEDF10A84ED0C0A9FEDEF0A84ED010A0020FFF784FC0020FFF77DFC00BF00BFBDEC0A8B70BD10B519F055F9A2
:40B1C000D0B1FAF7CBFEC4B22346FA22E44900200CF06EF89FEDE10AE24880ED060A9FEDDF0A80ED060A032180F8381080F890100020DD4948722EE0DA48FFF765FCDB48B4
:40B20000B0F8BE0118B90220D549087521E0D548D0ED010AD548B0F8BE0100EE100AB8EE400AF4EEC00AF1EE10FA09DBFAF796FEC4B22346FA22CA4901200CF039F808E075
:40B24000FAF78CFEC4B22346FA22C54900200CF02FF8FFF7B5FB10BDC3494872704731B50024BDF80000C82803DDC8200090022406E0BDF80000012802DA01200090032472
:40B2800000BF02226946BA48006800F5DF70FEF7EBF920B9BDF80000B449A1F8BE0100BF204638BD31B50024BDF80000B0F5FA7F04DD4FF4FA700090022406E0BDF80000BC
:40B2C000012802DA01200090032400BF02226946A748006800F5DF70FEF7C6F920B9BDF80000A249A1F8BE0100BF204638BD31B50024BDF80000322803DD322000900224A4
:40B3000006E0BDF80000012802DA01200090032400BF022269469648006800F5DF70FEF7A3F920B9BDF800009049A1F8BE0100BF204638BD31B50024BDF80000C82803DD80
:40B34000C8200090022406E0BDF80000012802DA01200090032400BF022269468448006800F5DF70FEF780F920B9BDF800007F49A1F8BE0100BF204638BD31B50024BDF8B8
:40B38000000040F26351884203DD08460090022406E0BDF80000012802DA01200090032400BF022269467248006800F5DF70FEF75BF920B9BDF800006C49A1F8BE0100BFE6
:40B3C000204638BD31B50024BDF8000045F2CC01884203DD08460090022406E0BDF80000012802DA01200090032400BF022269465F48006800F5DF70FEF736F920B9BDF872
:40B4000000005A49A1F8BE0100BF204638BD10B52DED028BB0EE408A0024544890F8BD010B2839D2DFE800F0061B07111C081226381D2F0000BF00BFBCEEC80A10EE101AED
:40B4400088B2FFF7BFFF04462FE000BFBCEEC80A10EE101A88B2FFF790FF044625E000BF00BFBCEEC80A10EE101A88B2FFF762FF04461AE0BCEEC80A10EE101A88B2FFF749
:40B4800036FF044611E0BCEEC80A10EE101A88B2FFF708FF044608E0BCEEC80A10EE101A88B2FFF7DCFE044600BF00BF4020F1F767FE0020FFF7D0FE2046BDEC028B10BD9F
:40B4C00010B52DED020B00BF042269462848006800F5E670FEF7C8F820B99DED000A234880ED730A00BF2348016D0120DFF888C000DF1CBD10B52DED020B00BF0422694622
:40B500001B48006800F5E470FEF7AEF820B99DED000A164880ED720A00BF1648016D0120DFF854C000DF1CBD10B52DED020B00BF042269460E48006800F5E270FEF794F853
:40B5400020B99DED000A094880ED710A00BF0948016D0120DFF820C000DF1CBD00000000E82700202C27002008270020081F0020A4030020F03F002081F3030810B52DED6B
:40B58000020B00BF04226946FE48006800F5E070FEF76AF820B99DED000AFB4880ED700A00BFFA48016D0120DFF8E4C300DF1CBD10B5F54890F830000A2818D1F24890F8AC
:40B5C000BD010A2813D19FEDF30AFFF720FF9FEDF20AFFF7D3FF9FEDF10AFFF7A5FF9FEDF00AFFF787FF9FEDEF0AFFF769FFE64890F83000702819D1E34890F8BD010A2878
:40B6000014D19FEDE90AFFF702FF9FEDE80AFFF7B5FF9FEDE70AFFF787FF9FEDE60AFFF769FF9FEDE50AFFF74BFF18E0D64890F8BD010A2813D19FEDDC0AFFF7E8FE9FEDAD
:40B64000D60AFFF79BFF9FEDD50AFFF76DFF9FEDDB0AFFF74FFFBBEE040AFFF731FFCA4890F8BD01012804D1B7EE000AFFF7CFFE44E0C54890F8BD01022804D19FEDD00A57
:40B68000FFF7C5FE3AE0C04890F8BD01032804D1B3EE040AFFF7BBFE30E0BB4890F8BD01042804D11FED530AFFF7B1FE26E0B64890F8BD01052804D19FEDC20AFFF7A7FE64
:40B6C0001CE0B14890F8BD01062804D19FEDBE0AFFF79DFE12E0AC4890F8BD01072804D1B1EE040AFFF793FE08E0A74890F8BD01092803D19FEDB40AFFF789FE10BD10B548
:40B70000A14890F8BD010A280DD19F4890F830000A2803D1FA20FFF7C5FD03E04FF49670FFF7C0FD00E000BF00BF10BD00B589B018F088FE002878D0934890F8BD010C2808
:40B7400074D2DFE800F07306292A4D74759873FEFDEB0020009001900290034602469B4903900846007818F06EFF002000900190029003460246964903900846007818F01F
:40B7800062FF01219148007819F00BFB01219048007819F006FB6DE100BF002000900190029003460322894903900846007818F04AFF002000900190029003460322844952
:40B7C00003900846007818F03EFF03217F48007819F0E7FA03217E48007819F0E2FA49E101200021009101910B460A46CDE9021076490846007818F026FF0120002100919A
:40B8000001910B460A46CDE9021071490846007818F019FF01216D48007819F0C2FA01216B48007819F0BDFA24E124E1FDE000BF0020009001900290034603226349039026
:40B840000846007818F0FFFE0020009001900290034603225E4903900846007818F0F3FE00215A48007819F09CFA00215848007819F097FAFEE0002000900190029003461C
:40B880000222524903900846007818F0DCFE0020009001900290034603224D4903900846007818F0D0FE002000900190029003460222484903900846007818F0C4FE022171
:40B8C0004248007819F06DFA02214248007819F068FA002000900190034614220121029004A81CF005FF04A85FEDE40A9FED3A0A0223002239490090344800781CF0E0FD2A
:40B9000004A85FEDEA0A9FED340A0223032234490090304800781CF0D3FDABE0002000900190029003460222284903900846007818F089FE0020009001900290034601E00D
:40B9400075E073E00322224903900846007818F07AFE0020009001900290034602221D4903900846007818F06EFE06211748007819F017FA06211748007819F012FA0020F8
:40B9800000902FE0A4030020081F0020F03F002081F3030800007A43C6DCB53DB8AF833E52B8444114AE4740000096436744293EE5F25F3E52B862416666E6C133331B417A
:40B9C000000016430080BB440000C842D6060020D9060020DA0600200050434700040040000001400190034614220121029004A81CF07EFE04A8DFEDF90A1FED090A022354
:40BA00000022F7490090F74800781CF059FD04A8DFEDF20A1FED100A02230322F2490090F24800781CF04CFD24E000BF00BF002000900190029003460322EA49039008466E
:40BA4000007818F000FE002000900190029003460322E74903900846007818F0F4FD0121E048007819F09DF90121E148007819F098F900BF00BFDF4890F8BD01DE4908703D
:40BA80000020FFF7E9FB0020DC49087209B000BDDB49097D012900D100E0002108467047D748407D7047D648007D08B9012070470020FCE7D34909880143D24A118070478D
:40BAC000F7EE000AB0EE600A7C220270C94A92F8BD210B2A1DD2DFE802F00611070812090A161C13190000BF00BF00BF00BF01224270DFEDC50AB0EE600A0BE000BF00BF61
:40BB00000222427006E00422427003E00522427000E000BF00BFB84AD2ED060A60EE800AFCEEE00A10EE902A91B281700A0AC270B14AD2ED1C0A60EE800AFCEEE00A10EE1E
:40BB4000902A91B201710A0A4271AA4AB2F8BE1181710A0AC2717047A74890ED010A704701B500BF01226946A848006800F2BD10FDF77AFD20B99DF800009E4981F8BD01AF
:40BB800000BFFFF715FD012000F0C3FC1D20F1F7F7FA08BD01B500BF022269469B48006800F5E870FDF760FD20B9BDF800009149A1F8D00100BF08BD00208E4991F8BD113E
:40BBC0000B2916D2DFE801F0160C09060D0A070F1117130000BF01200EE000BF01200BE000BF012008E0012006E0012004E0012002E000BF00BF00BF00BF704700207D49CF
:40BC000091F8BD110B2919D2DFE801F0190E0A060F0B0711131A150000BF40F2635010E000BF45F2CC000CE000BFC82009E0322007E0C82005E04FF4FA7002E000BF00BF46
:40BC400000BF00BF704700206B4991F8381009B9142012E0684991F83810012901D116200BE0654991F8901009B9152005E0624991F89010012900D11720704770B50424A6
:40BC8000634880780A2876D2DFE800F0051376E1E1E1E1DBDDDF00205D490870C8808860FFF778FF5A4880785949487001208870CEE0FFF7C8FF564908700846007810B116
:40BCC0000720887056E05248806820B91AF05FFF4F4988604EE04E4988684FF47A711AF05CFF002846D0FFF737FFBCEEC00A10EE100A85B22846FFF74DFF3E48B0F8AC00AD
:40BD000068B13C48B0F8AC003A49B1F8D011884205DD3848B0F8AC003D49C88021E03548B0F8D001002803DC01203949C88018E0304890F8BD01032804D02E4890F8BD015D
:40BD4000062805D12B48B0F8D00100F5FA7006E02848B0F8D0018000032190FBF1F02C49C88002202A4988701AF011FF28498860002008736CE06AE0FFF7EEFE2448C08811
:40BD800000EE900AF8EE600AB4EEE00AF1EE10FA05DB1F48007B401C1D49087302E000201B490873FFF74FFF194908700846007810B10720887043E01548007B042829DB67
:40BDC0001348C08800EE900AF8EE600AB0EE600AFFF71DFB09200E49887031E00000000000040040D606002000000140DA060020D9060020081F00202C27002008270020A0
:40BE0000E8270020B0030020C0A90646A4030020002800205F49886841F288311AF0BDFE70B15C48C08800EE900AF8EE600AB0EE600AFFF7ECFA07205649887018200870BC
:40BE400006E0012404E0022402E0032400E000BF00BF5048007818B14E490878F8F746FE204670BD4B48807870474A4800787047002048498870C870704701B500BF02225C
:40BE8000694645480068AC30FDF7EEFB20B9BDF800004249A1F8AC0000BF08BD10B52DED028B3E4890F8BD0103280ED03B4890F8BD01062809D0394890F8BD01022804D06D
:40BEC000364890F8BD0105280CD113F0F7FE10B1012806D102E0B7EE008A02E09FED308A00BF01E0B7EE008AB0EE480ABDEC028B10BDB7EE000AF0EE400A284890F8BD0133
:40BF00000B2815D2DFE800F0060F070810090A121411130000BF00BF00BF00BF1FED460AF0EE400A05E000BF00BF00BF00BF00E000BF00BF1B4890ED060A20EE200A704701
:40BF4000B7EE000AF0EE400A144890F8BD010B2815D2DFE800F0060F070810090A121411130000BF00BF00BF00BF1FED590AF0EE400A05E000BF00BF00BF00BF00E000BFD3
:40BF800000BF084890ED1C0A20EE200A70470648407A704700280020A4030020081F0020D7A3DC402C2700200827002010B518F05CFA18B1F94890F8860348B9F9F7CEFF77
:40BFC000C4B22346FA22F64903200BF071F917E0F448007818F062FE48B1F9F7BFFFC4B22346FA22EE4901200BF062F908E0F9F7B5FFC4B22346FA22E94900200BF058F9F7
:40C0000010BD10B518F031FA48B9F9F7A7FFC4B22346FA22E44903200BF04AF917E0E348007818F03BFE48B1F9F798FFC4B22346FA22DD4901200BF03BF908E0F9F78EFFEA
:40C04000C4B22346FA22D84900200BF031F910BD10B518F00AFA48B9F9F780FFC4B22346FA22D34903200BF023F933E008F050F8C0B1D048007818F011FE48B1F9F76EFF3F
:40C08000C4B22346FA22CA4900200BF011F921E0F9F764FFC4B223464122C54901200BF007F917E0C348007818F0F8FD48B1F9F755FFC4B22346FA22BD4901200BF0F8F8CC
:40C0C00008E0F9F74BFFC4B223464122B84900200BF0EEF810BDB848007D704710B5B7480BF04AF918F0C1F948B1F9F737FFC4B223464122B04903200BF0DAF81BE0B048D8
:40C10000007818F0CBFD18B9AC48407A012809D1F9F724FFC4B223464122A74901200BF0C7F808E0F9F71AFFC4B223464122A24900200BF0BDF8A3484078002866D0A2483C
:40C14000007800F0010070B9FFF7C5FF012800D100E0002040009C4908700846007840F0010008703EE098480078C0F34000D0B1FFF7B1FF012806D09348007840F0080053
:40C18000914908702EE0FFF7A6FF01282AD18E48007800F0080028B38B48007840F00400894908701EE088480078C0F34000C8B9FFF791FF012806D18348007840F00400BF
:40C1C000814908700EE0FFF786FF01280AD07E48007800F0040028B17B48007840F00800794908707848007800F0040070B17648007800F0080048B1002073490870734856
:40C20000D0F818111020DFF8C8C100DF10BD10B5032418F017F940B16E48007818F03EFD08B101243EE000243CE018F0F3F8002838D06948007818F031FD002832D06748D4
:40C24000007818F02BFD40B16248007818F026FD08B1012426E0002424E06148007818F01DFD30B15B48007818F018FD08B1012418E05B48007818F011FD30B9554800786B
:40C2800018F00CFD08B901240CE05548007818F005FD30B14F48007818F000FD08B9002400E00124204610BD70B5044618F0DDF848B1F9F753FEC5B22B46FA22494901202D
:40C2C0000AF0F6FF59E06078022824D1FFF79FFF012809D1F9F742FEC5B22B46FA22414901200AF0E5FF48E0FFF791FF48B9F9F735FEC5B22B46FA223A4900200AF0D8FF81
:40C300003BE0F9F72BFEC5B22B46FA22354903200AF0CEFF31E06078012817D1FFF777FF012809D1F9F71AFEC5B22B46FA222D4901200AF0BDFF20E0F9F710FEC5B22B46B5
:40C34000FA22284900200AF0B3FF16E0607803280AD1F9F703FEC5B22349487A2B46FA2220490AF0A5FF08E0F9F7F8FDC5B22B46FA221C4903200AF09BFF70BD01B500BFD7
:40C3800004226946194800689830FDF76DF918B902490098C1F8980000BF08BD081F002058280020A4060020882800202807002070280020A906002010280020A02800209D
:40C3C000A806002000FF0020BC030020F03F002081F30308A1060020A0060020AC060020D106002040280020B8280020A403002010B52DED028B18F00DF840B1FE480078D6
:40C4000018F04CFC08B101243BE0002439E018F02CF808B1032434E0F748007803F036FBB0EE408AF548B0F8800300EE100AB8EE400AB4EEC80AF1EE10FA0DD8EF48B0F892
:40C44000820300EE100AB8EE400AB4EEC80AF1EE10FA01DB012413E0E848B0F8800300EE100AB8EE400AB4EEC80AF1EE10FA06DDE24890F8BC01022801D1032400E00024C5
:40C4800000BF2046BDEC028B10BD70B50446A078022802D0A07801280CD1F9F75FFDC5B2FFF7A6FF06462B464FF41672D4490AF0FFFE18E0A07803280BD1F9F74FFDC5B2EF
:40C4C000D049487A2B464FF41672CD490AF0F0FE09E0F9F743FDC5B22B464FF41672C84903200AF0E5FEC648007D58B9C648007840B1C249D1F8B400FFF740FF0020C2494F
:40C50000087005E0BE48007D012801D1BE49087070BD10B50446BD48D0F82C112046DFF8F0C200DF10BD01B500BF02226946B948006800F28230FDF797F820B9BDF800005A
:40C54000AE49A1F8820300BF3420F0F719FE08BD01B500BF02226946AE48006800F56070FDF782F820B9BDF80000A449A1F8800300BF3320F0F704FE08BD13B50C4640F650
:40C58000C410FFF7E5FF4FF47A50FFF7CCFF00BF012269469F48006800F5DE70FDF764F820B99DF80000954981F8BC0100BF14B10120FFF7AEFF2D20F0F7E2FD1CBD10B511
:40C5C00004469548007820B18C4890F8BC01A07005E00020A070A0780021FFF7CEFF012060702070FFF7A2F82D20F0F7C9FD10BD08B50321854880F83011DFF820C200DFBA
:40C60000064631460120DFF808C200DF17F002FF20B101218248007817F03EFF00BF002214210120DFF8FCC100DF85B2012D0AD0DFF8F4C100DF044604F0010098B168468B
:40C64000FFF7BDFF0FE0FEF7B8FD6846FFF71DFF6846FFF729FEFFF741FDFFF7F9FCFFF7D0FCFFF7A3FC2B20F0F78AFD2C20F0F787FD2A20F0F784FD4820F0F781FDCEE7CA
:40C680006A48007D70476A48007D70476948407D70476948407D70475948407D704710B517F0B8FE08B1022405E017F0CBFE08B1012400E00024204610BD10B517F0AAFEB0
:40C6C00010B917F0BFFE08B1012400E00024204610BD7047704710B5029C10BD2DE9F04105460C4617469846069EB5F56F4F0DD12078B1280AD16078362807D1A078012856
:40C7000004D1822201214D480AF029FE4FF6467085420FD1207868B96078042805D18222012146480AF01BFE04E00022114643480AF015FEBDE8F0812DE9F04104460D461D
:40C7400017469846069E4FF6B07084420FD1A87800F01000102805D18222012137480AF0FEFD04E00022114634480AF0F8FDBDE8F0812DE9F04106460C4617469846069DC6
:40C78000607800F003002E4908706078032101EAA0002B4948706078032101EA2010284988706078032101EAA0102549C870A078888008468088E1784FF47F4202EA01216E
:40C7C00008431F498880207900F0030088712079032101EAA0001A49C8712079032101EA201017490872A0794872E0798872084641780022114825E0A5060020081F0020A4
:40C8000028280020AC280020B4030020F03F002081F30308A4030020A2030020C1FF0308BD060020E1F3030829F3030858280020702800204028002010280020A02800208F
:40C84000C42800200AF08BFD4C48C17900224C480AF085FDBDE8F0812DE9F84305460E4617469846089C474991F83000FAF763FC38B143463A46314628460094FFF779FFD3
:40C880001AE0404991F83000FAF75DFC38B143463A46314628460094FFF74EFF0CE0394991F83000FAF725FC30B143463A46314628460094FFF712FFBDE8F88310B5324842
:40C8C000007818F0EBF958B93048007818F0E6F930B92F48007818F0E1F908B9012000E000200446204610BD10B52648D0F8B4002449D1F89810401AB0F5B46F08D92148DA
:40C9000090F8BC0120B1F9F729FB08B9012010BD0020FCE710B501241E48007D58B941F658311D4800681AF038F910B9F9F716FB68B900240BE0FFF7D7FF20B1F9F70EFBE5
:40C9400008B9002403E01AF022F913490860204610BD01B500BF012269461048006800F28630FCF781FE20B99DF80000054981F8860300BF3220F0F703FC08BDC42800202C
:40C98000AC280020081F0020F2060020F9060020E306002028280020B8030020A4030020B5EEC00AF1EE10FA04DDF4EEE10AF1EE10FA09DAB5EEC00AF1EE10FA06D2F4EE0A
:40C9C000C10AF1EE10FA01D8012070470020FCE7FD480078704710B52DED028B0446B0EE408AB7EE000AF0EE408AFFF7F1FF80B3F8F7BBFD68BBF2EE0A0AB4EEE08AF1EE24
:40CA000010FA03DBDFEDF10AB0EE608AFDEEC80A10EE901A08B200EE900AF8EEE00A38EE600A04F1140101EB8001D1ED000AB7EE001A31EE401A60EE810A04F11401421C00
:40CA400001EB820191ED001A41EE000AF0EE608A00BFB0EE680ABDEC028B10BD70B52DED028B04460D46B7EE000AB0EE408AF8F77CFD40B9D64800EBC40000EB850090ED41
:40CA8000000AB0EE408AB0EE480ABDEC028B70BDD0ED000A91ED001A60EE810A90ED011AD1ED011A41EE210A90ED021AD1ED021A41EE210A90ED031A60EE810AB0EE600A66
:40CAC000704710B52DED068B04469FEDC20AF0EE409A94F8C200012804D194ED210A84ED220A87E004F1900104F14C00FFF7D0FFB0EE408AB64A4C3A92F8421092F8410098
:40CB0000FFF7ACFF20EE080AB0EE408A11F0EBF8B0EE40AA2046FFF75EFF20EE080AB0EE408AB5EEC08AF1EE10FA06DD94ED1B0A20EE080AB0EE408A05E094ED170A20EEA3
:40CB4000080AB0EE408A94F87C0001283AD194ED220A30EE080A84ED220A94ED220AD4ED180AB4EEE00AF1EE10FA43DD94ED220AD4ED1C0AB4EEE00AF1EE10FA3AD2B5EEA8
:40CB8000C08AF1EE10FA0ED294ED220AD4ED1C0A30EE600AB0EE408A94ED180A30EE080AB0EE408A26E094ED220AD4ED180A30EE600AB0EE408A94ED1C0A30EE080AB0EEA8
:40CBC000408A17E084ED228AB5EEC08AF1EE10FA08DD94ED220AD4ED1C0A30EE200A84ED220A07E094ED220AD4ED180A30EE200A84ED220A94ED220AD4ED1D0AB4EEE00AA6
:40CC0000F1EE10FA04DD94ED1D0A84ED220A0CE094ED220AD4ED190AB4EEE00AF1EE10FA03D294ED190A84ED220AA06819F0D7FF00EE100AB8EE409A94ED030A60EE098AFF
:40CC400094ED220AD4ED1C0AB4EEE00AF1EE10FA08DB94ED230AD4ED1C0AB4EEE00AF1EE10FA11D394ED220AD4ED180AB4EEE00AF1EE10FA14D894ED230AD4ED180AB4EEB6
:40CC8000E00AF1EE10FA0BDD94ED180AB0EEC00AD4ED1C0A30EE200A30EE280AF0EE408A94ED220AD4ED230A30EE600AB4EEE80AF1EE10FA06DD94ED230A30EE280A84ED95
:40CCC000220A12E094ED220AD4ED230A30EE600AF1EE680AB4EEE00AF1EE10FA05D294ED230A30EE680A84ED220A19F050FFA06094ED220A84ED230A35484C3890F830001F
:40CD00000A2806D1FAF70DFB18B1B7EE000AF0EE409AF9F795F9B8B1F5EEC09AF1EE10FA1ED094ED1E2AF0EE421A94ED1A2AB0EE421A94ED202AF0EE420A94ED232AB0EEA3
:40CD4000420AFFF72DFE58B1F8F715FD102807D09FED200A84ED220A9FED1E0A84ED230A0120BDEC068B10BD70B52DED088B05460C46B0EE408A94ED010AD4ED000A30EE14
:40CD8000600A84ED040A18EE100A23F0DFFF41EC190B94ED040A10EE101A084623F0D6FF41EC1B0BB0EE4B0AF0EE6B0A20F0A8FBB0EE40AAF0EE60AA53EC192B51EC1A0B9A
:40CDC00023F092FC0CD207E0D80300200AD74F41541F0020000000001FED020A84ED040A94ED040AD5ED040A30EE600A84ED060A94ED070A10EE101A084623F0A7FF41ECE1
:40CE0000190B94ED060A10EE101A084623F09EFF41EC1B0BB0EE4B0AF0EE6B0A20F070FBB0EE40AAF0EE60AA53EC192B51EC1A0B23F094FD04D21FED190A84ED050A12E093
:40CE4000F9F7FEF878B194ED040AD5ED040A30EE200AF0EE000AC0EE208A94ED050A30EE280A84ED050ABDEC088B70BDFD4A92F8281092F83020702A38D19FEDFB0A80ED6F
:40CE8000030A9FEDFA0A80ED040A9FEDF90A80ED050A9FEDF80A80ED060A9FEDF70A80ED070A9FEDF60A80ED080A9FEDF50A80ED090A9FEDF40A80ED0A0A9FEDF30A80ED22
:40CEC0000B0A9FEDF20A80ED0C0A9FEDF10A80ED0D0A9FEDF00A80ED0E0A9FEDEF0A80ED0F0AB7EE000A80ED100A0AE3DD4A92F830200A2A38D19FEDDF0A80ED030A9FED15
:40CF0000E70A80ED040A9FEDE60A80ED050AB6EE080A80ED060A9FEDDC0A80ED070A9FEDE10A80ED080A9FEDE00A80ED090A9FEDDF0A80ED0A0AB7EE000A80ED0B0A9FEDCB
:40CF4000DC0A80ED0C0A9FEDDB0A80ED0D0A9FEDDA0A80ED0E0A9FEDD90A80ED0F0AB7EE040A80ED100ACCE2BE4A92F84A20032A7CD10E297CD2DFE801F07B077C7B407F96
:40CF800080817B7B7B7B7E7D9FEDBA0A80ED030A9FEDC20A80ED040A9FEDC10A80ED050AB6EE080A80ED060A9FEDB70A80ED070A9FEDBC0A80ED080A9FEDBB0A80ED090A79
:40CFC0009FEDBA0A80ED0A0AB7EE000A80ED0B0A9FEDB70A80ED0C0A9FEDB60A80ED0D0A9FEDB50A80ED0E0A9FEDB40A80ED0F0AB7EE040A80ED100A79E09FEDB10A80EDA8
:40D00000030A9FEDB00A80ED040A9FEDAF0A80ED050A9FEDAE0A80ED060A9FEDAD0A80ED070A9FEDAC0A80ED080A9FEDAB0A80ED090A9FEDAA0A80ED0A0A9FEDA90A80EDF0
:40D040000B0A9FEDA80A80ED0C0A9FEDA70A80ED0D0A9FEDA60A80ED0E0A9FEDA50A80ED0F0A9FEDA40A80ED100A40E040E0FFE700BF00BF00BF00BF00BF00BFB7EE000A87
:40D0800080ED030AB7EE000A80ED040AB7EE000A80ED050AB7EE000A80ED060AB7EE000A80ED070AB7EE000A80ED080AB7EE000A80ED090AB7EE000A80ED0A0AB7EE000A0C
:40D0C00080ED0B0AB7EE000A80ED0C0AB7EE000A80ED0D0AB7EE000A80ED0E0AB7EE000A80ED0F0AB7EE000A80ED100A00BF08E20E297AD2DFE801F079077A40B4B3B2B1C2
:40D1000079797979B0AFB6EE000A80ED030A9FED660A80ED040AB7EE040A80ED050A9FED760A80ED060AB0EE000A80ED070AB0EE020A80ED080A9FED710A80ED090A9FEDF3
:40D14000700A80ED0A0A9FED6F0A80ED0B0A9FED6D0A80ED0C0A9FED6B0A80ED0D0A9FED690A80ED0E0A9FED670A80ED0F0A9FED650A80ED100AC3E19FED630A80ED030A82
:40D180009FED620A80ED040A9FED610A80ED050A9FED600A80ED060A9FED5F0A80ED070A9FED390A80ED080A9FED5C0A80ED090A9FED400A80ED0A0AB7EE040A80ED0B0A57
:40D1C0009FED570A80ED0C0AB7EE080A80ED0D0A9FED490A80ED0E0A9FED520A80ED0F0AB0EE000A80ED100A8AE14DE19FED480A80ED030A9FED460A80ED040A9FED440A61
:40D2000080ED050A9FED430A80ED060A9FED420A80ED070A9FED1C0A80ED080A9FED3F0A80ED090A9FED230A80ED0A0AB7EE040A80ED0B0A9FED3A0A80ED0C0AB7EE080AC7
:40D2400080ED0D0A9FED2C0A80ED0E0A9FED2A0A80ED0F0A68E06CE0A4E018E116E114E1D9E00000081F00208FC2F53EB81E053F295C0F3F9A99193F0AD7233F7B142E3F65
:40D28000EC51383F5C8F423FCDCC4C3F3D0A573FAE47613F1F856B3F8FC2753F6666263F3333333F9A99593F6666663F3333733F6666863FCDCC8C3F3333933F9A99993FD0
:40D2C000A69B443D6F12833D6F12033EF4FD543E6F12833E96438B3EBC74933EE3A59B3E0AD7A33E3108AC3E5839B43E7F6ABC3EA69BC43ECDCCCC3E3333D33FCDCC1C4002
:40D300000AD7234066662640CDCCCC3DCDCC4C3E9A99993E7B14EE3EAE47213F48E17A3F3333B33F6666E63F1FED0D0A80ED100AE6E01FED2B0A80ED030A1FED2D0A80ED92
:40D34000040A1FED2F0A80ED050A9FEDF70A80ED060A1FED330A80ED070A1FED350A80ED080A1FED370A80ED090A1FED310A80ED0A0AB7EE000A80ED0B0A1FED320A80EDC8
:40D380000C0A1FED330A80ED0D0A1FED340A80ED0E0A1FED360A80ED0F0A1FED380A80ED100AADE01FED4D0A80ED030A9FEDDF0A80ED040A9FEDDE0A80ED050A9FEDDD0A57
:40D3C00080ED060A9FEDDC0A80ED070A9FEDDB0A80ED080A9FEDDA0A80ED090A9FEDD90A80ED0A0A9FEDD80A80ED0B0A9FEDD70A80ED0C0A9FEDD60A80ED0D0A9FEDD50AB5
:40D4000080ED0E0A9FEDD40A80ED0F0A9FEDD30A80ED100A74E09FEDD20A80ED030A1FED6E0A80ED040A9FEDCF0A80ED050A1FED620A80ED060A1FED610A80ED070AB7EEE2
:40D44000040A80ED080A9FEDC80A80ED090A9FEDC60A80ED0A0A9FEDC40A80ED0B0A9FEDC20A80ED0C0A9FEDC00A80ED0D0A9FEDBE0A80ED0E0A9FEDBC0A80ED0F0A9FED96
:40D48000BA0A80ED100A3BE000BF00BF00BFB7EE000A80ED030AB7EE000A80ED040AB7EE000A80ED050AB7EE000A80ED060AB7EE000A80ED070AB7EE000A80ED080AB7EE1F
:40D4C000000A80ED090AB7EE000A80ED0A0AB7EE000A80ED0B0AB7EE000A80ED0C0AB7EE000A80ED0D0AB7EE000A80ED0E0AB7EE000A80ED0F0AB7EE000A80ED100A00BF7E
:40D5000000BF704799490870704710B50446984890F842106830405C00EE100AB8EE400ADFED940A80EE201A84ED151A904890F842106C3000EB810090ED000A84ED160AEB
:40D540008B4890F842107C3000EB810090ED000A84ED170AF9F7D7FE20B19FED870A84ED180A13E016F056FF40B106F0EBF95FEDB30A20EE200A84ED180A07E006F0E2F9E2
:40D580005FEDB60A20EE200A84ED180A784890F842106A30405C00EE100AB8EE400ADFED750A80EE201A84ED191A714890F84210743000EB810090ED000A84ED1A0A6C48C2
:40D5C00090F84210843000EB810090ED000A84ED1B0AF9F798FE20B19FED660A84ED1C0A13E016F017FF40B106F0EAF95FEDD30A20EE200A84ED1C0A07E006F0E1F95FED56
:40D60000D50A20EE200A84ED1C0A594890F841105C3000EB4100564991F84210405C00EE100AB8EE400ADFED530A80EE201A84ED111A4F4890F84110603000EB41004C49CE
:40D6400091F84210405C00EE100AB8EE400ADFED490A80EE201A84ED121A454890F84110643000EB4100424991F84210405C00EE100AB8EE400ADFED3F0A80EE201A84ED89
:40D68000131AF9F718FE50B1394890F830000A2800D004E09FED390A84ED140A0EE0F9F732FE38B116F0E1FE20B1B1EE040A84ED140A03E09FED320A84ED140A2C4890EDA5
:40D6C0007E0A84ED010A9FED2F0A84ED020A0120FFF718FF264890F82800072806D116F0B1FE18B1012084F8740002E0002084F874002046FFF7BAFB0A20EFF741FD0B2087
:40D70000EFF73EFD0C20EFF73BFD0E20EFF738FD0D20EFF735FD1120EFF732FD1020EFF72FFD012010BD00007B144E3F3789213F4C37293FE926313F8716393F2506413F14
:40D7400039B4483FD7A3503F7593583F8941603F2731683FC520703FD9CE773F77BE7F3F3333B33ED7A3303F6666A63FD8030020081F00200000C8420000C8C20000FA433D
:40D7800000C05A45000000002DED028B3026FE48FE490860001DFE490860001DFD4908600C38FD4908603430FC490860401CFC490860B938FB490860FFF7A7FEFA4890F873
:40D7C0002800F14990390870F74890ED0F0A084680ED010A9FEDF50A80ED270A90ED1E0AF34880ED1C0A084690ED1A0AF04880ED1D0ADFF8C0C300DFDFF8BCC300DF804660
:40D800003022012119F0CDFADFF8ACC300DF8046012119F0F5FA0321E84880F8401000BF002231464CF20300DFF894C300DF0446012C17D100BFE14890F8410040F001019B
:40D84000DE4880F84110B0F84C004FF6FF71884207DADA48B0F84C00401C81B2D748A0F84C10DDE7022CDBD1DFF858C300DF054605F0020038B3C4488838FFF746FECA48F9
:40D8800090F82800C04990390870C74890ED0F0A084680ED010A1021C548DFF82CC300DF012810D0B848903890ED1E0AC04880ED1C0AB548903890ED1A0ABD4880ED1D0A10
:40D8C000DFF808C300DF05F001000028A8D01021B748DFF8F4C200DF01287DD02022AA49103901F120001EF050FC19F050F90746A548903890F8C00007286ED2DFE800F053
:40D90000049EA4B5CCE1F300A94890F84100012812D1A748816B384619F070F9FA280BD203209949903981F8C000012081F8C100002081F8C20080E003F02CFCD0B1F8F714
:40D940000DFBB8B19A4890F85900012812D19848016D384619F052F9FA280BD205208A49903981F8C000012081F8C100002081F8C20062E003F00EFCD0B1F8F7EFFAB8B197
:40D980008B4890F86500012812D18948C16D384619F034F9FA280BD206207B49903981F8C000012081F8C100002081F8C20044E003F0F0FBE0B1F8F7D1FAC8B17C4890F835
:40D9C0004D00012814D17A48416C384619F016F9FA280DD2042001E0BDE095E06A49903981F8C000012081F8C10081F8C20024E003F0D0FBD0B1F8F7B1FAB8B16C4890F8E2
:40DA00003500012812D16A48C16A384619F0F6F8FA280BD202205C49903981F8C000012081F8C100002081F8C20006E000205649903981F8C10081F8C2006BE000205249EC
:40DA4000903981F8C00065E0F8F788FA28B101204D49903981F8C10006E000204A49903981F8C10081F8C00054E0514890F8410030B14F48816B384619F0C0F8FA2805D94D
:40DA800000204149903981F8C00004E001203E49903981F8C1003DE0F8F760FA38B101203949903981F8C10081F8C20008E000203549903981F8C10081F8C20081F8C000FE
:40DAC00028E0F8F74BFA28B101202F49903981F8C10006E000202C49903981F8C10081F8C00017E0FFE7F8F739FA28B101202649903981F8C10006E000202349903981F89F
:40DB0000C10081F8C00005E000201F49903981F8C10000BF00BF1C48903890F8C10080B11948903890F8C00000EB40012048143000EB810090ED010A1348903880ED210A5F
:40DB400005E01FEDF00A1048903880ED210A1848DFF878C000DF0C48903890F8C10001287ED1F9F7A8FB98B305F0C7FE104880ED040A05499039087891ED011AF0EE410A13
:40DB80000B4991ED041A24E0D8290020C0030020C4030020C8030020CC030020D0030020D4030020DC030020081F002099A0063CD028002055F70308C1FF0308F03F002078
:40DBC000E1F3030829F3030849F8030865F7030816E0B0EE410A05F0A7FDFE4880ED200A0146087891ED011AF0EE410A91ED211AB0EE410A05F098FDF64880ED210A3BE071
:40DC0000F9F781FB28B1F7F7AEFFF24880ED200A32E0F9F76FFB38B305F06FFEEE4880ED040A10F05CF8B0EE408AEB48D0ED040AB0EE600AF0EE480A05F034FEE54880ED16
:40DC4000200A10F04CF8B0EE408AE248D0ED210AB0EE600AF0EE480A05F024FEDD4800E028E080ED210A07E0F9F786FB20B106F0AAF9D84880ED200AD648D0ED040AB0EEC8
:40DC8000600A00F18001A030FFF76EF8D148FEF718FF50B1CF4890ED230ACF4880ED1A0A0120CD4981F86C000DE00020CA4981F86C0008E09FEDC90AC74880ED1A0A0020A5
:40DCC000C54981F86C003F20EFF75AFA5020EFF757FAA5E510B5C248C16B012019F0CAF8BF48C16B0120DFF8FCC200DF10BD10B5BB48C16B012019F0DBF80446204610BD7D
:40DD000070B52DED028BB0EE408A04460D460026012C04D0022C03D0032C61D101E000BF00BFAD4890ED1D0AB4EEC80AF1EE10FA05DD90ED1D0AB0EE408A03260CE0A64843
:40DD400090ED1C0AB4EEC80AF1EE10FA04D290ED1C0AB0EE408A022610219F48DFF888C200DF01283AD004EB44019B48143000EB810080ED018A16F078FB98B104EB44019A
:40DD80009548143000EB810090ED010AFFEE000A20EE200A04EB44018F48143000EB810080ED010A18F0F3FE04EB44028A49143141F82200012104EB44028748143000EBF6
:40DDC0008200017204EB44018348143000EB810045728148DFF814C200DF00E0062601E0062600BF00BF3046BDEC028B70BD70B52DED028BB0EE408A04460D460026012CDF
:40DE000004D0032C03D0042C47D100BF00BF9FED780AB4EEC08AF1EE10FA05D29FED740AB0EE408A03260BE09FED720AB4EEC08AF1EE10FA04DD9FED6F0AB0EE408A0226B3
:40DE400010216548DFF8A0C100DF012823D004EB44016148143000EB810080ED018A18F096FE04EB44025C49143141F82200012104EB44025848143000EB8200017204EBEC
:40DE800044015548143000EB810045725248DFF85CC100DF00E0062601E0062600BF00BF3046BDEC028B70BD70B52DED028BB0EE408A04460D460026012C04D0032C03D042
:40DEC000052C47D100BF00BF9FED490AB4EEC08AF1EE10FA05D29FED460AB0EE408A03260BE09FED440AB4EEC08AF1EE10FA04DD9FED400AB0EE408A022610213648DFF8FC
:40DF0000E8C000DF012823D004EB44013248143000EB810080ED018A18F039FE04EB44022D49143141F82200012104EB44022A48143000EB8200017204EB4401264814308B
:40DF400000EB810045722448DFF8A0C000DF00E0062601E0062600BF00BF3046BDEC028B70BD70B52DED028BB0EE408A04460D460026012C04D0032C03D0062C6AD100BF66
:40DF800000BF05F084FF00EE100AB8EE400AB4EEC80AF1EE10FA09DD05F079FF00EE100AB8EE400AB0EE408A032626E005F06BFF00EE100AB8EE400AB4EEC80AF1EE10FA3F
:40DFC0001BD205F060FF00EE100AB8EE400AB0EE408A11E048290020D028002000000000F03F002081F3030849F8030865F703080000C8C20000C84202261021FE48DFF85B
:40E00000FCC300DF012823D004EB4401FA48143000EB810080ED018A18F0B9FD04EB4402F549143141F82200012104EB4402F248143000EB8200017204EB4401EE481430D4
:40E0400000EB81004572EC48DFF8B4C300DF00E0062601E0062600BF00BF3046BDEC028B70BDE54890ED1A0A7047E34890F86C007047E44890ED210A7047E24890ED200AF5
:40E08000704773B52DED020B04460D4600269DED000ADFEDDD0AB4EEE00AF1EE10FA05DD02269FEDD90A8DED000A0DE09DED000ADFEDD60AB4EEE00AF1EE10FA04D203263D
:40E0C0009FEDD20A8DED000A00BFD14909684C3101EBC40101EB850004226946FBF7C4FA40B99DED000ACB4800EBC40000EB850080ED000A00BFC7484C3890F84200A8428A
:40E100000BD1C4484C3890F84100A04205D1C248C16B0220DFF804C300DF1620EFF730F8304604B070BDF7B50C46154600269DF80000FF2803DD0226FF20009006E09DF815
:40E140000000012802DC03260120009000BFB04909685C3101EB4401481901226946FBF783FA30B99DF80010AA48103000EB4400415500BFA7484C3890F84200A8420BD1EE
:40E18000A4484C3890F84100A04205D1A248C16B0220DFF888C200DF0A20EEF7F1FF3046FEBDF7B50C46154600269DF80000FF2803DD0226FF20009006E09DF80000002871
:40E1C00002DC03260020009000BF91490968603101EB4401481901226946FBF745FA30B99DF800108B48143000EB4400415500BF88484C3890F84200A8420BD185484C38DA
:40E2000090F84100A04205D18348C16B0220DFF80CC200DF0B20EEF7B3FF3046FEBDF7B50C46154600269DF80000FF2803DD0226FF20009006E09DF80000002802DC032631
:40E240000020009000BF72490968643101EB4401481901226946FBF707FA30B99DF800106C48183000EB4400415500BF69484C3890F84200A8420BD166484C3890F8410049
:40E28000A04205D16448C16B0220DFF890C100DF0C20EEF775FF3046FEBD73B50C4600259DF80000FF2803DD0225FF20009006E09DF80000012802DA03250120009000BFC6
:40E2C000534909686831081901226946FBF7CCF920B99DF800104F481C30015500BF4D484C3890F84200A04205D14B48C16B0220DFF828C100DF0F20EEF742FF28467CBD41
:40E3000073B50C4600259DF80000FF2803DD0225FF20009006E09DF80000012802DA03250120009000BF3A4909686A31081901226946FBF799F920B99DF8001035481E3065
:40E34000015500BF33484C3890F84200A04205D13148C16B0220DFF8C4C000DF1220EEF70FFF28467CBD31B52DED020B0446002528484C3890F842107C3000EB810090ED5B
:40E38000000ADDED000AB4EEE00AF1EE10FA0CDD20484C3890F842107C3000EB810090ED000A8DED000A02250DE09DED000ADFED1C0AB4EEE00AF1EE10FA04DD9FED180A9A
:40E3C0008DED000A032500BF114909686C3101EB840004226946FBF747F938B99DED000A0C48203000EB840080ED000A00BF09484C3890F8420015E0D028002049F803080D
:40E4000065F7030848290020333323400AD7233CA4030020541F0020F03F002081F3030800000080A0420BD1FC48C16B0220DFF8F0C300DFF948016D0120DFF8E4C300DF4D
:40E440004E20EEF79DFE0E20EEF79AFE28463EBD31B52DED020B044600259DED000AB5EEC00AF1EE10FA05D29FEDEE0A8DED000A032519E0EC4890F84210843000EB810006
